:100000000C94DF060C9423070C9423070C9423070D
:100010000C9423070C9423070C9423070C942307B8
:100020000C9423070C940E170C9423070C942307AD
:100030000C94BB340C9423070C9423070C942307D3
:100040000C9423070C9423070C9483150C9423071A
:100050000C94530C0C9423070C941D0C0C94230744
:100060000C94231C0C9423070C945F300C942307EE
:100070000C945B770C9423070C9457724E1C531C02
:10008000581C611C781C8F1C9F1CAF1CCC1CB81EFC
:100090008F1C7A1D8B1DBA1DD81DF51D4F1EAA1E63
:1000A00088201A21D7215722C02270237B25D825EA
:1000B00045268F26DA2627277827D2273128CB28EE
:1000C0006629602A8730AE30F13061317931BA313A
:1000D0006D322D332D332D332D332D332D332D33E1
:1000E0002D332D332D332D33E432E632EB3203330F
:1000F00005330A0D426174743A002025642043657B
:100100006C6C732000204C6F77207761726E696E83
:1001100067206C6576656C3A2025642E2564000A9C
:100120000D466F756E6420424C2D4374726C3A20FC
:10013000002564000A0D0A0D2121204D4953534921
:100140004E4720424C2D4354524C3A2025642021E6
:1001500021000A0D3D3D3D3D3D3D3D3D3D3D3D3D8B
:100160003D3D3D3D3D3D3D3D3D3D3D3D3D3D3D3DBF
:100170003D3D3D3D3D3D3D000A0D43616C69627270
:100180006174696E67207072657373757265207330
:10019000656E736F722E2E004F4B0A0D000A0D46CE
:1001A0006C696768742D74696D65202575206D69AB
:1001B0006E2020546F74616C3A2575206D696E0055
:1001C0000A0D436F6E74726F6C3A2000486561646B
:1001D000696E67486F6C64004E6F726D616C2028A9
:1001E0004143432D4D6F646529000A0D3D3D3D3D62
:1001F0003D3D3D3D3D3D3D3D3D3D3D3D3D3D3D3D2F
:100200003D3D3D3D3D3D3D3D3D3D3D3D3D3D3D0A51
:100210000D00416E676C654E69636B2020202020C5
:100220002020416E676C65526F6C6C20202020206E
:1002300020204163634E69636B2020202020202012
:100240002020416363526F6C6C20202020202020EE
:1002500020205961774779726F20202020202020AC
:1002600020204865696768742056616C7565202098
:1002700020204163635A202020202020202020209D
:1002800020204761732020202020202020202020B3
:100290002020436F6D706173732056616C7565200B
:1002A0002020566F6C74616765205B302E31565D7F
:1002B00020205265636569766572204C6576656CB1
:1002C00020204779726F20436F6D70617373202017
:1002D00020204D6F746F722031202020202020209C
:1002E00020204D6F746F722032202020202020208B
:1002F00020204D6F746F722033202020202020207A
:1003000020204D6F746F7220342020202020202068
:1003100020203136202020202020202020202020B6
:1003200020203137202020202020202020202020A5
:100330002020313820202020202020202020202094
:100340002020313920202020202020202020202083
:100350002020536572766F2020202020202020202E
:100360002020486F7665726761732020202020204E
:10037000202043757272656E74205B302E31415DB2
:1003800020204361706163697479205B6D41685D11
:100390002020323420202020202020202020202037
:1003A0002020323520202020202020202020202026
:1003B0002020323620202020202020202020202015
:1003C0002020323720202020202020202020202004
:1003D00020204932432D4572726F72202020202048
:1003E0002020424C204C696D697420202020202060
:1003F00020204750535F4E69636B2020202020202F
:1004000020204750535F526F6C6C2020202020200A
:10041000202021212120494E434F4D504154494233
:100420004C4520212121002E000A0D20444143206B
:100430006F7220493243204552524F522120436867
:1004400065636B204932432C2033567265662C203D
:1004500044414320616E6420424C2D4374726C0011
:100460005B25695D005B25695D002B204D696B7222
:100470006F4B6F70746572202B0048573A56256495
:100480002E25642053573A25642E25642563005396
:10049000657474696E673A2564202573004861723B
:1004A0006477617265204572726F7220313A2564FB
:1004B000202121004D697373696E6720424C2D43E2
:1004C00074726C3A25642121004D6978657220456B
:1004D00072726F722100493243204552524F5221AD
:1004E0002121004865696768743A20202535690034
:1004F000536574706F696E743A2535690050726582
:1005000073737572653A253569004F666673657455
:100510003A20202535690048656967687420636F53
:100520006E74726F6C0044495341424C454400481C
:10053000656967687420636F6E74726F6C004449FC
:100540005341424C4544006163742E2062656172E0
:10055000696E67004E69636B3A20202020202025B9
:10056000356900526F6C6C3A202020202020253500
:100570006900436F6D706173733A202020253569DF
:10058000004B313A25346920204B323A253469201A
:10059000004B333A25346920204B343A2534692006
:1005A000004B353A25346920204B363A25346920F2
:1005B000004B373A25346920204B383A25346920DE
:1005C000004E693A2534692020526F3A253469205B
:1005D0000047733A253469202047693A2534692059
:1005E0000050313A253469202050323A25346920B0
:1005F0000050333A253469202050343A253469209C
:10060000004779726F202D2053656E736F72004E14
:1006100069636B25346920282533692E25692900F3
:10062000526F6C6C25346920282533692E25692981
:100630000047696572253469202825336929004EF1
:1006400069636B2025346920282533692E25782994
:1006500000526F6C6C2025346920282533692E25C3
:1006600078290059617720202534692028253369AD
:1006700029004E69636B20253469202825336929B8
:10068000282533692900526F6C6C20253469202895
:1006900025336929282533692900596177202025C8
:1006A00034692028253369292825336929004143E5
:1006B00043202D2053656E736F72004E69636B206B
:1006C00025346920282533692900526F6C6C202558
:1006D0003469202825336929005A20202020253418
:1006E0006920282533692900566F6C746167653A63
:1006F0002020202533692E253169560043757272FA
:10070000656E743A2020202533692E253169410019
:10071000506F7765723A20202020202534695700D9
:100720004469736368617267653A202535696D4174
:10073000680052656365697665720052432D5253B5
:1007400053493A202020202534690052432D517509
:10075000616C6974793A202534690052432D4368ED
:10076000616E6E656C733A25346900436F6D70611C
:1007700073730048656164696E673A2020253569A6
:100780000056616C75653A2020202025356900539C
:10079000746172743A2020202025356900506F74EE
:1007A00069313A202025336900506F7469323A204C
:1007B0002025336900506F7469333A20202533694E
:1007C00000506F7469343A202025336900506F74EB
:1007D00069353A202025336900506F7469363A2014
:1007E0002025336900506F7469373A20202533691A
:1007F00000506F7469383A202025336900536572C0
:10080000766F202000536574706F696E7420202508
:10081000336900506F736974696F6E3A20253369CC
:100820000052616E67653A2533692D2533690045AD
:10083000787465726E436F6E74726F6C2020004E18
:10084000693A2534692020526F3A253469200047DF
:10085000733A253469202047693A253469200048D5
:10086000693A253469202043663A253469200042DC
:100870004C2D4374726C204572726F727320002588
:10088000336420253364202533642025336420001D
:1008900025336420253364202533642025336420E8
:1008A00000253364202533642025336420253364F8
:1008B0002000424C2054656D7065726174757265DC
:1008C00000253369202533692025336920253369C4
:1008D00020002533692025336920253369202533FD
:1008E00069200025336920253369202533692025B7
:1008F00033692000424C2D4374726C20666F756E14
:1009000064200020256320202025632020202563EB
:10091000202020256320002025632020202563201F
:10092000202025632020202563200020256320200F
:10093000202D2020202D2020202D2000313000319E
:100940003100313200466C696768742D54696D65F9
:10095000202000546F74616C3A2535756D696E0006
:100960004163743A20202535756D696E00287265E3
:1009700073657429000A0D47656E65726174696E4E
:10098000672064656661756C7420506172616D6585
:1009900074657220536574202564000A0D557369CF
:1009A0006E6720506172616D657465722053657465
:1009B000202564000A0D47656E65726174696E6773
:1009C0002064656661756C74204D69786572205489
:1009D00061626C65000A0D4D697865722D436F6E1A
:1009E0006669673A202725732720282575204D6FD3
:1009F000746F727329000A0D3D3D3D3D3D3D3D3D07
:100A00003D3D3D3D3D3D3D3D3D3D3D3D3D3D3D3D16
:100A10003D3D3D3D3D3D000A0D414343206E6F7419
:100A20002063616C69627261746564210D0A000A59
:100A30000D506C6561736520636F6E6E6563742025
:100A40005370656B7472756D207265636569766548
:100A50007220666F722062696E64696E67204E4F05
:100A6000572E2E2E006F6B2E0A0D0054696D656F88
:100A700075742E0A0D0000008F001E01AD013B02AF
:100A8000CA025803E603740402058F051B06A70675
:100A90003307BE074808D2085B09E3096B0AF20A6C
:100AA000780BFD0B810C040D860D070E870E060FCB
:100AB000840F00107B10F5106E11E5115B12CF1240
:100AC0004213B31323149214FE146A15D3153B1664
:100AD000A11605176717C81727188318DE183719C6
:100AE0008E19E319361A871AD61A231B6E1BB61BEA
:100AF000FD1B411C831CC31C001D3C1D751DAB1D33
:100B0000E01D121E421E6F1E9A1EC31EE91E0D1FFF
:100B10002E1F4D1F691F841F9B1FB01FC31FD31F94
:100B2000E11FEC1FF51FFB1FFF1F0020030100004A
:100B3000AF6B00020101A26C01030202366D0200DC
:100B40000303936D2532692E2531695600253364E0
:100B5000256320253033646D005374617475730010
:100B60004552524F523A20253264002534692025DF
:100B700032693A25303269002534696D25630025D4
:100B80003369202533692025336920253369002501
:100B900033692025336920253369202533690054C2
:100BA000656D706572617475726573202020200018
:100BB0002563432020202020002532692E2531691D
:100BC0005620202533692E25316941002534695787
:100BD000202536696D4168002532756D2F732053CD
:100BE00061743A2564200020203344004E6F46781B
:100BF000004447505300486F6D653A2533646D20BB
:100C00002533642563004E6F204E6176694374720C
:100C10006C21000A0D7777772E4D696B726F4B6FE1
:100C2000707465722E6465202863292048695379A1
:100C30007374656D7320476D6248000A0D746865B2
:100C400020757365206F66207468697320736F6602
:100C50007477617265206973206F6E6C792070659E
:100C6000726D6974746564200A0D6F6E206F72690D
:100C700067696E616C204D696B726F4B6F70746544
:100C8000722D48617264776172650041435420445B
:100C9000534C004A65746920736174656C6C6974A7
:100CA000005370656B7472756D20736174656C6C44
:100CB000697420284C6F77207265736F6C75746946
:100CC0006F6E29005370656B7472756D207361745B
:100CD000656C6C6974202832303438290053706593
:100CE0006B7472756D20736174656C6C6974004D02
:100CF000756C74697369676E616C2050504D000AA1
:100D00000D52656365697665723A2000756E6B6E8B
:100D10006F776E2E205573696E672050504D2E2EC2
:100D20002E006E6F7420737570706F72746564201E
:100D3000627920686172647761726521000A0D3DF5
:100D40003D3D3D3D3D3D3D3D3D3D3D3D3D3D3D3DD3
:100D50003D3D3D3D3D3D3D3D3D3D3D3D3D3D3D3DC3
:100D60003D3D000A0D466C69676874436F6E74728E
:100D70006F6C0A0D48617264776172653A25642E62
:100D800025640A0D536F6674776172653A5625645F
:100D90002E2564256320000A0D3D3D3D3D3D3D3D32
:100DA0003D3D3D3D3D3D3D3D3D3D3D3D3D3D3D3D73
:100DB0003D3D3D3D3D3D3D3D3D3D3D3D0000112422
:100DC0001FBECFEFD0E1DEBFCDBF11E0A0E0B1E0AC
:100DD000E4EBF2EF02C005900D92A63FB107D9F700
:100DE00018E0A6EFB1E001C01D92A03AB107E1F70B
:100DF0006AEAE2E0F0E081E2809357007491AE018C
:100E00004F5F5F4F20EF37EFDA019FE0F9012F5F6F
:100E10003F4F84918D93915097FFF8CF773911F41C
:100E20000000FECFFA019EE0819168276095915005
:100E300097FFFACF8889681721F0773911F40000FD
:100E4000FECF0C94E4070C94000080910806E82F74
:100E5000FF27EE0FFF1FE15DF84F808191818D5ECE
:100E60009F4F14F010920301808191818A5B9F4F04
:100E7000CCF4809103018823A9F481E080930301DD
:100E800080915F048F5F80935F04853038F088EE37
:100E900093E0909326028093250204C066E970E0F7
:100EA0000E94253880915F0499279093D9058093FB
:100EB000D80508951F93CF93DF93182F882389F0C7
:100EC00082EF90E09F938F9387E692E19F938F93B9
:100ED000E0912B04F0912C0409950F900F900F9046
:100EE0000F9080912B06823308F044C084EF91E08C
:100EF0000E948E16EC01112329F0CE010E94971654
:100F00008823D9F3C2E0D0E026E530E080911D01CE
:100F100090911E018217930730F02196255D3F4F77
:100F2000C730D10598F380912B069927C89F90016F
:100F3000C99F300DD89F300D11242093000111233B
:100F4000D9F068EC70E08C2F0E942538DF93CF93A6
:100F50008AEF90E09F938F9387E692E19F938F9320
:100F6000E0912B04F0912C0409958DB79EB706965D
:100F70008DBF02C080930001112311F18091000107
:100F80006AE00E948578892F99279F938F9380919B
:100F900000010E94857899279F938F9385E091E0C7
:100FA0009F938F9387E692E19F938F93E0912B0419
:100FB000F0912C0409952DB73EB7285F3F4F2DBF08
:100FC000DF91CF911F910895CFEFD0E1DEBFCDBF6C
:100FD0008824992414B815B807EE13E00253104082
:100FE00017FFFCCF189B06C0199B02C08DE007C0FD
:100FF0008BE005C0199B02C084E101C08AE08093A8
:10100000020181E887B93E9A8FEF88B98BE184B9F4
:1010100081E085B98EE38AB987E48BB9469A84B7B3
:10102000877F84BF80916000886180936000109208
:10103000600084EC99E09093260280932502109240
:101040001A0310921903109234071092330710926A
:101050001C0310921B0310921E0310921D0320917B
:101060000201243128F084EC94E0A0E0B0E004C058
:101070008BE095E0A0E0B0E08093990190939A0115
:10108000A0939B01B0939C012A3011F0243110F001
:10109000289801C0289A0E94F7160E94C8160E943C
:1010A0006F120E949F340E94DC1A0E9416300E9428
:1010B000BA630E94826E0E948E76809102018C300B
:1010C00010F4299A01C0299878940E94352F8091B4
:1010D0006F02826080936F02109271020E948D43B2
:1010E00084EF91E00E948E168C0180916F0280FD4A
:1010F00005C0C8010E9497168823B9F38FE191E0DB
:101100009F938F93B7E6AB2EB2E1BB2EBF92AF9207
:10111000E0912B04F0912C04099580EA9FE00E9455
:101120008E168C01C0E0D0E00F900F900F900F90C2
:10113000A1EDEA2EA6E0FA2EF5E8CF2EF6E0DF2E9E
:101140000E948D4380916F0280FD05C0C8010E94FE
:1011500097168823B9F3F60180811816ACF40BC0FA
:101160000E948D4380916F0280FD05C0C8010E94DE
:1011700097168823B9F3C8010E949716882321F493
:10118000F7018081882364F7F701808187FF18C009
:101190002196DF93CF93219781E391E09F938F93E3
:1011A000BF92AF92E0912B04F0912C0409958091AD
:1011B000F6018F5F8093F6018DB79EB706968DBFBF
:1011C0002196E4E0F0E0CE0EDF1E88E090E0E80E2D
:1011D000F91ECC30D10508F4B3CFC0E0D0E00EEC5E
:1011E00016E0E5E8EE2EE6E0FE2EF801838187FDAD
:1011F0001CC0F70180811816C4F42196DF93CF93A9
:10120000219784E391E09F938F9387E692E19F93E8
:101210008F93E0912B04F0912C04099582E0809348
:1012200023028DB79EB706968DBFF8018381807823
:101230008383219684E090E0E80EF91E085F1F4F3B
:10124000CC30D10590F282E591E09F938F93C7E671
:10125000D2E1DF93CF93E0912B04F0912C04099518
:10126000909106068091F6010F900F900F900F90CD
:10127000981728F48091450480618093450488E79D
:1012800091E09F938F93DF93CF93E0912B04F091A4
:101290002C04099588EE93E00E948E168C010E9422
:1012A000E21A0F900F900F900F90C8010E949716AE
:1012B0008823D9F388E991E09F938F93DF93CF93AD
:1012C000E0912B04F0912C04099580E00E94E7380E
:1012D000809102010F900F900F900F908A3011F0C3
:1012E000843110F0289801C0289A80ED97E09093FF
:1012F00026028093250285E5809361048EE090E0CC
:101300000E94042E9927182F00278FE090E00E945A
:10131000042E080F111D1093FC010093FB018AE0BD
:1013200090E00E94042E9927182F00278BE090E070
:101330000E94042E080F111D1093FA010093F90169
:101340000F5F1F4F39F08091FB019091FC018F5F7F
:101350009F4F41F41092FC011092FB011092FA0190
:101360001092F9018091F9019091FA019F938F9366
:101370008091FB019091FC019F938F938DE991E007
:101380009F938F93DF93CF93E0912B04F0912C04E4
:1013900009958DB79EB708968DBF80EC91E09F931D
:1013A0008F93DF93CF93E0912B04F0912C04099558
:1013B000809114060F900F900F900F90E0912B04E6
:1013C000F0912C0482FF07C08CEC91E09F938F93E7
:1013D000DF93CF9308C088ED91E09F938F9387E6CA
:1013E00092E19F938F9309950F900F900F900F901C
:1013F0000E94FF1F88E893E19093920180939101EE
:1014000081E0809360040E945A0780912E060E941A
:10141000F4758AEE91E09F938F93DF93CF93E091E1
:101420002B04F0912C04099580ED97E00E948E1614
:101430008C018AEF90E00E948E16EC0183E080938D
:10144000B0050F900F900F900F90CE010E9497164D
:10145000882339F084E690E00E948E16EC010E9409
:101460004A7780912902882309F4DFC180910F0116
:10147000882309F4DAC11092290280915F0488233D
:1014800019F00E94250702C00E943C460E948D432D
:10149000209102012A3011F0243110F0289801C067
:1014A000289A80911F0390914504882339F08091F8
:1014B0001F03815080931F03977F0AC080916F00A4
:1014C000806280936F001092300710922F0798600F
:1014D000909345048091910190919201019790938E
:1014E0009201809391018091910190919201892BB9
:1014F00029F080917002882309F43EC08091910107
:1015000090919201892B01F50E943C3085E090E09A
:1015100090939201809391018091EA059091EB055F
:1015200001969093EB058093EA058091EB02806829
:101530008093EB0280914504816080934504809103
:10154000B10582608093B1058091080190910901F5
:101550008F5F9F4F19F5809116038823F9F080E182
:1015600097E2909326028093250280E890E0909382
:1015700009018093080112C02A3011F0243110F0C3
:10158000289801C0289A8091250290912602892BE3
:1015900029F48091EB028F778093EB0280912902EE
:1015A000882309F042C10E94B3120E94910EC80123
:1015B0000E949716882309F434C10C5E1F4F809156
:1015C000700290914504882339F09260909345040D
:1015D0008091B10582600CC09D7F909345048091FD
:1015E000910190919201079728F08091B1058D7F2C
:1015F0008093B1058091910190919201079728F015
:10160000809145048E7F8093450480910501882355
:1016100021F081508093050125C080936B041092C6
:10162000F7021092F6021092F5021092F402109254
:10163000F3021092F20280910801909109018F5FEC
:101640009F4F81F480911F03882361F488E99AE316
:10165000909326028093250280E09CE090930901FC
:10166000809308018091EC01893C70F08150809357
:10167000EC018091EB028F7B8093EB02809145041B
:101680008B7F8093450435C080910D08882309F134
:101690008091EB0280648093EB028091450484602A
:1016A0008093450480910801909109018F5F9F4FBD
:1016B00081F480911603882361F088E99AE390937E
:1016C00026028093250280E098EA90930901809396
:1016D00008011092FD031092FC031092FB0310927C
:1016E000FA038FEF9FEF90933B0880933A08109294
:1016F000EC0180910001282F332780911D019091EA
:101700001E0182179307CCF48091EB0280628093D4
:10171000EB0280910801909109018F5F9F4FC1F406
:1017200080E797E1909326028093250280E093E082
:1017300090930901809308010BC08091250290913C
:101740002602892B29F48091EB028F7D8093EB0296
:101750000E94B86784E08093240280911603882356
:1017600029F45AEA852E55E0952E12C08091FD018C
:101770008F5F8093FD01813359F41092FD018091B8
:10178000F7019091F80101969093F8018093F70189
:101790000894811C911CF2E78F16FBE09F0609F06C
:1017A00040C0882499242091FB013091FC012F5FD7
:1017B0003F4F3093FC012093FB018091F901909100
:1017C000FA0101969093FA018093F901832F9927EA
:1017D000682F8EE090E00E940A2E8091FB0190918C
:1017E000FC019070682F8FE090E00E940A2E80919B
:1017F000F9019091FA01892F9927682F8AE090E0EA
:101800000E940A2E8091F9019091FA019070682F40
:101810008BE090E00E940A2E84E190E00E948E16F8
:101820008C010E9408680E94996E8091240288238E
:1018300009F00BCE0E94DB6308CE1F920F920FB609
:101840000F9211248F939F93EF93FF938091070141
:101850008823E1F4809117029091180201969093E9
:10186000180280931702FC01E05FFA4FE081ED302F
:1018700019F0803A910539F410921802109217026B
:1018800081E080930701E093C60004C01092180223
:1018900010921702FF91EF919F918F910F900FBEC1
:1018A0000F901F9018951F920F920FB60F92112450
:1018B0002F933F934F935F936F937F938F939F9358
:1018C000AF93BF93CF93EF93FF9390E08091C600C7
:1018D00080930F0250911D02503A10F090931E0217
:1018E00080910F028D3009F065C080911E02823018
:1018F00009F060C090931E02852F992782599B4F53
:10190000FC01329740812091190230911A02241B68
:101910003109DC0111978C91281B3109C9019F7095
:1019200090931A028093190246E0969587954A95FE
:10193000E1F7982F935C90931B022F733070235C18
:1019400020931C028081981729F48C91281711F498
:1019500091E006C090E080910C028F5F80930C02B2
:10196000C0910E02CC2309F074C0992309F471C010
:1019700081E080930E02580F50930B025150E52FD7
:10198000FF27E259FB4F8DE0808380917004823500
:1019900009F05FC00E94FF1F88E190E02CE00FB6C5
:1019A000F894A895809360000FBE20936000C093C8
:1019B00023024FC020911E02822F9927813091056A
:1019C000F9F0823091051CF4892B21F040C0029778
:1019D00011F13DC080910F02833239F480910E02E3
:1019E000882319F481E080931E0280910F02809376
:1019F0006E0481E080931D0280910F02992722C01E
:101A00002F5F20931E02E52FFF27E259FB4F8091A5
:101A10000F02808309C0E52FFF27E259FB4F809119
:101A20000F028083503A20F45F5F50931D0202C082
:101A300010921E0220910F028091190290911A02B9
:101A4000820F911D90931A028093190202C0109286
:101A50001E02FF91EF91CF91BF91AF919F918F9116
:101A60007F916F915F914F913F912F910F900FBE9A
:101A70000F901F901895AC01A0E0B0E09D01A81751
:101A8000B90748F4E0E1F5E08191280F311D119686
:101A9000A417B507C8F33F70FD01E05FFA4FC90115
:101AA00056E0969587955A95E1F7835C8083119669
:101AB000FD01E05FFA4F2F733070822F835C8083CB
:101AC000AF5EBA4F8DE08C931092070180911005A4
:101AD0008093C6000895A0E0B0E0E1E7FDE00C943B
:101AE000FE782C859D850E85BB2483E280931005AE
:101AF0009F59909311052093120533E0E32EF12CAA
:101B0000002309F49EC0CF84D888BE016D5E7F4F4C
:101B1000A989BA890150109709F493C01097B9F0B8
:101B2000F601EB0DF11DB3949081119791F4002310
:101B300049F1FB016E5F7F4FDB01C080D1806E5F9A
:101B40007F4F0D90BC91A02DBB24015002C090E0AE
:101B500019C01097B9F0F601EB0DF11DB394408157
:101B6000119791F4002341F1FB016E5F7F4FDB0180
:101B7000C080D1806E5F7F4F0D90BC91A02DBB24A3
:101B8000015002C040E018C01097B1F0F601EB0D13
:101B9000F11DB3941081119781F4002371F0FB01C2
:101BA0003296DB01CD90DC90BF016E5F7F4FA0814C
:101BB000B181BB24015001C010E0F701E05FFA4F92
:101BC000892F86958695835C80830894E11CF11C9F
:101BD000F701E05FFA4F892F99278370907024E016
:101BE000880F991F2A95E1F755279A0194E03695B9
:101BF00027959A95E1F7822B835C80830894E11CFA
:101C0000F11CF701E05FFA4F4F705070440F551F01
:101C1000440F551F812F992726E0969587952A9581
:101C2000E1F7842B835C80830894E11CF11CF701AD
:101C3000E05FFA4F1F73135C10830894E11CF11CE2
:101C40006ACFC7010E943B0DE9E00C941A79A3E02A
:101C50007A2F40910B024650442309F458C0E72FD5
:101C6000FF27E259FB4F80818D537F5FE72FFF27CE
:101C7000E259FB4F20812D537F5FE72FFF27E25969
:101C8000FB4F30813D537F5FE72FFF27E259FB4F2A
:101C900060816D537F5F9927880F991F880F991F67
:101CA000522F52955F70582B822F99278F7090700A
:101CB000F4E0880F991FFA95E1F7232F26952695D2
:101CC000282B832F992783709070E6E0880F991F47
:101CD000EA95E1F7682B41504F3FC9F0EA2FFF2703
:101CE000E259FB4F5083AF5F41504F3F81F0EA2FE5
:101CF000FF27E259FB4F2083AF5F41504F3F39F040
:101D0000EA2FFF27E259FB4F6083AF5FA5CF81E742
:101D100094E090930A0280930902A350A0930802D2
:101D20000895A2E0B0E0E7E9FEE00C940479809128
:101D30000E02882309F4C7C30E94270E80916F0406
:101D4000823609F081C2809170049927813791050C
:101D500009F4C0C082379105C4F48D36910509F4A9
:101D600082C08E36910544F48B34910531F186366C
:101D7000910509F454C168C28E36910509F45BC01F
:101D80008037910509F49FC05FC28537910509F43A
:101D9000E2C18637910544F48337910509F4DCC02C
:101DA0008437910539F150C28737910509F410C283
:101DB0008937910509F46AC147C2E0910902F0919F
:101DC0000A028081918190933203809331032091A4
:101DD0002F0330913003821B930B845E9D4F68E686
:101DE00071E00E94A578845B904090932E038093CD
:101DF0002D032AC280910B02A0910902B0910A0220
:101E0000853140F080E1E9E4F4E00D9001928A959B
:101E1000E1F70DC08D919D910D90BC91A02D809307
:101E2000490490934A04A0934B04B0934C0480EF70
:101E3000809306024BC0809107018823E1F38DE473
:101E400090E09F938F9388E796E09F938F9381E034
:101E50008F938F938EE48F930E946B0D8DB79EB7F7
:101E600007968DBFF1C1A0910902B0910A021C91A1
:101E7000113081F48DE4E8E7F6E00D9001928A9547
:101E8000E1F70E94C12E1983809145048F7E8093D3
:101E9000450401C01982809107018823E1F381E0A4
:101EA00090E09F938F93CE0101969F938F9381E053
:101EB0008F938F938DE48F930E946B0DADB7BEB758
:101EC0001796ADBFC1C181E0809311028FEF80935F
:101ED0000501BAC1E0910902F0910A0280818F3FA9
:101EE00039F40E94262FE0910902F0910A028083C2
:101EF000E0910902F0910A028081882311F481E0C7
:101F000003C0863010F085E08083E0910902F091F3
:101F10000A0280810E94192EE0910902F0910A02C2
:101F200080818983809107018823E1F380E790E035
:101F30009F938F9387E096E09F938F9381E090E04B
:101F40009F938F93CE0101969F938F9382E08F93FF
:101F500081E08F9381E571C12091090230910A02DD
:101F6000D9018C918150853008F040C0F901818100
:101F70008435E1F52F5F3F4F80E7E7E0F6E0D901D8
:101F80000D9001928A95E1F7F90182910E945D2EF0
:101F9000809146069927AA27BB27BC01CD0124ECD6
:101FA00039E040E050E00E946678DC01CB0180938C
:101FB000B9019093BA01A093BB01B093BC01809189
:101FC00047069927AA27BB27BC01CD010E94667846
:101FD000DC01CB018093B5019093B601A093B701CA
:101FE000B093B8010E94262F898301C01982809185
:101FF00007018823E1F381E090E09F938F93CE0166
:1020000001969F938F9381E08F938F9383E58F93B6
:102010000E946B0D8DB79EB707968DBF26C0E091CD
:102020000902F0910A02E0818E2F8150853018F468
:102030008E2F0E94192E0E94262F898380910701DE
:102040008823E1F381E090E09F938F93CE01019686
:102050009F938F9381E08F938F9386E48F930E9459
:102060006B0DADB7BEB71796ADBF80911603882331
:1020700029F46EE670E089810E94253880E00E9494
:102080005A0780912E060E94F475DEC0E091090285
:10209000F0910A028081992787FD909590934A07D5
:1020A000809349078181992787FD909590934C07EC
:1020B00080934B078281992787FD909590934E07D7
:1020C00080934D078381992787FD909590935007C2
:1020D00080934F078481992787FD909590935207AD
:1020E000809351078581992787FD90959093540798
:1020F000809353078681992787FD90959093560783
:10210000809355078781992787FD9095909358076D
:10211000809357078085992787FD909590935A075C
:10212000809359078185992787FD909590935C0747
:1021300080935B078285992787FD909590935E0732
:1021400080935D078385992787FD9095909360071D
:1021500080935F0779C0E0910902F0910A028081C3
:102160000E94F8338A83882319F481E0898301C0AF
:102170001982809107018823E1F388E090E09F9322
:102180008F9386EC96E09F938F9321E030E03F930E
:102190002F938091090290910A029F938F933F930E
:1021A0002F93CE0102969F938F933F932F93CE014F
:1021B000820F931F9F938F9384E08F9381E08F937F
:1021C00085E58F930E946B0DEDB7FEB773963BC00C
:1021D000809108028930C0F12091090230910A02F1
:1021E0002F5F3F4F88E0A6ECB6E0F90101900D9219
:1021F0008A95E1F7D9018E910E944E338A83882314
:1022000019F481E0898301C0198280910701882334
:10221000E1F321E030E03F932F93CE0102969F93AC
:102220008F933F932F93CE01820F931F9F938F9392
:1022300082E08F9381E08F9387E58F930E946B0DEF
:10224000EDB7FEB73B96EDBF8091700499278436B9
:10225000910509F4CDC085369105ACF48136910520
:1022600009F481C0823691052CF48B34910509F470
:102270005DC021C18236910509F482C08336910583
:1022800009F491C018C18C36910509F4FFC08D3650
:1022900091054CF48736910509F40AC188369105F9
:1022A00009F4C4C008C18437910529F08637910527
:1022B00009F4FAC000C180910B02A0910902B0910B
:1022C0000A02803140F080E1E9E4F4E00D900192EF
:1022D0008A95E1F70DC08D919D910D90BC91A02D37
:1022E0008093490490934A04A0934B04B0934C0408
:1022F000809107018823E1F31F92809104018F935D
:1023000084E58F930E946B0D8AEF809306028FEF16
:102310008093050180EA9FE00E948E169093FF0152
:102320008093FE010F900F900F90C5C0E0910902BD
:10233000F0910A028081918190933203809331035E
:1023400020912F0330913003821B930B845E9D4FAD
:1023500068E671E00E94A578845B904090932E031C
:1023600080932D03A8C0E0910902F0910A028081B8
:1023700080930601803298F08FE1809306010FC0B0
:10238000A0910902B0910A028BE0E1E6F4E00D9021
:1023900001928A95E1F780916A048093F2058FEFAC
:1023A0008093050188C08091020290910302892BDD
:1023B00089F4E0910902F0910A02E081EE2351F0E4
:1023C0008AE0E89FC00111240E948E1690933C047D
:1023D00080933B04E0910902F0910A0290818AE027
:1023E000989FC0011124909303028093020215C0AC
:1023F0008FEF80930501E0910902F0910A0290812C
:102400008AE0989FC00111249093050280930402F2
:10241000892B19F081E08093130280EA9FE00E94EB
:102420008E169093FF018093FE0145C08FEF80933D
:102430000501E0910902F0910A02908197FD08C020
:1024400082E08093100210920102109200021AC0E2
:10245000909580916802892B8093680291818AE02F
:10246000989FC0011124909301028093000284E0A0
:102470008093100280EA9FE00E948E169093FF01E5
:102480008093FE0181E08093140215C08FEF80934A
:102490000501E0910902F0910A02808180936902AE
:1024A00081E08093150207C081E08093120203C08F
:1024B00081E08093160210920E0210920A0210928E
:1024C000090210920802E3E0CE5F0C942079982F65
:1024D0008091C00085FFFCCF9093C60008950F93B4
:1024E0001F9388E18093C1008091C0008260809337
:1024F000C0008091C10080688093C1008091C100BC
:1025000080648093C10000E010E00093C5008AE27F
:1025100090E08093C40080910402909105020E9493
:102520008E1690933E0480933D048CED90E00E94C3
:102530008E1690936D0480936C0410923F0480E596
:102540008093400485E0809343048BE080934104B2
:102550001092420410930A0200930902109208029A
:102560001F910F910895A0E1B0E0E9EBF2E10C9426
:10257000017980910701882309F4C1C28091FE018D
:102580009091FF010E949716882361F0109201023A
:10259000109200021092050210920402109203029F
:1025A000109202028091000290910102892B41F069
:1025B00080910E0590910F050E949716882329F4AB
:1025C00080911402882309F460C080910701882358
:1025D00009F45BC08091100200E211E08430A8F0A1
:1025E0000E94132080E590E09F938F931F930F9399
:1025F00081E08F938F9388E48F930E946B0D2DB7AA
:102600003EB7295F3F4F2DBF34C010926A0282E16E
:1026100094E09F938F9388E090E29F938F93E09153
:102620002B04F0912C04099584E190E09F938F9303
:102630001F930F9381E090E09F938F9380E192E04E
:102640009F938F9382E08F9381E08F9388E48F93A1
:102650000E946B0D80911002982F8F5F8093100263
:102660002DB73EB7215F3F4F2DBF943010F0109231
:10267000100280910002909101020E948E169093A8
:102680000F0580930E051092140280911502882385
:1026900051F180910701882331F10E94132080E5D8
:1026A00090E09F938F9380E291E09F938F9321E03E
:1026B00030E03F932F938FE191E09F938F933F936F
:1026C0002F9389E692E09F938F9383E08F9381E02D
:1026D0008F938CE48F930E946B0D109215028DB72F
:1026E0009EB70F968DBF809112028823D1F0809102
:1026F00007018823B1F08AE090E09F938F938FE3E6
:1027000094E09F938F9381E08F938F9386E58F93CF
:102710000E946B0D109212022DB73EB7295F3F4FFA
:102720002DBF809116028823D9F08091070188235C
:10273000B9F08BE090E09F938F9381E694E09F93B4
:102740008F9381E08F93809104018F9387E48F931F
:102750000E946B0D109216028DB79EB707968DBF23
:1027600080916C0490916D040E949716882309F45F
:1027700061C080910701882309F45CC08091230621
:102780009927880F991F880F991F7C010027F7FC54
:102790000095102F8091730390917403A09175039D
:1027A000B0917603BC01CD01A80197010E94DA78AF
:1027B00030935A042093590480916B0390916C03D9
:1027C000A0916D03B0916E03BC01CD01A8019701EA
:1027D0000E94DA7830935C0420935B0480910003BC
:1027E00080935D048091FF0280935E0488E090E016
:1027F0009F938F9389E594E09F938F9381E08F93CC
:1028000083E08F938BE68F930E946B0D80915F0422
:102810002DB73EB7295F3F4F2DBF853018F086E0BA
:1028200080935F0483E690E00E948E1690936D047F
:1028300080936C048091040290910502892B41F0F1
:1028400080913D0490913E040E949716882321F4C4
:1028500080911302882339F180910701882319F1AF
:102860000E941B3782E490E09F938F9380EB95E06A
:102870009F938F9381E08F938F9384E48F930E9433
:102880006B0D109213028DB79EB707968DBF809186
:10289000040290910502009731F00E948E169093E9
:1028A0003E0480933D048091020290910302892BA3
:1028B00009F4B8C080913B0490913C040E949716A3
:1028C000882309F4AFC080910701882309F4AAC0C6
:1028D000809123069927880F991F880F991F7C01E3
:1028E0000027F7FC0095102F8091730390917403DB
:1028F000A0917503B0917603BC01CD01A8019701A9
:102900000E94DA7830932E0420932D0480916B037B
:1029100090916C03A0916D03B0916E03BC01CD0149
:10292000A80197010E94DA783093300420932F0495
:102930002091F5073091F6074091F7075091F8077D
:10294000DA01C90163E0880F991FAA1FBB1F6A95AE
:10295000D1F7820F931FA41FB51F820F931FA41FCF
:10296000B51F2091990130919A0140919B0150919E
:102970009C01BC01CD010E94DA783093320420938F
:10298000310480913B0390913C03A0913D03B091B1
:102990003E0339E0B595A795979587953A95D1F778
:1029A000809333048091370390913803A0913903C9
:1029B000B0913A0329E0B595A795979587952A9503
:1029C000D1F7809334048091430390914403A09104
:1029D0004503B091460309E0B595A795979587956E
:1029E0000A95D1F7809335048EE090E09F938F9302
:1029F0008DE294E09F938F9381E08F938F9383E494
:102A00008F930E946B0D80910202909103020E94AD
:102A10008E1690933C0480933B042DB73EB7295FFC
:102A20003F4F2DBF809106018F3F71F1992714E030
:102A3000880F991F1A95E1F78E5E9D4F40E150E097
:102A4000BC01CE0101960E94947780E190E09F93B3
:102A50008F93CE0101969F938F9381E090E09F9397
:102A60008F9386E091E09F938F9382E08F9381E034
:102A70008F9381E48F930E946B0D8FEF80930601FB
:102A80008DB79EB70B968DBF8091F2058823D1F04C
:102A9000809107018823B1F081E090E09F938F93AC
:102AA00082EF95E09F938F9381E08F938F9382E4E1
:102AB0008F930E946B0D1092F2052DB73EB7295FE0
:102AC0003F4F2DBF809111028823C9F080910701EB
:102AD0008823A9F084E390E09F938F938FE297E09F
:102AE0009F938F9381E08F938F9380E58F930E94C4
:102AF0006B0D109211028DB79EB707968DBFE6E061
:102B0000C05F0C941D791F920F920FB60F92112483
:102B10002F933F935F936F937F938F939F93AF9385
:102B2000BF93EF93FF9320E080912402882329F044
:102B30008091240281508093240280910E04882386
:102B400019F0815080930E0480912C028150809363
:102B50002C028F3F09F05BC089E080932C028091AA
:102B60002A0290912B02019690932B0280932A02C5
:102B700080910A018F5F817080930A01882319F484
:102B800081E080932902349903C081E080932D0273
:102B90008091250290912602892B21F180912502B6
:102BA000909126020B9750F0809125029091260279
:102BB0000A97909326028093250204C01092260261
:102BC0001092250280912502909126022091080101
:102BD0003091090182239323892B11F021E008C051
:102BE00020E006C08FEF9FEF9093090180930801CA
:102BF00080910201222331F08A3011F45A9A07C0E1
:102C0000479A05C08A3011F45A9801C047988091BC
:102C10002D02882309F472C02091EC01222309F0CF
:102C20006DC08091140683FF69C086B19927FC01AD
:102C3000E071F07084FF14C0809127029091280207
:102C40000196909328028093270280912702909109
:102C50002802895E934008F451C020932D024EC093
:102C60008091270290912802892B09F443C080911A
:102C70002702909128028A569140E0F58091270220
:102C80009091280269E270E00E9491788091270279
:102C900090912802860F971F909328028093270215
:102CA00080912702909128020B9750F08091270283
:102CB000909128020A97909332038093310304C0C5
:102CC000F0933203E093310380913103909132030A
:102CD00020912F0330913003821B930B845E9D4F14
:102CE00068E671E00E94A578845B904090932E0383
:102CF00080932D031092280210922702FF91EF91EA
:102D0000BF91AF919F918F917F916F915F913F9113
:102D10002F910F900FBE0F901F90189520912A02AF
:102D200030912B02280F391FC90101960895209177
:102D30002A0230912B02821B930B892F99278695AB
:102D4000807490700895CF93DF930E948E16EC01EB
:102D5000CE010E9497168823D9F3DF91CF91089571
:102D6000CF93DF930E948E16EC0109C080910F0172
:102D7000882329F090930F018FEC80937A00CE0185
:102D80000E949716982F882389F3DF91CF91089599
:102D90009FB7F8945F983E9A469A8091B0008F70E2
:102DA0008093B0008091B00083608093B0008091E8
:102DB000B1008B738093B1008091B1008B608093E0
:102DC000B1001092B2008FEF8093B3008091B000F9
:102DD00080688093B000809170008A7F809370003B
:102DE000809170008260809370009FBF08958AE098
:102DF00090E00E948E16909335028093340282E018
:102E000085BD83EA84BD17BC84EB88BD86E086BDA2
:102E100080916E00816080936E0008951F920F92E2
:102E20000FB60F9211242F933F934F935F936F939D
:102E30007F938F939F93AF93BF93CF93DF93EF9342
:102E4000FF938091020190912E02843108F011C10C
:102E5000992309F06AC38091B00086FFECC080918D
:102E6000B0008F7B8093B00089EA93E090933002AA
:102E700080932F0280910B0190910C019C01220FF5
:102E8000331F280F391F8091A5019927880F991F9B
:102E9000880F991F280F391F37FF02C02D5F3F4F42
:102EA000C901959587959595879590930C01809389
:102EB0000B01909322028093210280916906609118
:102EC000350620917303309174034091750350913E
:102ED000760380FF2CC0772788279927EA01D9013C
:102EE00057FF04C0A158BF4FCF4FDF4FE7E0D59544
:102EF000C795B795A795EA95D1F79D01AE010E94B8
:102F000066789B01AC0197FF04C0215C3F4F4F4F97
:102F10005F4F66E055954795379527956A95D1F7A8
:102F20008091210290912202820F931F2BC077275C
:102F300088279927EA01D90157FF04C0A158BF4F3C
:102F4000CF4FDF4F27E0D595C795B795A7952A9521
:102F5000D1F79D01AE010E9466789B01AC0197FFFD
:102F600004C0215C3F4F4F4F5F4FF6E055954795AA
:102F700037952795FA95D1F78091210290912202F9
:102F8000821B930B9093220280932102809136063C
:102F9000282F3327220F331F220F331F8091210246
:102FA00090912202821793077CF080913706282F98
:102FB0003327220F331F220F331F8091210290915C
:102FC00022022817390724F4309322022093210289
:102FD00020912F02309130028091210290912202A3
:102FE000280F391F205032403093300220932F0297
:102FF000809121029091220297FD039695958795E5
:1030000095958795909322028093210245E02D3D6E
:10301000340718F08CED95E005C02757314030F4A7
:1030200087E791E09093300280932F0280912F02E6
:103030009091300243C28091B00080648093B000D0
:1030400080913C06282F33278DED96E0289FA00124
:10305000299F500D389F500D1124CA012091310233
:1030600030913202821B930B9093300280932F0297
:1030700059C2992309F059C28091B00086FF23C23A
:103080008091B0008F7B8093B000E0913302EE23FB
:10309000F1F480913C06282F33278DED96E0289F90
:1030A000A001299F500D389F500D1124CA01209175
:1030B000310230913202821B930B90933002809345
:1030C0002F021092320210923102469A2BC289EAE4
:1030D00093E09093300280932F028E2F99278330B4
:1030E000910509F4A4C1843091053CF48130910527
:1030F00061F0029709F4D2C0AAC18430910509F4A5
:1031000099C1059709F4A0C1A2C180910B019091CA
:103110000C019C01220F331F280F391F8091A5013C
:103120009927880F991F880F991F280F391F37FF7C
:1031300002C02D5F3F4FC90195958795959587955D
:1031400090930C0180930B019093220280932102B3
:103150008091690660913506209173033091740364
:10316000409175035091760380FF2CC07727882704
:103170009927EA01D90157FF04C0A158BF4FCF4F8B
:10318000DF4F27E0D595C795B795A7952A95D1F735
:103190009D01AE010E9466789B01AC0197FF04C0BF
:1031A000215C3F4F4F4F5F4FA6E0559547953795B0
:1031B0002795AA95D1F78091210290912202820F42
:1031C000931F27C077278827992757FF04C02158C6
:1031D0003F4F4F4F5F4FF7E05595479537952795F0
:1031E000FA95D1F70E9466789B01AC0197FF04C065
:1031F000215C3F4F4F4F5F4FE6E055954795379520
:103200002795EA95D1F78091210290912202821BA5
:10321000930B909322028093210280913606282FEF
:103220003327220F331F220F331F809121029091E9
:103230002202821793077CF080913706282F3327CC
:10324000220F331F220F331F8091210290912202FF
:103250002817390724F43093220220932102809109
:103260002F02909130022091210230912202820F90
:10327000931F805092409093300280932F02809150
:1032800021029091220297FD039695958795959539
:1032900087959093220280932102ECC080910D01CA
:1032A00090910E019C01220F331F280F391F80912E
:1032B000A4019927880F991F880F991F280F391F7C
:1032C00037FF02C02D5F3F4FC901959587959595B2
:1032D000879590930E0180930D0190932002809327
:1032E0001F028091690660913906A0916B03B0912D
:1032F0006C03C0916D03D0916E0381FF2AC07727C4
:10330000882799279D01AE01D7FF04C021583F4F60
:103310004F4F5F4FA7E05595479537952795AA954D
:10332000D1F70E9466789B01AC0197FF04C0215C35
:103330003F4F4F4F5F4FF6E055954795379527958F
:10334000FA95D1F780911F0290912002820F931F6E
:1033500029C07727882799279D01AE01D7FF04C090
:1033600021583F4F4F4F5F4FE7E0559547953795B1
:103370002795EA95D1F70E9466789B01AC0197FFEB
:1033800004C0215C3F4F4F4F5F4F76E05595479506
:10339000379527957A95D1F780911F029091200259
:1033A000821B930B9093200280931F0280913A0618
:1033B000282F3327220F331F220F331F80911F0224
:1033C00090912002821793077CF080913B06282F72
:1033D0003327220F331F220F331F80911F0290913A
:1033E00020022817390724F43093200220931F026B
:1033F00080912F029091300220911F023091200283
:10340000820F931F805092409093300280932F023E
:1034100080911F029091200297FD039695958795C4
:10342000959587959093200280931F0223C08091E9
:10343000C30702C080919D079927880F991F880FA5
:10344000991F87559E4F12C08091CB07F5CFFF275C
:10345000EE0FFF1FE15DF84F20813181220F331FF6
:1034600080912F0290913002820F931F909330022F
:1034700080932F0280912F029091300255E08D3D74
:10348000950718F08CED95E005C08757914030F412
:1034900087E791E09093300280932F0220912F02D2
:1034A000309130022C5B30403093300220932F0259
:1034B0008091310290913202820F931F90933202D9
:1034C000809331022FC08091B00080648093B0005F
:1034D0008CEB90E09093300280932F028091310228
:1034E0009091320284549F4F909332028093310224
:1034F00080912302882321F080911F03853B20F4D3
:1035000080912302823011F4469801C0469A80913E
:1035100033028F5F8093330290913C06981710F42A
:103520001092330281E080932E0220912F0230917D
:10353000300241E02F37340730F08FEF8093B30033
:103540002F5F30400FC02F3F3105C9F0C0F0A901F7
:103550004F5F50404F37510550F480E88093B300DF
:10356000205830403093300220932F0212C08FEF4A
:103570008093B3005093300240932F020AC0809191
:103580002F028093B3001092300210922F021092FB
:103590002E02FF91EF91DF91CF91BF91AF919F915B
:1035A0008F917F916F915F914F913F912F910F90EC
:1035B0000FBE0F901F90189510927C008FEC809397
:1035C0007A000895CF93DF9383E090E00E94042E69
:1035D000C82FDD27C531D10508F02A97C7BD109245
:1035E0003A0284E690E00E94B01680911301909117
:1035F00014018052934010F4C0E0D0E0CA3FD105DE
:10360000F8F4C7BD82E390E00E94B01687E294E030
:103610009F938F9387E692E19F938F93E0912B0482
:10362000F0912C04099580911301909114010F9051
:103630000F900F900F908052934010F02196DECFA4
:103640006C2F83E090E00E940A2EC09303068091C5
:10365000140680FF09C08C2F8A508B3E28F0809181
:103660004404806480934404C7BD8CE291E00E94CE
:10367000B016DF91CF910895EF92FF921F93CF93F1
:1036800010E080ED97E00E948E167C01CCE81330AC
:1036900019F4CB3008F0C9E010E080914A02909113
:1036A0004B028C5F934024F48091120181500AC038
:1036B00080914A0290914B028750944034F080915F
:1036C00012018F5F8093120101C011E080914802C6
:1036D000909149028C5F934024F4809111018150B4
:1036E0000AC080914802909149028750944034F07A
:1036F000809111018F5F8093110101C01F5F809144
:103700004602909147028C5F934024F4809110010F
:1037100081500AC0809146029091470287509440A0
:10372000C4F0809110018F5F8093100113C089E273
:1037300094E09F938F9387E692E19F938F93E0911C
:103740002B04F0912C0409950F900F900F900F907F
:103750005FC01F5F82E18093740280916F028E7F51
:1037600080936F0285EA8093BC00809112018A30B9
:1037700040F4809144048160809344048AE0809303
:10378000120180911201863F40F0809144048160D3
:103790008093440485EF80931201809111018A3057
:1037A00040F4809144048260809344048AE08093D2
:1037B000110180911101863F40F0809144048260A4
:1037C0008093440485EF80931101809110018A3029
:1037D00040F4809144048460809344048AE08093A0
:1037E000100180911001863F40F080914404846074
:1037F0008093440485EF80931001809174028823A4
:1038000039F0C7010E949716882309F090CFF5CFB1
:1038100010920F018FEC80937A0080910F01882322
:10382000E1F3CA3020F48AE090E00E94B016C15063
:1038300009F02DCF86E490E00E94B016CF911F9141
:10384000FF90EF9008951F920F920FB60F921124E0
:10385000AF92BF92CF92DF92EF92FF920F931F939E
:103860002F933F934F935F936F937F938F939F9388
:10387000AF93BF93EF93FF9380915302282F332789
:10388000442755278F5F80935302F9012231310578
:1038900008F08CC3E25CFF4F0C942C798091780087
:1038A0009091790046C080917800909179002CC168
:1038B0008091780090917900909356028093550200
:1038C00057C180917C0390917D03209178003091C5
:1038D0007900821B930B9093F4058093F3058091FC
:1038E000F3059091F4059093600280935F025EC1AE
:1038F000809178009091790020917E0330917F0330
:10390000821B930B9093020680930106809101061F
:1039100090910206909362028093610249C3809164
:10392000590290915A022091780030917900820FCB
:10393000931F90935A028093590281E03AC3809179
:103940005702909158022091780030917900820FAF
:10395000931F909358028093570284E02AC380916A
:103960001D0190911E019C01220F331F280F391F4A
:10397000809178009091790063E070E00E949178E6
:10398000260F371F369527953695279530931E01BC
:1039900020931D0185E00DC38091780090917900FE
:1039A0004091780350917903841B950B90934102C9
:1039B000809340028091400290914102029704F16D
:1039C00022E04E3E520784F4209154022B5F209354
:1039D000540225508091EC029091ED02845F914059
:1039E00018F4215F2093540280915402853684F1AB
:1039F0004F5F5F4F5093790340937803845626C0FE
:103A000080914002909141028F5F9F4F0CF532E010
:103A100047325307ECF02091540225502093540272
:103A20002B5F8091EC029091ED02845F914018F43D
:103A30002F5020935402809154028C394CF4415001
:103A4000504050937903409378038C5980935402EB
:103A500081E080933F02809178009091790090936B
:103A6000FA058093F90580914002909141029C01F2
:103A7000442737FD4095542F8091330390913403B0
:103A8000A0913503B0913603820F931FA41FB51F79
:103A90008093330390933403A0933503B09336039C
:103AA0002091330330913403409135035091360314
:103AB00057FF04C021503C4F4F4F5F4F0AE05595D0
:103AC0004795379527950A95D1F7809133039091C3
:103AD0003403A0913503B0913603821B930BA40BE2
:103AE000B50B8093330390933403A0933503B093C5
:103AF00036032EC180915702909158022091780090
:103B000030917900820F931F90935802809357024F
:103B10001092520250C2809102018A3071F4809159
:103B20007800909179002091550230915602820FD1
:103B3000931F01969695879517C040915502509115
:103B40005602843158F02091780030917900240F8A
:103B5000351F8FEF97E0821B930B06C08091780092
:103B600090917900840F951F9093470280934602AD
:103B700086E01FC280917C0390917D0320917800A4
:103B800030917900821B930B9093F4058093F30599
:103B90008091F3059091F40520915F0230916002CD
:103BA000820F931F909345028093440287E001C2E5
:103BB000809178009091790020917E0330917F036D
:103BC000821B930B9093020680930106809101065D
:103BD000909102062091610230916202820F931F40
:103BE0009093430280934202E3C1209159023091A5
:103BF0005A028091780090917900280F391F3093F4
:103C00005A0220935902809102018A3019F4220F3E
:103C1000331F04C0220F331F220F331F30935A0269
:103C2000209359022091590230915A02C90137FD5F
:103C30000796A3E095958795AA95E1F790934B0297
:103C400080934A0280915B0290915C02820F931FE5
:103C500097FD01969595879590935C0280935B0202
:103C60002091880330918903821B930B90931C0150
:103C700080931B01209150023091510280911B01D1
:103C800090911C01280F391F37FF02C02F5F3F4F53
:103C90003595279530935102209350024ECE2091B6
:103CA0005702309158028091780090917900280F46
:103CB000391F3093580220935702809102018A30B5
:103CC00019F4220F331F04C0220F331F220F331F9A
:103CD0003093580220935702209157023091580296
:103CE000C90137FD079663E0959587956A95E1F7D9
:103CF000909349028093480280915D0290915E0208
:103D0000820F931F97FD01969595879590935E027C
:103D100080935D022091860330918703821B930B71
:103D200090931A018093190120914E0230914F0215
:103D30008091190190911A01280F391F37FF02C095
:103D40002F5F3F4F3595279530934F0220934E02BA
:103D500083E02FC11092530281E080930F01809184
:103D60003602909137020196909337028093360283
:103D700080917800909179009093140180931301C1
:103D80008091130190911401AA27BB27A090630290
:103D9000B0906402C0906502D0906602A80EB91E71
:103DA000CA1EDB1EA0926302B0926402C09265023A
:103DB000D0926602809167028F5F809367028231A2
:103DC00008F4F6C08091150190911601A091170199
:103DD000B09118017C018D0123E0EE0CFF1C001F47
:103DE000111F2A95D1F7E81AF90A0A0B1B0BEA0CE6
:103DF000FB1C0C1D1D1D80913A02992787FD909593
:103E0000A92FB92FBC01CD0126EC34E240E050E0EF
:103E10000E946678DC01CB01E81AF90A0A0B1B0B39
:103E2000D801C7010496A11DB11DB7FF05C0D80177
:103E3000C7010B96A11DB11D13E0B595A7959795E8
:103E400087951A95D1F78093150190931601A09349
:103E50001701B09318018091FB059091FC057C013E
:103E60000027F7FC0095102F809115019091160105
:103E7000A0911701B0911801E81AF90A0A0B1B0B5F
:103E8000E0921103F09212030093130310931403B2
:103E900020913B0230913C0240913D0250913E0204
:103EA00057FF04C0215F3F4F4F4F5F4FF4E05595E0
:103EB000479537952795FA95D1F780913B029091D8
:103EC0003C02A0913D02B0913E02821B930BA40BD9
:103ED000B50B80933B0290933C02A0933D02B093BC
:103EE0003E0280913B0290913C02A0913D02B09134
:103EF0003E028E0D9F1DA01FB11F80933B02909329
:103F00003C02A0933D02B0933E0280913802909112
:103F10003902AC01E5E0440F551FEA95E1F7481B73
:103F2000590B80913B0290913C02A0913D02B091CF
:103F30003E02B7FF03C00F96A11DB11D74E0B595F9
:103F4000A795979587957A95D1F720911103309190
:103F50001203281B390B63E0220F331F6A95E1F728
:103F6000240F351F37FF02C0215E3F4F45E03595D6
:103F700027954A95E1F73093390220933802D6010C
:103F8000C501D7FE03C00196A11DB11DB595A7952A
:103F9000979587958093630290936402A09365023E
:103FA000B093660289E08093670202C010925302C8
:103FB00082E0809352028091520280937C00809133
:103FC0005302882319F08FEC80937A00FF91EF91D0
:103FD000BF91AF919F918F917F916F915F914F9121
:103FE0003F912F911F910F91FF90EF90DF90CF9015
:103FF000BF90AF900F900FBE0F901F90189590E25A
:10400000E0E2F1E08FE49193815087FFFCCF0895C7
:1040100090916A02E0E2F1E0E90FF11D80839F5F79
:1040200090936A020895EF92FF920F931F93CF939C
:10403000DF932091680220FF0AC0809169028823E3
:1040400011F0815002C080911F018093690221FF0D
:104050000CC09091690280911F01981719F4109279
:10406000690203C09F5F90936902822F992780FFA6
:1040700004C081FF02C0109269020E94FF1F80915C
:104080006902282F3327C8E0EC2EC0E2FC2EC09135
:104090002B04D0912C048A3098F481E180936A0239
:1040A0003F932F9380E694E09F938F93FF92EF923C
:1040B000FE0109952DB73EB72A5F3F4F2DBF11C0B6
:1040C00080E180936A023F932F9385E694E09F936B
:1040D0008F93FF92EF92FE0109958DB79EB70696DA
:1040E0008DBF20916902822F9927AA27BB27FC0147
:1040F000429710F00C94C02AE05BFF4FB8E0EB2E23
:10410000B0E2FB2EC0912B04D0912C040C942C799E
:1041100010926A028AE694E09F938F9308E010E27F
:10412000FF92EF92FE01099584E180936A020F905D
:104130000F900F900F9086E690E09F938F9380E50D
:1041400090E09F938F931F921F92809102016AE0EB
:104150000E948578892F99279F938F9380910201E0
:104160000E94857899279F938F938AE794E09F9385
:104170008F93FF92EF92E0912B04F0912C0409951C
:1041800088E280936A022DB73EB7225F3F4F2DBF72
:1041900089E796E09F938F930E94262F99279F93FC
:1041A0008F938FE894E09F938F93FF92EF92E0912B
:1041B0002B04F0912C0409958DB79EB708968DBFFE
:1041C00090914404992351F08CE380936A02892FE3
:1041D00099279F938F938DE994E085C69091700203
:1041E000992371F08CE380936A02892F99279F931A
:1041F0008F9384EB94E09F938F931F930F9391C0C1
:104200008091450484FF07C08CE380936A0289ECA7
:1042100094E00C94522A809191019091920106971A
:1042200010F00C94C92A8CE380936A0286ED94E026
:104230000C94522A80911406A8E0EA2EA0E2FA2EED
:10424000C0912B04D0912C0480FF74C010926A029C
:104250008091110390911203A0911303B091140364
:10426000BC01CD0125E030E040E050E00E94DA786A
:104270003F932F9383EE94E09F938F93FF92EF925F
:10428000FE01099584E180936A022DB73EB72A5F4B
:104290003F4F2DBF80910D0390910E03A0910F030E
:1042A000B0911003BC01CD0125E030E040E050E0CA
:1042B0000E94DA783F932F9380EF94E09F938F933F
:1042C000FF92EF92E0912B04F0912C04099588E283
:1042D00080936A028DB79EB706968DBF80911301B9
:1042E000909114019F938F938DEF94E09F938F9300
:1042F000FF92EF92E0912B04F0912C0409958CE34E
:1043000080936A022DB73EB72A5F3F4F2DBF87B516
:1043100099279F938F938AE095E09F938F93FF92C5
:10432000EF92E0912B04F0912C0409958DB79EB784
:1043300006962FC710926A0287E195E09F938F93AC
:10434000FF92EF92FE01099584E180936A020F903B
:104350000F900F900F9086E295E09F938F93FF92BE
:10436000EF92E0912B04F0912C04099588E2809360
:104370006A020F900F900F900F908FE295E09F933D
:104380008F93FF92EF92E0912B04F0912C0409950A
:104390008CE380936A020F900F900F900F908EE342
:1043A00095E09F938F93FF92EF920C94562A109270
:1043B0006A0287E495E09F938F9308E010E2FF92F2
:1043C000EF92FE01099584E180936A020F900F90AD
:1043D0000F900F908091730390917403A0917503D7
:1043E000B0917603B7FF04C081509C4FAF4FBF4FD1
:1043F000FAE0B595A79597958795FA95D1F7BF936C
:10440000AF939F938F9384E595E09F938F931F9332
:104410000F93E0912B04F0912C04099588E280938E
:104420006A022DB73EB7285F3F4F2DBF80916B03C7
:1044300090916C03A0916D03B0916E03B7FF04C01F
:1044400081509C4FAF4FBF4FEAE0B595A795979528
:104450008795EA95D1F7BF93AF939F938F9383E6A8
:1044600095E09F938F931F930F93E0912B04F0910E
:104470002C0409958CE380936A028DB79EB7089649
:104480008DBF80913103909132039F938F9382E788
:1044900095E09F938F931F930F93E0912B04F091DE
:1044A0002C0409952DB73EB72A5F3F4F0DC71092D8
:1044B0006A0280913307909134079F938F93809184
:1044C0003107909132079F938F9381E895E09F93F6
:1044D0008F93FF92EF92FE01099584E180936A0227
:1044E0008DB79EB708968DBF80913707909138079A
:1044F0009F938F9380913507909136079F938F9369
:1045000081E995E09F938F93FF92EF92E0912B04C6
:10451000F0912C04099588E280936A022DB73EB78A
:10452000285F3F4F2DBF80913B0790913C079F93A1
:104530008F938091390790913A079F938F9381EAE7
:1045400095E09F938F93FF92EF92E0912B04F0916F
:104550002C0409958CE380936A028DB79EB7089668
:104560008DBF80913F07909140079F938F938091DB
:104570003D0790913E079F938F9381EB95E0A2C0FA
:1045800010926A0280910906E82FFF27EE0FFF1FA5
:10459000E15DF84F808191819F938F938091080610
:1045A000E82FFF27EE0FFF1FE15DF84F808191811B
:1045B0009F938F9381EC95E09F938F93FF92EF925F
:1045C000FE01099584E180936A028DB79EB7089633
:1045D0008DBF80910B06E82FFF27EE0FFF1FE15DD7
:1045E000F84F808191819F938F9380910A06E82FE5
:1045F000FF27EE0FFF1FE15DF84F80819181885802
:104600009F4F9F938F9381ED95E09F938F93FF92A0
:10461000EF92E0912B04F0912C04099588E28093AD
:104620006A022DB73EB7285F3F4F2DBF80910D0620
:10463000E82FFF27EE0FFF1FE15DF84F808191818A
:1046400082599F4F9F938F9380910C06E82FFF27ED
:10465000EE0FFF1FE15DF84F8081918182599F4FDE
:104660009F938F9381EE95E09F938F93FF92EF92AC
:10467000E0912B04F0912C0409958CE380936A025D
:104680008DB79EB708968DBF80910F06E82FFF2744
:10469000EE0FFF1FE15DF84F8081918182599F4F9E
:1046A0009F938F9380910E06E82FFF27EE0FFF1F39
:1046B000E15DF84F8081918182599F4F9F938F9345
:1046C00081EF95E09F938F93FF92EF92E0912B04FF
:1046D000F0912C0409952DB73EB7285F3F4FF4C5E4
:1046E00010926A0281E096E09F938F9308E010E2B7
:1046F000FF92EF92FE010995809102010F900F90B9
:104700000F900F908A3009F0A1C084E180936A0273
:1047100080918803909189039C0197FF02C0295FD3
:104720003F4F287F821B930B9F938F938091880329
:104730009091890397FD079673E0959587957A95F3
:10474000E1F79F938F93209188033091890337FF7E
:1047500002C0295F3F4F63E0359527956A95E1F7E1
:1047600080914A0290914B02821B930B9F938F93EF
:104770008FE096E09F938F931F930F93E0912B040C
:10478000F0912C04099588E280936A028DB79EB758
:104790000A968DBF80918603909187039C0197FFB5
:1047A00002C0295F3F4F287F821B930B9F938F93FB
:1047B000809186039091870397FD079653E0959526
:1047C00087955A95E1F79F938F93209186033091B7
:1047D000870337FF02C0295F3F4F43E03595279598
:1047E0004A95E1F78091480290914902821B930B10
:1047F0009F938F9380E296E09F938F931F930F93E5
:10480000E0912B04F0912C0409958CE380936A02CB
:104810002DB73EB7265F3F4F2DBF80918403909107
:1048200085039F938F9380918403909185032091BA
:10483000460230914702821B930B9F938F9381E333
:1048400096E09F938F931F930F93A3C38B3019F020
:10485000843108F4ADC084E180936A0280918803BA
:10486000909189039C0197FF02C0215F3F4F207FF9
:10487000821B930B97FD0196959587959F938F9338
:10488000809188039091890397FD0F9624E0959578
:1048900087952A95E1F79F938F9320918803309114
:1048A000890337FF02C0295F3F4F83E03595279585
:1048B0008A95E1F780914A0290914B02821B930BFB
:1048C0009F938F938FE396E09F938F931F930F9304
:1048D000E0912B04F0912C04099588E280936A0200
:1048E0002DB73EB7265F3F4F2DBF80918603909135
:1048F00087039C0197FF02C0215F3F4F207F821BEF
:10490000930B97FD0196959587959F938F93809133
:1049100086039091870397FD0F96B4E09595879550
:10492000BA95E1F79F938F93209186033091870387
:1049300037FF02C0295F3F4FA3E035952795AA9521
:10494000E1F78091480290914902821B930B9F935B
:104950008F9381E596E09F938F931F930F93E09140
:104960002B04F0912C0409958CE380936A028DB797
:104970009EB70A968DBF809184039091850397FD21
:104980000196959587959F938F938091840390913D
:1049900085032091460230914702821B930B9F931F
:1049A0008F9383E696E09F938F931F930F938ECE02
:1049B0008D3009F0EEC584E180936A028091120186
:1049C00099279F938F93809188039091890397FDF6
:1049D0000F96E4E095958795EA95E1F79F938F937D
:1049E000209188033091890337FF02C0295F3F4F30
:1049F00073E0359527957A95E1F780914A02909179
:104A00004B02821B930B9F938F9382E796E09F93B9
:104A10008F931F930F93E0912B04F0912C04099531
:104A200088E280936A028DB79EB70A968DBF809107
:104A3000110199279F938F9380918603909187030B
:104A400097FD0F9664E0959587956A95E1F79F939A
:104A50008F93209186033091870337FF02C0295F2F
:104A60003F4F53E0359527955A95E1F780914802DD
:104A700090914902821B930B9F938F9386E896E057
:104A80009F938F931F930F93E0912B04F0912C042D
:104A900009958CE380936A022DB73EB7265F3F4F9E
:104AA0002DBF8091100199279F938F93809184034C
:104AB0009091850397FD0196959587959F938F9388
:104AC00080918403909185032091460230914702A2
:104AD000821B930B9F938F938AE996E09F938F930A
:104AE0001F930F93E0912B04F0912C0409958DB73F
:104AF0009EB70A964EC310926A028EEA96E09F9382
:104B00008F93FF92EF92FE01099584E180936A02F0
:104B10000F900F900F900F9080917E0390917F03E4
:104B20009F938F9380914202909143029F938F9322
:104B30008BEB96E09F938F93FF92EF92E0912B0483
:104B4000F0912C04099588E280936A022DB73EB754
:104B5000285F3F4F2DBF80917C0390917D039F93F1
:104B60008F9380914402909145029F938F938AEC9A
:104B700096E09F938F93FF92EF92E0912B04F09138
:104B80002C0409958CE380936A028DB79EB7089632
:104B90008DBF80917803909179039F938F9380913B
:104BA0004002909141029F938F9389ED96E08ACDC8
:104BB00010926A0280911D0190911E016AE070E0DE
:104BC0000E94A5789F938F9380911D0190911E0163
:104BD0006AE070E00E94A5787F936F9388EE96E07C
:104BE0009F938F93FF92EF92FE01099584E180934A
:104BF0006A028DB79EB708968DBF80916C08909120
:104C00006D086AE070E00E9491789F938F93809185
:104C10006C0890916D086AE070E00E9491787F9333
:104C20006F938CEF96E09F938F93FF92EF92E091BA
:104C30002B04F0912C04099588E280936A022DB729
:104C40003EB7285F3F4F2DBF80916E0890916F084F
:104C50009F938F9380E197E09F938F93FF92EF92C2
:104C6000E0912B04F0912C0409958CE380936A0267
:104C70008DB79EB706968DBF809170089091710890
:104C80009F938F9380E297E02EC110926A0282E395
:104C900097E09F938F93FF92EF92FE01099584E135
:104CA00080936A020F900F900F900F9080912F07C2
:104CB000909130079F938F938BE397E09F938F930F
:104CC000FF92EF92E0912B04F0912C04099588E279
:104CD00080936A028DB79EB706968DBF80911F03A1
:104CE00099279F938F938BE497E09F938F93FF92E5
:104CF000EF92E0912B04F0912C0409958CE38093C2
:104D00006A022DB73EB72A5F3F4F2DBF80912E0715
:104D1000992701979F938F938BE597E0FECA109296
:104D20006A028BE697E09F938F93FF92EF92FE01CA
:104D3000099584E180936A020F900F900F900F9075
:104D400080912D0390912E039F938F9383E797E09B
:104D50009F938F93FF92EF92E0912B04F0912C049C
:104D6000099588E280936A022DB73EB72A5F3F4FCC
:104D70002DBF80913103909132039F938F9381E8EF
:104D800097E09F938F93FF92EF92E0912B04F09125
:104D90002C0409958CE380936A028DB79EB7069622
:104DA0008DBF80912F03909130039F938F938FE855
:104DB00097E099C010926A028091200399279F93EF
:104DC0008F938DE997E09F938F93FF92EF92FE016F
:104DD000099584E180936A028DB79EB706968DBFD0
:104DE0008091210399279F938F9389EA97E09F935E
:104DF0008F93FF92EF92E0912B04F0912C04099590
:104E000088E280936A022DB73EB72A5F3F4F2DBFDD
:104E10008091220399279F938F9385EB97E09F932F
:104E20008F93FF92EF92E0912B04F0912C0409955F
:104E30008CE380936A028DB79EB706968DBF8091F2
:104E4000230399279F938F9381EC97E04CC0109296
:104E50006A028091240399279F938F938DEC97E0AA
:104E60009F938F93FF92EF92FE01099584E18093C7
:104E70006A028DB79EB706968DBF8091250399274C
:104E80009F938F9389ED97E09F938F93FF92EF927B
:104E9000E0912B04F0912C04099588E280936A023A
:104EA0002DB73EB72A5F3F4F2DBF8091260399272C
:104EB0009F938F9385EE97E09F938F93FF92EF924E
:104EC000E0912B04F0912C0409958CE380936A0205
:104ED0008DB79EB706968DBF8091270399279F9324
:104EE0008F9381EF97E09F938F93FF92EF92D5CAB4
:104EF00010926A028DEF97E09F938F93FF92EF924B
:104F0000FE01099584E180936A020F900F900F9043
:104F10000F908091A50199279F938F9385E098E04A
:104F20009F938F93FF92EF92E0912B04F0912C04CA
:104F3000099588E280936A028DB79EB706968DBF69
:104F400080912102909122029F938F9383E198E0B8
:104F50009F938F93FF92EF92E0912B04F0912C049A
:104F600009958CE380936A022DB73EB72A5F3F4FC5
:104F70002DBF8091370699279F938F938091360696
:104F800099279F938F9381E298E09F938F93FF924D
:104F9000EF92E0912B04F0912C0409958DB79EB708
:104FA0000896F7C010926A028FE298E09F938F9361
:104FB000FF92EF92FE01099584E180936A020F90BF
:104FC0000F900F900F9080916504992787FD909521
:104FD0009F938F9380916404992787FD90959F9369
:104FE0008F938FE398E09F938F93FF92EF92E091DE
:104FF0002B04F0912C04099588E280936A022DB766
:105000003EB7285F3F4F2DBF80916604992787FDEB
:1050100090959F938F938091670499279F938F9387
:105020008FE498E09F938F93FF92EF92E0912B048F
:10503000F0912C0409958CE380936A028DB79EB79A
:1050400008968DBF80916B0499279F938F938091D1
:105050006804992787FD90959F938F938FE598E03B
:1050600031CB10926A028FE698E09F938F93FF9264
:10507000EF92FE01099584E180936A020F900F90F0
:105080000F900F908091E90699278F7790709F93EA
:105090008F938091E10699278F7790709F938F93DC
:1050A0008091D90699278F7790709F938F938091E5
:1050B000D10699278F7790709F938F938FE798E011
:1050C0009F938F93FF92EF92E0912B04F0912C0429
:1050D000099588E280936A028DB79EB70C968DBFC2
:1050E0008091090799278F7790709F938F93809174
:1050F000010799278F7790709F938F938091F9067E
:1051000099278F7790709F938F938091F1069927BD
:105110008F7790709F938F9380E998E09F938F9300
:10512000FF92EF92E0912B04F0912C0409958CE30F
:1051300080936A022DB73EB7245F3F4F2DBF809109
:10514000290799278F7790709F938F9380912107DC
:1051500099278F7790709F938F9380911907992744
:105160008F7790709F938F938091110799278F77F6
:1051700090709F938F9381EA98E09F938F93FF9213
:10518000EF92E0912B04F0912C0409958DB79EB716
:105190000C968DBFFEC110926A0282EB98E09F933D
:1051A0008F93FF92EF92FE01099584E180936A024A
:1051B0000F900F900F900F908091ED06992787FD2B
:1051C00090959F938F938091E506992787FD909501
:1051D0009F938F938091DD06992787FD90959F93EC
:1051E0008F938091D506992787FD90959F938F93F4
:1051F00081EC98E09F938F93FF92EF92E0912B04C4
:10520000F0912C04099588E280936A022DB73EB78D
:10521000245F3F4F2DBF80910D07992787FD909503
:105220009F938F9380910507992787FD90959F9372
:105230008F938091FD06992787FD90959F938F937B
:105240008091F506992787FD90959F938F9382ED26
:1052500098E09F938F93FF92EF92E0912B04F0914F
:105260002C0409958CE380936A028DB79EB70C9647
:105270008DBF80912D07992787FD90959F938F93E0
:1052800080912507992787FD90959F938F93809113
:105290001D07992787FD90959F938F938091150700
:1052A000992787FD90959F938F9383EE98E09F9326
:1052B0008F93FF92EF92E0912B04F0912C040995CB
:1052C0002DB73EB7245F3F4F2DBF63C110926A02D6
:1052D00084EF98E09F938F9308E010E2FF92EF92A3
:1052E000FE01099584E180936A020F900F900F9060
:1052F0000F908091E906881F8827881F97E0899F73
:10530000C00111248D969F938F938091E106881F91
:105310008827881F96E0899FC00111248D969F934E
:105320008F938091D906881F8827881F95E0899FD1
:10533000C00111248D969F938F938091D106881F71
:105340008827881F9927880F991F880F991F8D9686
:105350009F938F9383E099E09F938F93FF92EF92B7
:10536000E0912B04F0912C04099588E280936A0265
:105370008DB79EB70C968DBF80910907881F88272F
:10538000881F9BE0899FC00111248D969F938F9366
:1053900080910107881F8827881F9AE0899FC00194
:1053A00011248D969F938F938091F906881F8827EB
:1053B000881F99E0899FC00111248D969F938F9338
:1053C0008091F106881F8827881F992723E0880F7E
:1053D000991F2A95E1F78D969F938F9387E199E026
:1053E0009F938F93FF92EF92E0912B04F0912C0406
:1053F00009958CE380936A022DB73EB7245F3F4F37
:105400002DBF80911107881F8827881F9CE0899FE6
:10541000C00111248D969F938F938BE299E09F9307
:105420008F93FF92EF92E0912B04F0912C04099559
:10543000809119072DB73EB72A5F3F4F2DBF87FFD9
:1054400012C080E480936A028CE399E09F938F936B
:10545000FF92EF92E0912B04F0912C0409950F90AC
:105460000F900F900F908091210787FF12C084E466
:1054700080936A028FE399E09F938F931F930F931A
:10548000E0912B04F0912C0409950F900F900F9050
:105490000F908091290787FF7CC088E480936A027F
:1054A00082E499E09F938F931F930F93E0912B04D5
:1054B000F0912C0409950F900F900F900F9069C0F8
:1054C00010926A0285E499E09F938F93FF92EF9286
:1054D000FE01099584E180936A020F900F900F906E
:1054E0000F908091F9019091FA019F938F9383E53A
:1054F00099E09F938F93FF92EF92E0912B04F091AC
:105500002C04099588E280936A028DB79EB70696AF
:105510008DBF8091FB019091FC019F938F9380E65A
:1055200099E09F938F93FF92EF92E0912B04F0917B
:105530002C04099589E480936A022DB73EB72A5F4F
:105540003F4F2DBF8DE699E09F938F93FF92EF928F
:10555000E0912B04F0912C040995809168020F9042
:105560000F900F900F9083FF14C01092FC011092C7
:10557000FB0160E070E08EE090E00E94142E09C014
:1055800080911F01281719F4215020931F011092B8
:10559000690210926802E6E0CDB7DEB70C941D797F
:1055A0004AEA20E030E02617370740F4FC018191F9
:1055B000480F2F5F3F4F26173707C8F3842F9927CF
:1055C0000895AC019AEA20E030E02617370750F43E
:1055D000DA01A20FB31F0E943279802D980F2F5F3E
:1055E0003F4FF3CF892F9927089581E080930A06D2
:1055F00082E08093090683E08093080684E080932C
:105600000B0685E080930C0686E080930D0687E00C
:1056100080930E0688E080930F0689E08093100641
:105620008AE0809311068BE0809312068CE08093D1
:10563000130608951F93CF93DF9384E580930706A5
:1056400080910201843150F08AE080932706109205
:1056500049068BE1809323068EE40AC083E08093A1
:10566000270680E2809349068EE18093230685E534
:1056700080934606809347068AE68093140683E06B
:1056800080936A06AEE1A09315068FEF809317060C
:10569000EFE0E0931806A093160610921A06F8E0C1
:1056A000F0931B0680E480931C0610921D0684E193
:1056B000809319068EE080931E06B0E1B0931F061A
:1056C0001CE010932006F093210686EE80932206BC
:1056D00080E88093240650E55093250686E9809360
:1056E0002606509328068093290676E070932A06B2
:1056F00081E280932B068DE280932C069AE59093AD
:105700002D0680E280932F0610923006109231060B
:10571000109232061092330610924B0610924C06ED
:1057200010924D0610924E0634E63093340648E24D
:105730004093350661E0609369061092360627EFC4
:105740002093370670933C068DE780933D06809347
:105750003E0680933F0630933806409339061092F8
:105760003A0620933B0682E38093400690934106DD
:105770008093420610926806909343065093440625
:1057800060934506B093480630934A068FE58093B0
:105790004F0683EF809351068AEA809353068093E5
:1057A0005406E0935006E09352068EEF8093550620
:1057B0003093560690935706909358069093590647
:1057C0008BE480935A0680935B0680935C0610926C
:1057D0005D0670935E06F0935F0690936006A0935B
:1057E0006106309362063093630682E0809364061C
:1057F00060932E061092660610926706ABE6B6E03E
:10580000E0E7F1E0ED01019009921A95E1F760E718
:1058100070E0CD01845690400E94D02A8093770694
:10582000DF91CF911F910895CF93DF9384E580930B
:10583000070680910201843150F08AE080932706A8
:10584000109249068BE1809323068EE40AC083E020
:105850008093270680E2809349068EE18093230699
:1058600085E580934606809347068AE68093140672
:1058700083E080936A067EE1709315068FEF809334
:1058800017069FE0909318067093160610921A065A
:1058900068E060931B0680E480931C0610921D064E
:1058A000909319068AE080931E0680E180931F067C
:1058B00056E0509320066093210686EE80932206E0
:1058C00080E8809324062AE52093250688E78093C4
:1058D0002606209328068093290650932A0681E203
:1058E00080932B068DE280932C0620932D06E0E218
:1058F000E0932F0610923006109231061092320675
:105900001092330610924B0610924C0610924D06E0
:1059100010924E0644E64093340638E23093350642
:10592000F1E0F09369061092360697EF90933706F0
:1059300050933C068DE780933D0680933E0680930E
:105940003F06409338063093390610923A069093FA
:105950003B0682E3809340062093410680934206F3
:10596000109268062093430680E5809344068CE3FA
:1059700080934506E09348069BE490934A068FE5A2
:1059800080934F0683EF809351068AEA80935306F3
:105990008093540684E180935006809352068EEFE4
:1059A0008093550640935606209357062093580639
:1059B0002093590690935A0690935B0690935C0649
:1059C00010925D0650935E0660935F06209360061A
:1059D00070936106409362064093630682E0809371
:1059E0006406F0932E061092660610926706ABE6E8
:1059F000B6E08CE0E7E7F1E0ED01019009928A95CD
:105A0000E1F760E770E0CD01845690400E94D02A13
:105A100080937706DF91CF910895CF93DF9384E54C
:105A20008093070680910201843150F08AE08093D0
:105A30002706109249068BE1809323068EE40AC064
:105A400083E08093270680E2809349068EE180936D
:105A5000230685E580934606809347068AE6809371
:105A6000140683E080936A066EE1609315068FEF5B
:105A7000809317069FE09093180660931606109285
:105A80001A0678E070931B0680E480931C0610923F
:105A90001D069093190670931E0690E190931F06C1
:105AA00056E0509320067093210686EE80932206DE
:105AB00080E88093240634E63093250688E78093B7
:105AC0002606309328068093290650932A0681E201
:105AD00080932B068DE280932C062AE520932D06D9
:105AE00090932F06109230061092310610923206D3
:105AF0001092330610924B0610924C0610924D06EF
:105B000010924E063093340648E240933506E1E0A9
:105B1000E09369061092360697EF909337065093FC
:105B20003C068DE780933D0680933E0680933F06BA
:105B3000309338064093390610923A0690933B060C
:105B400082E38093400620934106809342061092A0
:105B500068062093430680E58093440696E490937C
:105B6000450680E28093480690934A068FE580932D
:105B70004F0683EF809351068AEA80935306809301
:105B8000540660935006609352068EEF809355063C
:105B900030935606209357062093580620935906B3
:105BA0008BE480935A0680935B0680935C06109288
:105BB0005D0650935E0670935F06209360066093C7
:105BC0006106309362063093630682E08093640638
:105BD000E0932E061092660610926706ABE6B6E0DA
:105BE0008CE0EFE7F1E0ED01019009928A95E1F791
:105BF00060E770E0CD01845690400E94D02A8093E7
:105C00007706DF91CF910895DC010E943279802DD3
:105C100099270895DC01062E0E9444790895DC013D
:105C20000E943F79CF010895DC010B010E94507959
:105C30000895FF920F931F93CF93DF93982F815076
:105C4000853008F093E081E7F82E9F9D80011124B4
:105C5000E8012D9760E770E0CE010E94E12A982FBD
:105C6000D801AD59BF4F0E943279802D891731F488
:105C7000DE010E943279802D843519F080E090E0B9
:105C80000AC0E7E0F6E0DE011F2C0E943A790E948C
:105C9000F96781E090E0E5E0CDB7DEB70C941E79BE
:105CA000863010F085E003C0882309F481E0A2E08B
:105CB000B0E0082E0E94447908951F93CF93DF939C
:105CC000182FC7E0D6E080910706843591F516308D
:105CD00010F015E002C0112361F160E770E087E089
:105CE00096E00E94D02A8093770681E7189FD00122
:105CF00011241D97FE01182E0E945579E8E0F6E068
:105D0000A0E5B0E02CE030E0122E0E945579B901F8
:105D100088E096E00E94D02AACE5B0E0082E0E9410
:105D20004479812F0E94502E0E94F96781E090E013
:105D300002C080E090E0DF91CF911F9108956DE463
:105D400070E088EE93E00E94E12AA5E3B4E00E94AF
:105D50003279902D981739F4A8EEB3E00E94327989
:105D6000802D813019F080E090E00895E8E7F6E0BA
:105D7000A8EEB3E08EE4182E0E943A7981E090E01C
:105D80000895CF93DF93C8E7D6E0809178068130FD
:105D900089F46DE470E0CE010E94D02A8093C5069C
:105DA000A8EEB3E08EE4FE01182E0E94557981E042
:105DB00090E002C080E090E0DF91CF910895CF9312
:105DC000DF9381E080937806E8E7F6E08FE01586C0
:105DD00016861786108A8150349687FFF8CF80E4A4
:105DE00080938506809386061092870680938806A6
:105DF0008093890690EC90938A0610928B0680938C
:105E00008C0680938D0610928E0690938F06909349
:105E10009006809391061092920680939306909339
:105E20009406A9E7B6E087E0E9E8F1E0ED0101902A
:105E300009928A95E1F76DE470E0CD0101970E9427
:105E4000D02A8093C506DF91CF910895A2E0B0E0FB
:105E50000E943279802D863030F083E0A2E0B0E0FD
:105E6000082E0E94447999270895DF92EF92FF92BD
:105E70000F931F93CF93FF24DF2CEF2C81E090E052
:105E80000E94042E843539F031E0E32E64E581E090
:105E900090E00E940A2E6CE070E080E590E00E94A5
:105EA000E12AC82FACE5B0E00E943279802D8C1732
:105EB00011F421E0D22EC1E001E010E0EE2029F43F
:105EC0008C2F0E94192E8823B1F591E0F92E1F9393
:105ED0000F9385E799E09F938F9387E692E19F93D5
:105EE0008F93E0912B04F0912C0409958DB79EB708
:105EF00006968DBF0230110549F0033011054CF4B0
:105F00000130110531F40E941A2B05C00E94142C97
:105F100002C00E940D2DDD2049F0E8E0F6E0A0E58A
:105F2000B0E08CE0182E0E943A7902C00E94F52A57
:105F30008C2F0E945D2ECF5F0F5F1F4FC63008F47D
:105F4000BDCFFF2019F083E00E94502E0E94262F23
:105F5000C82F0E94192E8C2F99279F938F938BE91E
:105F600099E09F938F9307E612E11F930F93E091BF
:105F70002B04F0912C0409958DB79EB706968DBF22
:105F8000EE2021F40E949F2E882399F484EB99E05F
:105F90009F938F931F930F93E0912B04F0912C0408
:105FA00009950E94DF2E0E94C12E0F900F900F9036
:105FB0000F901092060690E0E5E8F6E0CFE08081D1
:105FC000349618160CF49F5FC150C7FFF8CF90931A
:105FD0000606892F99279F938F9389E796E09F93D1
:105FE0008F9385ED99E09F938F931F930F93E0918B
:105FF0002B04F0912C0409958DB79EB708968DBFA0
:1060000086EF99E09F938F931F930F93E0912B045A
:10601000F0912C0409950F900F900F900F90CF9155
:106020001F910F91FF90EF90DF9008959FB7F89424
:106030003998389A88B1836088B98091B9008C7F8B
:106040008093B9008AE28093B80010927402109293
:10605000720210927102EEECF6E08BE01082118277
:10606000128213821482158216821782815038960A
:1060700087FFF4CF9FBF08951092740284E9809344
:10608000BC00109272021092710280E88093BC00F2
:106090001092BD001092BA001092BB001092B9008D
:1060A0001092B8000E9416301092BB0085E88093D1
:1060B000BC0080916F02826080936F0208951F92EE
:1060C0000F920FB60F9211242F933F934F935F932C
:1060D0008F939F93EF93FF9380917402282F332720
:1060E000442755278F5F80937402F90127313105CA
:1060F00008F0B3C2EE59FF4F0C942C7980917202D4
:106100008C3090F4809172028F5F80937202809144
:106110007202E82FFF27EE0FFF1FEE0FFF1FE85858
:10612000F94F8585181654F7809172028C3070F003
:1061300010926E0210926D021092720285E08093AE
:10614000740280917102880F8D5A04C0809172028E
:10615000880F8E5A8093BB0085E874C280917202CA
:10616000E82FFF2783E0EE0FFF1F8A95E1F7E25348
:10617000F94F81818093BB0085E88093BC008091BA
:106180007202E82FFF27EE0FFF1FEE0FFF1FEE0F2B
:10619000FF1FE253F94F808180FF91C0809172020E
:1061A000E82FFF27EE0FFF1FEE0FFF1FEE0FFF1F61
:1061B000E253F94F8281882329F0809106068730C7
:1061C00008F45FC280916D0290916E02892B09F0F4
:1061D00058C280916B0290916C02892B09F051C2D8
:1061E0006EC08091720221E030E002C0220F331FA6
:1061F0008A95E2F780916B0290916C0228233923F3
:10620000232B79F080917202E82FFF27EE0FFF1FFA
:10621000EE0FFF1FEE0FFF1FE253F94F80E1848363
:106220000DC080917202E82FFF27EE0FFF1FEE0FC7
:10623000FF1FEE0FFF1FE253F94F1482809172028D
:10624000E82FFF2753E0EE0FFF1F5A95E1F7E253C7
:10625000F94F8481282F332743E0220F331F4A95BB
:10626000E1F780917202E82FFF2793E0EE0FFF1F06
:106270009A95E1F7E253F94F82818770822B8093E0
:10628000BB0085E88093BC002091720281E090E021
:1062900002C0880F991F2A95E2F720916D02309174
:1062A0006E0282239323892B51F086EC96E0909323
:1062B00078028093770288E080937902E2C184E0DB
:1062C00080C1E0917702F091780281918093BB00C8
:1062D00085E88093BC00F0937802E0937702809188
:1062E0007902815080937902882309F4CAC183E03E
:1062F00068C18091B900803351F58091750288237F
:1063000029F4809172028F5F8093750280917202EE
:10631000E82FFF2783E0EE0FFF1F8A95E1F7E25396
:10632000F94F838199278F7790708F3791057CF48F
:1063300080917202E82FFF27EE0FFF1FEE0FFF1F65
:10634000EE0FFF1FE253F94F83818F5F838310921B
:10635000740284E98093BC008AE090E090939201FB
:1063600080939101809172028F5F809372021092EC
:10637000740262C18091B9008034A9F180917102E8
:10638000E82FFF27EE0FFF1FEE0FFF1FEE0FFF1F7F
:10639000E253F94F83818F778383809171028F5FFE
:1063A00080937102809171028C30A0F01092710282
:1063B00010926C0210926B02809176028F5F809334
:1063C00076028C3038F01092760280916F028D7FC9
:1063D00080936F0280916F02816080936F021092B0
:1063E000740284E971C080917102E82FFF27EE0FDB
:1063F000FF1FEE0FFF1FEE0FFF1FE253F94F8381C8
:106400008068838380917102E82FFF27EE0FFF1FC2
:10641000EE0FFF1FEE0FFF1FE253F94F808180FF49
:106420002FC080917102E82FFF2753E0EE0FFF1F6E
:106430005A95E1F7E253F94F84819927009751F07B
:106440004097D9F586EC96E0909378028093770296
:1064500088E031C080917102992743E0880F991F2D
:106460004A95E1F78D52994F909378028093770285
:1064700090917102809176029817E1F483E01BC03D
:1064800080917102992733E0880F991F3A95E1F7BF
:106490008D52994F909378028093770280916F028A
:1064A00081FD06C09091710280917602981711F4D7
:1064B00082E001C081E0809379028091790281308D
:1064C00011F485E801C085EC8093BC0080917502D1
:1064D0008093700210927502D4C0E0917702F0911F
:1064E00078028091BB00808380917702909178023E
:1064F000019690937802809377028091790281507F
:1065000080937902823010F085EC58C0813011F40C
:1065100085E854C080916F0281FF2DC08091EB020D
:1065200080FD1DC080917102E82FFF2723E0EE0F50
:10653000FF1F2A95E1F7E253F94F86818A3F79F4EC
:1065400080917102E82FFF2793E0EE0FFF1F9A95CD
:10655000E1F7E253F94F8081816080830CC0809124
:106560007102E82FFF2783E0EE0FFF1F8A95E1F706
:10657000E253F94F1082809171028F5F8093710214
:10658000809171028C30A0F01092710210926C0216
:1065900010926B02809176028F5F809376028C302E
:1065A00038F01092760280916F028D7F80936F0297
:1065B0001092740284E98093BC0049C08093BC00AF
:1065C00086E0809374025DC088E9C4CD8091730237
:1065D000880F805FBFCD809173029927813091052C
:1065E00061F0823091051CF4892B21F04AC002979A
:1065F00039F047C080911201ADCD80911101AACD33
:1066000080911001A7CD80E8A5CD1092740284E995
:106610008093BC008AE090E0909392018093910176
:1066200080917302823088F4809173028F5F80932F
:10663000730282E18093740280916F028E7F809357
:106640006F0285EA8093BC001CC010927302809197
:106650006F02816080936F0214C01092740284E90B
:106660008093BC0080916F02816080936F028AE00A
:1066700090E0909392018093910110927202109297
:106680007102FF91EF919F918F915F914F913F9197
:106690002F910F900FBE0F901F9018951F93CF93BF
:1066A000DF93182F80911603882321F4809106022E
:1066B000882319F081E090E097C01D3008F092C067
:1066C0001123B1F0E12FFF2723E0EE0FFF1F2A95E2
:1066D000E1F7E253F94F35978081359688230CF026
:1066E00081C03897808180FD03C083E090E07CC04A
:1066F0008091C606823019F084E090E075C067E0B2
:1067000070E086EC96E00E94D02A9091CD06891721
:1067100019F085E090E068C080ED97E00E948E1649
:10672000EC0180916F0280FD05C0CE010E9497169A
:106730008823B9F3112319F48FEF90E00BC0212FB8
:1067400033272150304081E090E002C0880F991F2C
:106750002A95E2F790936E0280936D02A1E0B0E07B
:10676000EEECF6E040E050E06BE0CD01042E02C01C
:10677000880F991F0A94E2F720916D0230916E0202
:1067800082239323892B11F01182128261504F5F73
:106790005F4F389667FFE9CF109272021092740231
:1067A00080916F028E7F80936F0285EA8093BC0098
:1067B00080916F0280FD05C0CE010E94971688234C
:1067C000B9F380916D0290916E02892B29F0CE0170
:1067D0000E949716882311F380916D0290916E02AA
:1067E000009711F082E090E0DF91CF911F91089522
:1067F0000F931F93CF93DF93982F809116038823D5
:1068000021F480910602882319F081E090E092C083
:106810009D30A0F4992319F486E090E08BC0C92F35
:10682000DD27FE0133E0EE0FFF1F3A95E1F7E2535B
:10683000F94F35978081359687FD03C082E090E05F
:1068400079C03897808180FD03C083E090E072C0FA
:1068500080ED97E00E948E168C0180916F0280FD82
:1068600005C0C8010E9497168823B9F3219721E03B
:1068700030E0C90102C0880F991FCA95E2F79093D2
:106880006C0280936B02D901EEECF6E040E050E040
:106890006BE0CD01042E02C0880F991F0A94E2F725
:1068A00020916B0230916C0282239323892B11F08B
:1068B0001182128261504F5F5F4F389667FFE9CFB8
:1068C000109271021092C6061092CD0610927402B8
:1068D00080916F028E7F80936F0285EA8093BC0067
:1068E00080916F0280FD05C0C8010E949716882321
:1068F000B9F380916B0290916C02892B29F0C80149
:106900000E949716882311F38091C606823019F0F1
:1069100084E090E00FC067E070E086EC96E00E94B3
:10692000D02A9091CD06891719F085E090E002C039
:1069300080E090E0DF91CF911F910F91089589E160
:10694000A3E6B7E0EFE2F7E01182108232961196EB
:106950001C921E921296815087FFF6CF10928503EB
:106960001092840310928703109286031092890379
:106970001092880308951F920F920FB60F92112460
:106980000F931F932F933F934F935F936F937F9337
:106990008F939F93AF93BF93CF93DF93EF93FF9327
:1069A00080916A0682FDCFC0409186005091870099
:1069B00080917B0290917C02481B590B809186004C
:1069C0009091870090937C0280937B02CA018D5442
:1069D0009440A0917D02B0917E02835F9A4178F449
:1069E00080917D0280932E07149714F010929301EA
:1069F00081E090E090937E0280937D0207C2AD30EB
:106A0000B1050CF003C2CA018B5F9040845B9140DA
:106A100008F074C0425D5140FD01EA0FFB1FE15DCB
:106A2000F84F80819181FA01E81BF90BCF01F7FF44
:106A300003C0909581959F4F06975CF480911F034A
:106A4000883C20F480911F03865F01C088EC80930E
:106A50001F03FD01EA0FFB1FE15DF84F808191816B
:106A60009C01220F331F280F391F240F351F37FFBA
:106A700002C02D5F3F4FE901D595C795D595C795C4
:106A8000CA0101968C179D0714F4219706C0415046
:106A90005040C417D5070CF4219680911F03833C06
:106AA000E0F08D010A0F1B1FF801E15DF84F8081B6
:106AB00091819E01281B390BC90163E070E00E949F
:106AC000A578CB01880F991F860F971F0D59184F76
:106AD000D80111969C938E9307C0AA0FBB1FAD5986
:106AE000B84F11961C921E92E0917D02F0917E02A9
:106AF000EE0FFF1FE15DF84FD183C08320917D022F
:106B000030917E022F5F3F4F30937E0220937D02B3
:106B100080910201843108F079C12530310511F4EA
:106B20005D9A01C05D9880917D0290917E028630D1
:106B3000910511F45C9A01C05C98079711F45B9A77
:106B400065C15B9863C14091860050918700809138
:106B50007F0290918002481B590B80918600909192
:106B600087009093800280937F02CA018D549440E5
:106B70006091E902835F9A4108F07AC060937A02DB
:106B800080917A02843008F453C090912E0780914E
:106B90007A02981709F04CC05091EA025B3008F471
:106BA0003FC0109293011092E90240E05F31C0F0C3
:106BB000E42FFF27EE0FFF1F9F012B543D4FDF01F6
:106BC000A15DB84F8D919C91D9018D939C93DF016C
:106BD000AD59B84F8D919C91E153FD4F91838083C6
:106BE000E42FFF27EE0FFF1F9F01215D384FDF01CC
:106BF000AF57BD4F8D919C91D90111969C938E9367
:106C0000DF01A556BD4F8D919C91ED59F84F9183B1
:106C10008083842F8F5F482F8D3040F28093E9026C
:106C20008091EA028F3FB9F08F5F8093EA0213C030
:106C30008091EA02853620F08AE08093EA0202C061
:106C40001092EA02809102018A3011F0843110F032
:106C5000289A01C0289881E08093E9028091160368
:106C6000882309F0D3C080917A0280932E07CEC08A
:106C70006D3008F0A3C0CA018B5F9040845B9140E7
:106C800008F07EC0425D5140E62FFF27EE0FFF1F48
:106C9000EF57FD4F80819181FA01E81BF90BCF017D
:106CA00005960B97B0F48091EA028A3120F080912A
:106CB0001F03865F05C08B3028F080911F038E5F15
:106CC00080931F0380911F03893C18F088EC809308
:106CD0001F03E62FFF27EE0FFF1FEF57FD4F8081A9
:106CE00091819C01220F331F280F391F240F351F5C
:106CF00037FF02C02D5F3F4FE901D595C795D59568
:106D0000C795CA0101968C179D0714F4219706C0F8
:106D100041505040C417D5070CF4219680911F03B1
:106D20008E3BD8F0E62FFF27EE0FFF1FDF01AF5796
:106D3000BD4F8D919C919E01281B390BC90163E0C9
:106D400070E00E94A578CB01880F991F860F971FCE
:106D5000E556FD4F9183808308C0E62FFF27EE0F95
:106D6000FF1FE556FD4F118210828091E902E82F46
:106D7000FF27EE0FFF1FEF57FD4FD183C08309C0E0
:106D8000809102018A3011F0843110F0289A01C0FC
:106D9000289880910201843188F48091E90285303D
:106DA00011F45D9A05C05D98863011F45C9A05C0B7
:106DB0005C98873011F45B9A01C05B988091E9027E
:106DC000843120F48F5F8093E90220C08431F1F494
:106DD000809102018A3011F0843110F0289A01C0AC
:106DE00028988EE18093E9022CE0C3E6D7E0A5EB7A
:106DF000B2E0EFE2F7E08D919D919183808332962E
:106E0000198218822296215027FFF5CFFF91EF912A
:106E1000DF91CF91BF91AF919F918F917F916F91B2
:106E20005F914F913F912F911F910F910F900FBE46
:106E30000F901F901895EF92FF920F931F938091E0
:106E400023069927880F991F880F991F7C01002717
:106E5000F7FC0095102F8091730390917403A0911B
:106E60007503B0917603BC01CD01A80197010E9482
:106E7000DA783093B3052093B20580916B0390913B
:106E80006C03A0916D03B0916E03BC01CD01A8010C
:106E900097010E94DA783093B5052093B40580916C
:106EA000E9079091EA0797FD039695958795959543
:106EB00087959093B7058093B6058091F9079091D7
:106EC000FA0797FD039695958795959587959093E5
:106ED000B9058093B8058091840390918503209132
:106EE000460230914702821B930B9093BB0580931F
:106EF000BA058091110390911203A0911303B091F0
:106F00001403BC01CD0125E030E040E050E00E94D8
:106F1000DA783093BD052093BC05809140029091B2
:106F200041029093BF058093BE05809131039091FB
:106F300032039093C3058093C20580911D01909107
:106F40001E019093C5058093C40580911F03992766
:106F50009093C7058093C6058091F5079091F60739
:106F6000A091F707B091F8072091990130919A010B
:106F700040919B0150919C01BC01CD010E94DA78A7
:106F80003093C9052093C8058091CF069927909327
:106F9000CB058093CA058091D70699279093CD059C
:106FA0008093CC058091DF0699279093CF0580933D
:106FB000CE058091E70699279093D1058093D0055F
:106FC00080912102909122029093DB058093DA0553
:106FD00080916C0890916D089093DF058093DE0599
:106FE00080917008909171089093E1058093E0057D
:106FF0008091720899279093ED058093EC0580911C
:10700000FC039091FD039093EF058093EE05809132
:10701000FA039091FB039093F1058093F005809122
:107020004404882321F480914504882321F0809131
:10703000B105816003C08091B1058E7F8093B10559
:107040001F910F91FF90EF9008951F93CF93DF93BF
:10705000182FEB01809116038823A1F411501F3FD4
:1070600089F0D0932602C093250280912502909149
:107070002602892BD1F7CE018C0F9D1F0E94A316EB
:10708000115078F7DF91CF911F910895CF93DF933F
:10709000809102018D3011F40E943C1B10927A0005
:1070A00080914A0290914B029093B0078093AF0772
:1070B00080914802909149029093A1078093A00784
:1070C00080914602909147029093EF078093EE07DC
:1070D0002091420230914302C901880F991F880F05
:1070E000991F820F931F820F931F9093EA0780933B
:1070F000E9072091440230914502C901880F991F88
:10710000880F991F820F931F820F931F9093FA0786
:107110008093F9078FEC80937A00A0E2B3E0CCE093
:10712000D6E097E08991E82FFF27EE0FFF1FE15D82
:10713000F84F0190F081E02DE259FF4F1E161F0617
:107140001CF0E0E0F0E005C0EF3FF10514F0EFEFD8
:10715000F0E08C91282F3327E217F30714F48150C5
:1071600004C02E173F0714F48F5F8C939150119633
:1071700097FFD8CF809146069927AA27BB27BC0145
:10718000CD0124EC39E040E050E00E946678DC015B
:10719000CB018093B9019093BA01A093BB01B09346
:1071A000BC01809147069927AA27BB27BC01CD01C6
:1071B0000E946678DC01CB018093B5019093B60103
:1071C000A093B701B093B801DF91CF910895A0E0EB
:1071D000B0E0EDEEF8E30C94FB78882EC0E0D0E050
:1071E0007E016E0110924404469AD0937F03C093AF
:1071F0007E03D0937D03C0937C03D0937903C09327
:107200007803D0938903C0938803D0938703C093F6
:107210008603D0938503C09384031092A201109239
:10722000A10110923A020E94463884E690E00E9442
:10723000B0160E9446388091140680FF10C08091DD
:10724000130190911401875B934038F480911301EE
:10725000909114018E5E924010F40E94E21A0FE1A8
:107260008AE090E00E94B016809146029091470219
:10727000C80FD91F80914A0290914B02E80EF91E67
:107280008091480290914902C80ED91E015007FF13
:10729000E7CF9701205F3F4F369527953695279585
:1072A0003093890320938803C6014096969587956D
:1072B0009695879590938703809386036096F5E073
:1072C000D695C795FA95E1F7D0938503C0938403CB
:1072D00090938303809382033093810320938003F0
:1072E000882009F441C08091E9079091EA0797FF4F
:1072F00003C0909581959F4F6CE070E00E94A57847
:107300009B0170937F0360937E038091F9079091B6
:10731000FA0797FF03C0909581959F4F6CE070E04E
:107320000E94A57870937D0360937C038091F9059A
:107330009091FA059093790380937803B90184E0E2
:1073400090E00E94142E60917C0370917D0386E092
:1073500090E00E94142E609178037091790388E088
:1073600090E00E94142E65C084E090E00E940F2EF1
:1073700090937F0380937E0386E090E00E940F2E1F
:1073800090937D0380937C0388E090E00E940F2E11
:107390009C01909379038093780380917E03909170
:1073A0007F038150984050F480917C0390917D033D
:1073B0008150984018F421503440D8F187E19AE088
:1073C0009F938F9387E692E19F938F93E0912B0495
:1073D000F0912C0409958091E9079091EA0797FFB5
:1073E00003C0909581959F4F6CE070E00E94A57856
:1073F00070937F0360937E038091F9079091FA0761
:1074000097FF03C0909581959F4F6CE070E00E94BC
:10741000A57870937D0360937C038091F90590912A
:10742000FA0590937903809378030F900F900F9053
:107430000F901092B0071092AF071092A107109210
:10744000A0071092EF071092EE0784E690E00E94EA
:10745000B01680914202909143029C01220F331F8B
:10746000220F331F280F391F280F391F3093EA07C7
:107470002093E90780914402909145028C01000F0E
:10748000111F000F111F080F191F080F191F10934C
:10749000FA070093F90780912306C82EDD24EE2415
:1074A000FF24442737FD4095542FC701B6010E94A1
:1074B00066784B015C01609373037093740380934F
:1074C0007503909376039801442737FD4095542F18
:1074D000C701B6010E946678DC01CB0180936B0383
:1074E00090936C03A0936D03B0936E0380924F034F
:1074F00090925003A0925103B0925203809347039D
:1075000090934803A0934903B0934A031092430316
:107510001092440310924503109246038091150186
:1075200090911601A0911701B09118019093FC055C
:107530008093FB05109239021092380210923303A7
:107540001092340310923503109236038091310368
:10755000909132039093300380932F030E949063A5
:1075600082E390E090932602809325028091460664
:107570009927AA27BB27BC01CD0124EC39E040E0C4
:1075800050E00E946678DC01CB018856954CAF4FE5
:10759000BF4F8093B9019093BA01A093BB01B09300
:1075A000BC01809147069927AA27BB27BC01CD01C2
:1075B0000E946678DC01CB018856954CAF4FBF4FD7
:1075C0008093B5019093B601A093B701B093B80131
:1075D00010929E0110929D0180913103909132038F
:1075E000AA2797FDA095BA2F2091990130919A0171
:1075F00040919B0150919C01BC01CD010E94667895
:10760000DC01CB018093F5079093F607A093F70771
:10761000B093F80710922A031092290381E0809317
:1076200001010E94F9678091EB0284608093EB0274
:107630008FEF809367081092680880E28093690852
:10764000C0E2D3E0ACE0B6E007E08D91E82FFF2781
:10765000EE0FFF1FE15DF84F808191818259899380
:10766000015007FFF2CF84E680931F03809123022D
:10767000882311F0469A579A809188039091890344
:1076800080569940815C9B4228F08091440481603F
:10769000809344048091860390918703805699409B
:1076A000815C9B4228F08091440482608093440472
:1076B00080918403909185038C5291408957954025
:1076C00028F08091440484608093440480917E0378
:1076D00090917F038C529140835C914028F080917F
:1076E000440488608093440480917C0390917D03DE
:1076F0008C529140835C914028F0809144048061D9
:107700008093440480917803909179038050924053
:107710008355914028F08091440480628093440412
:10772000ECE0CDB7DEB70C941779A3E1B0E0EBE95C
:10773000FBE30C94F578809184039091850320916C
:10774000460230914702821B930B9093EF07809380
:10775000EE07809150029091510297FD07969C018F
:1077600053E0359527955A95E1F73093B00720936C
:10777000AF0780914E0290914F0297FD079643E02C
:10778000959587954A95E1F79093A1078093A00777
:107790003093BB072093BA079093B3078093B20747
:1077A0008091E9079091EA07AC01440F551F480FFB
:1077B000591F2091420230914302C901880F991F3D
:1077C000880F991F820F931F820F931F480F591F15
:1077D00057FF02C04D5F5F4F5595479555954795AB
:1077E0005093EA074093E9078091F9079091FA07CF
:1077F000AC01440F551F480F591F2091440230918E
:107800004502C901880F991F880F991F820F931F86
:10781000820F931F480F591F57FF02C04D5F5F4FE4
:1078200055954795559547955093FA074093F90715
:107830002091420230914302C901880F991F880F9D
:10784000991F820F931F820F931F9C01442737FDBE
:107850004095542F8091630390916403A091650338
:10786000B0916603820F931FA41FB51F809363031B
:1078700090936403A0936503B09366032091440240
:1078800030914502C901880F991F880F991F820FF7
:10789000931F820F931F9C01442737FD4095542F5F
:1078A00080915F0390916003A0916103B0916203A6
:1078B000820F931FA41FB51F80935F0390936003F3
:1078C000A0936103B09362038091C4079091C507B0
:1078D0002091420230914302820F931F9093C5077B
:1078E0008093C4078091F1079091F20720914402A0
:1078F00030914502820F931F9093F2078093F10716
:1079000080917A0390917B03019690937B038093FF
:107910007A038091F9059091FA05209178033091CE
:107920007903821B930B9C01442737FD4095542F0C
:1079300080915B0390915C03A0915D03B0915E0325
:10794000820F931FA41FB51F80935B0390935C036A
:10795000A0935D03B0935E038FEC80937A00109246
:107960000F0120914B0330914C0340914D035091F6
:107970004E0329873A874B875C8729543B46414011
:1079800050402CF028E43BE641E050E00DC08985F2
:107990009A85AB85BC85885B9449AE4FBF4F4CF44C
:1079A00028EB34E94EEF5FEF2D833E834F835887FA
:1079B00008C089859A85AB85BC858D839E83AF83FE
:1079C000B88720915303309154034091550350914F
:1079D00056032D873E874F87588B29543B4641409D
:1079E00050402CF028E43BE641E050E00DC08D858E
:1079F0009E85AF85B889885B9449AE4FBF4F4CF4E4
:107A000028EB34E94EEF5FEF29833A834B835C83A5
:107A100008C08D859E85AF85B88989839A83AB839D
:107A2000BC83A091EE07B091EF07BB8BAA8BFD0141
:107A3000CF01AA2797FDA095BA2FA0904303B0903D
:107A40004403C0904503D0904603A80EB91ECA1E39
:107A5000DB1EA0924303B0924403C0924503D09230
:107A60004603E090F507F090F6070091F7071091B4
:107A7000F807E80EF91E0A1F1B1FE092F507F092A7
:107A8000F6070093F7071093F807F0910603F98BB8
:107A9000FF2309F098C180910503882309F093C161
:107AA0008091140686FF8FC18091A0079091A10755
:107AB000AA2797FDA095BA2FBC01CD0129813A8153
:107AC0004B815C810E9466789B01AC0197FF04C0EA
:107AD0002150384F4F4F5F4F6BE055954795379585
:107AE00027956A95D1F78091A101682E7724882483
:107AF0009924CA01B901A40193010E946678DC01AE
:107B0000CB018093940390939503A0939603B09335
:107B10009703B7FF04C08150904FAF4FBF4F1C0178
:107B20002D013CE055944794379427943A95D1F72A
:107B300020929403309295034092960350929703BB
:107B40008091AF079091B007AA2797FDA095BA2F13
:107B5000BC01CD012D813E814F8158850E94667800
:107B600097FF04C06150784F8F4F9F4F2BE0959542
:107B70008795779567952A95D1F7A40193010E947F
:107B80006678DC01CB018093980390939903A093CE
:107B90009A03B0939B03B7FF04C08150904FAF4F3F
:107BA000BF4F9C01AD018CE05595479537952795C2
:107BB0008A95D1F7209398033093990340939A03C1
:107BC00050939B0380919403909195039093980711
:107BD00080939707809198039091990390939C07C5
:107BE00080939B0722193309440955092093980370
:107BF0003093990340939A0350939B03E20EF31E34
:107C0000041F151FE092F507F092F6070093F7079F
:107C10001093F8078091A0018823B1F457FF04C0A6
:107C20002F5F3F4F4F4F5F4F55954795379527959E
:107C3000A21AB30AC40AD50AA0924303B09244031D
:107C4000C0924503D09246032A893B8979010027D7
:107C5000F7FC0095102F8091980390919903A091C3
:107C60009A03B0919B03E80EF91E0A1F1B1FC8015F
:107C7000B70129813A814B815C810E9466789B0122
:107C8000AC0197FF04C02150384F4F4F5F4FBBE00E
:107C90005595479537952795BA95D1F78091A201CB
:107CA000A82EBB24CC24DD24CA01B901A60195016C
:107CB0000E946678DC01CB0180938C0390938D0346
:107CC000A0938E03B0938F03B7FF04C08150904FF1
:107CD000AF4FBF4F3C014D01ACE095948794779432
:107CE0006794AA95D1F760928C0370928D0380926D
:107CF0008E0390928F03C801B7012D813E814F8181
:107D000058850E94667897FF04C06150784F8F4F66
:107D10009F4FFBE09595879577956795FA95D1F7F5
:107D2000A60195010E946678DC01CB018093900347
:107D300090939103A0939203B0939303B7FF04C071
:107D40008150904FAF4FBF4FAC01BD01ECE0759536
:107D5000679557954795EA95D1F7409390035093CF
:107D6000910360939203709393032A893B8937FFB1
:107D700003C0309521953F4F21343105E4F1D40102
:107D8000C30197FE07C0B095A095909581959F4F30
:107D9000AF4FBF4F81389105A105B10584F4DB01D8
:107DA000CA0177FF07C0B095A095909581959F4F28
:107DB000AF4FBF4F81389105A105B105E4F081E0D7
:107DC00080932B0318C010929C0710929B0710926F
:107DD00098071092970710929003109291031092B7
:107DE00092031092930310928C0310928D031092C1
:107DF0008E0310928F038091900390919103A09134
:107E00009203B0919303BC01CD0124E630E040E041
:107E100050E00E94DA78E0908C03F0908D03E21A33
:107E2000F30AF092AE07E092AD0780918C03909137
:107E30008D03A0918E03B0918F03BC01CD0124E688
:107E400030E040E050E00E94DA78DA01C901209188
:107E50009003309191038C01021B130B1093A30725
:107E60000093A2078091990190919A01A0919B01A2
:107E7000B0919C01BC01CD0128E631E040E050E02A
:107E80000E9466782091F5073091F6074091F70738
:107E90005091F807261737074807590764F0261B43
:107EA000370B480B590B2093F5073093F607409397
:107EB000F7075093F8072091F5073091F6074091A6
:107EC000F7075091F80757FF0CC0260F371F481FC0
:107ED000591F2093F5073093F6074093F707509307
:107EE000F8076091A0077091A1076E0D7F1D9B019F
:107EF000442737FD4095542F8091470390914803C4
:107F0000A0914903B0914A03820F931FA41FB51F8C
:107F10008093470390934803A0934903B0934A0387
:107F200080910B0390910C03681B790BCB01AA275E
:107F300097FDA095BA2F29853A854B855C85820FE0
:107F4000931FA41FB51F80934B0390934C03A093E2
:107F50004D03B0934E03C090B501D090B601E090B0
:107F6000B701F090B801C816D906EA06FB06C4F4BA
:107F700088EA91E6A0E0B0E08C199D09AE09BF093E
:107F800080934B0390934C03A0934D03B0934E0307
:107F90008093470390934803A0934903B0934A0307
:107FA00022273327A9012C193D094E095F09809129
:107FB0004B0390914C03A0914D03B0914E03821757
:107FC0009307A407B507B4F4D701C601885A9146B0
:107FD000A040B04080934B0390934C03A0934D037B
:107FE000B0934E038093470390934803A0934903B3
:107FF000B0934A036091AF077091B007600F711F93
:108000009B01442737FD4095542F80914F03909159
:108010005003A0915103B0915203820F931FA41FEC
:10802000B51F80934F0390935003A0935103B093D7
:1080300052038091090390910A03681B790BCB01CD
:10804000AA2797FDA095BA2F2D853E854F85588983
:10805000820F931FA41FB51F809353039093540363
:10806000A0935503B0935603E090B901F090BA0184
:108070000091BB011091BC01E816F9060A071B0725
:10808000C4F488EA91E6A0E0B0E08E199F09A00B45
:10809000B10B8093530390935403A0935503B09373
:1080A000560380934F0390935003A0935103B093D2
:1080B000520322273327A9012E193F09400B510BE8
:1080C0008091530390915403A0915503B0915603AE
:1080D00082179307A407B507B4F4D801C701885ADB
:1080E0009146A040B0408093530390935403A093D3
:1080F0005503B093560380934F0390935003A0937E
:108100005103B09352038091430390914403A09193
:108110004503B09146038093570390935803A0936F
:108120005903B0935A038091530390915403A09143
:108130005503B09156038093730390937403A093F7
:108140007503B093760380914B0390914C03A091FB
:108150004D03B0914E0380936B0390936C03A093F7
:108160006D03B0936E0380914F0390915003A091E3
:108170005103B091520380936F0390937003A093C7
:108180007103B09372038091470390914803A091CB
:108190004903B0914A038093670390936803A093C7
:1081A0006903B0936A0380911B0190911C0197FDB4
:1081B000079633E0959587953A95E1F79093B00748
:1081C0008093AF078091190190911A0197FD07964E
:1081D00023E0959587952A95E1F79093A1078093E1
:1081E000A00780914A0290914B020F9734F488E1E6
:1081F0009CEF9093B0078093AF0780914A029091D3
:108200004B02079734F480E398EF9093B007809384
:10821000AF07209102012A30A9F480914A0290917F
:108220004B02835F934034F088EE93E09093B00765
:108230008093AF0780914A0290914B028A5F9340EE
:10824000DCF014C080914A0290914B02815D97400E
:1082500034F088EE93E09093B0078093AF0780915D
:108260004A0290914B02805E974034F080ED97E097
:108270009093B0078093AF07809148029091490294
:108280000F9734F488E19CEF9093A1078093A007A7
:108290008091480290914902079734F480E398EF67
:1082A0009093A1078093A0072A30A9F480914802F7
:1082B00090914902835F934034F088EE93E090936D
:1082C000A1078093A00780914802909149028A5F9C
:1082D0009340DCF014C08091480290914902815D86
:1082E000974034F088EE93E09093A1078093A00725
:1082F0008091480290914902805E974034F080ED71
:1083000097E09093A1078093A007E091AC01EE2342
:1083100009F4B7C040911B0150911C0180919C034E
:1083200090919D03481B590B5093A3034093A203C4
:1083300020911B0130911C01280F391F37FF02C00B
:108340002F5F3F4F3595279530939D0320939C03D6
:10835000413851051CF080E890E005C040585F4F5F
:1083600034F480E89FEF9093A3038093A2038E2FB1
:108370009927A091A203B091A303A89FA001A99F50
:10838000500DB89F500D112457FF02C0415F5F4F41
:1083900014E0559547951A95E1F78091AF079091B4
:1083A000B007840F951F9093B0078093AF0760913B
:1083B000190170911A0180919E0390919F03681B8F
:1083C000790B7093A1036093A00340911901509120
:1083D0001A01480F591F57FF02C04F5F5F4F559555
:1083E000479550939F0340939E03613871051CF09D
:1083F00080E890E005C060587F4F34F480E89FEF3C
:108400009093A1038093A0032E2F33278091A00384
:108410009091A103829FB001839F700D929F700D78
:108420001124AB0177FF02C0415F5F4FE4E0559537
:108430004795EA95E1F78091A0079091A107840FF5
:10844000951F9093A1078093A007A29FC001A39FAF
:10845000900DB29F900D11249C0180911B01909171
:108460001C01820F931F90931C0180931B0180912C
:10847000190190911A01860F971F90931A0180930A
:1084800019010091B2071091B3078091970790915D
:108490009807101611065CF59C0197FF04C022276F
:1084A0003327281B390BC901AA2797FDA095BA2F9E
:1084B0002091A001332744275527BC01CD010E94FC
:1084C00066789B01AC0197FF04C0215C3F4F4F4F82
:1084D0005F4F76E055954795379527957A95D1F773
:1084E0008091AD079091AE07820F931F27C097FF31
:1084F00003C0909581959F4FAA2797FDA095BA2F0D
:108500002091A001332744275527BC01CD010E94AB
:1085100066789B01AC0197FF04C0215C3F4F4F4F31
:108520005F4F66E055954795379527956A95D1F742
:108530008091AD079091AE07821B930B9093AE078D
:108540008093AD07E090BA07F090BB0780919B073E
:1085500090919C071E141F045CF59C0197FF04C0BA
:1085600022273327281B390BC901AA2797FDA0957D
:10857000BA2F2091A001332744275527BC01CD01F4
:108580000E9466789B01AC0197FF04C0215C3F4FBD
:108590004F4F5F4F96E055954795379527959A959C
:1085A000D1F78091A2079091A307820F931F27C054
:1085B00097FF03C0909581959F4FAA2797FDA0959F
:1085C000BA2F2091A001332744275527BC01CD01A4
:1085D0000E9466789B01AC0197FF04C0215C3F4F6D
:1085E0004F4F5F4F86E055954795379527958A956C
:1085F000D1F78091A2079091A307821B930B9093D0
:10860000A3078093A2078091140687FF44C099892D
:10861000992309F040C0809105038823E1F5A1E08A
:10862000EA16A1E0FA064CF08091AF079091B007EE
:108630008E0D9F1D805091400DC0B0E0EB16BFEF36
:10864000FB0664F48091AF079091B0078E0D9F1DDB
:1086500080509F4F9093B0078093AF07E1E00130C7
:108660001E074CF08091A0079091A107800F911FE9
:10867000805091400CC0FFEF00301F0764F48091E0
:10868000A0079091A107800F911F80509F4F90935A
:10869000A1078093A007A0E2B3E06CE076E057E08A
:1086A000FB018191BF01E82FFF27EE0FFF1FE15D66
:1086B000F84F0190F081E02DE259FF4FEF3FF105B7
:1086C00021F01CF0EFEFF0E004C0F7FF02C0E0E0A3
:1086D000F0E04C91242F3327E217F307B1F0CF01DC
:1086E000821B930B97FD079613E0959587951A9536
:1086F000E1F7242F280F2C93822F9927E817F907E9
:1087000014F4215001C02F5F2C935150119657FF44
:10871000C7CFE2E1CD5E0C941179809116038823D6
:1087200001F58091EB028C7F8093EB02A9E4B4E029
:10873000EEECF6E09BE080910602882309F48C932E
:108740008D91818312829150389697FFF4CF80915A
:108750000602882359F08091060281508093060218
:1087600005C08091EB0281608093EB02109272024F
:108770001092740280916F028E7F80936F0285EA5F
:108780008093BC00089580911606883F38F0EFEF83
:10879000F0E0E81BF109E05EFC4F80818093B201BC
:1087A0008091B201882329F0843618F084E6809302
:1087B000B20180911806883F38F0EFEFF0E0E81B37
:1087C000F109E05EFC4F80818093B0018091B0019F
:1087D000882329F0843618F084E68093B0018091D4
:1087E0002506883F38F0EFEFF0E0E81BF109E05E86
:1087F000FC4F80818093AB018091AB018B3010F4F2
:108800008AE002C08F3F11F48093AB018091500643
:10881000883F38F0EFEFF0E0E81BF109E05EFC4F35
:1088200080818093C6078091C607823010F481E072
:1088300002C08F3F11F48093C60780915206883F93
:1088400038F0EFEFF0E0E81BF109E05EFC4F8081CB
:108850008093EC078091EC07823010F481E002C035
:108860008F3F11F48093EC0780913D06883F38F0EC
:10887000EFEFF0E0E81BF109E05EFC4F80818093B0
:10888000C30780913E06883F38F0EFEFF0E0E81B29
:10889000F109E05EFC4F808180939D0780913F0647
:1088A000883F38F0EFEFF0E0E81BF109E05EFC4FA5
:1088B00080818093CB0790911706983F18F490938E
:1088C000B10109C0EFEFF0E0E91BF109E05EFC4FF8
:1088D00080818093B101983F18F49093B10109C051
:1088E000EFEFF0E0E91BF109E05EFC4F808180933F
:1088F000B10180911A06883F38F0EFEFF0E0E81BF5
:10890000F109E05EFC4F80818093AF0180911C06ED
:10891000883F38F0EFEFF0E0E81BF109E05EFC4F34
:1089200080818093AD0180912406883F38F0EFEF7D
:10893000F0E0E81BF109E05EFC4F80818093AE011E
:1089400080912606883F38F0EFEFF0E0E81BF10950
:10895000E05EFC4F80818093AA0180912706883FCA
:1089600038F0EFEFF0E0E81BF109E05EFC4F8081AA
:108970008093AC0180912806883F38F0EFEFF0E05B
:10898000E81BF109E05EFC4F80818093A901809192
:108990002906883F38F0EFEFF0E0E81BF109E05ED0
:1089A000FC4F80818093A80180912F06883F38F08A
:1089B000EFEFF0E0E81BF109E05EFC4F808180936F
:1089C000A60180913006883F38F0EFEFF0E0E81B19
:1089D000F109E05EFC4F80818093000380913106B5
:1089E000883F38F0EFEFF0E0E81BF109E05EFC4F64
:1089F00080818093FF0280913206883F38F0EFEF4C
:108A0000F0E0E81BF109E05EFC4F80818093FE02FC
:108A100080913306883F38F0EFEFF0E0E81BF10972
:108A2000E05EFC4F80818093FD0280914B06883F81
:108A300038F0EFEFF0E0E81BF109E05EFC4F8081D9
:108A40008093FC0280914C06883F38F0EFEFF0E015
:108A5000E81BF109E05EFC4F80818093FB0280916E
:108A60004D06883F38F0EFEFF0E0E81BF109E05EDB
:108A7000FC4F80818093FA0280914E06883F38F047
:108A8000EFEFF0E0E81BF109E05EFC4F808180939E
:108A9000F90280913406883F38F0EFEFF0E0E81BF0
:108AA000F109E05EFC4F80818093A501809138063A
:108AB000883F38F0EFEFF0E0E81BF109E05EFC4F93
:108AC00080818093A40180914006883F38F0EFEFC9
:108AD000F0E0E81BF109E05EFC4F80818093A30188
:108AE00080914306883F38F0EFEFF0E0E81BF10992
:108AF000E05EFC4F80818093A20180914406883F14
:108B000038F0EFEFF0E0E81BF109E05EFC4F808108
:108B10008093A10180914506883F38F0EFEFF0E0A7
:108B2000E81BF109E05EFC4F80818093A0018091F9
:108B30004A06883F38F0EFEFF0E0E81BF109E05E0D
:108B4000FC4F808180939F0180916506883F38F0BB
:108B5000EFEFF0E0E81BF109E05EFC4F80818093CD
:108B6000FC078091A601282F33272F5F3F4F8CE30E
:108B700098E2B9010E94A5787093B4016093B301A3
:108B8000809122068093ED07809121068093B4079F
:108B900080910003813011F0843049F481E090E04D
:108BA000909397018093960183E090E008C083E062
:108BB00090E0909397018093960181E090E09093EC
:108BC00095018093940190916706933320F181E0A1
:108BD0008093F802983F58F0EFEFF0E0E91BF109BD
:108BE000E05EFC4F8081823310F41092F802809195
:108BF0003A0890913B0897FF08C08091F8028823BB
:108C000021F080914404806803C0809144048F77F0
:108C10008093440402C01092F80280913A08909127
:108C20003B0897FF1DC0809116038823C9F08091EF
:108C3000F8028823A9F080910801909109018F5FC3
:108C40009F4F71F488E99AE390932602809325025E
:108C500080E094EA90930901809308011092F80251
:108C60008091F802882339F08091A201823D18F4A6
:108C7000825E8093A2010895A5E3B0E0E2E4F6E409
:108C80000C94F5780E94953B309102013C3010F431
:108C9000299A01C02998E0901703F0901803F9A2CF
:108CA000E8A28091B40799270A96E816F90614F409
:108CB00099A388A380911F03843608F05CC080913B
:108CC000B8039091B903009731F001979093B903DD
:108CD0008093B80307C0109216038091EB028F7E39
:108CE0008093EB023A3011F0343110F0289A01C031
:108CF00028988091EC029091ED02895E9340C0F13A
:108D000080912C06282F332739A328A38091EB02CA
:108D100080618093EB0280910806A82FBB27AA0FE1
:108D2000BB1FFD01ED59F84F118210828091090699
:108D3000282F3327220F331FC9018D59984FFC016B
:108D400011821082A15DB84F11961C921E92215D76
:108D5000384FD90111961C921E9280910B06E82F74
:108D6000FF27EE0FFF1FE15DF84F11821082D5C281
:108D700010921603D2C280911F038D3808F4CDC221
:108D80008091EB028F7E8093EB0290912D0682E31F
:108D9000989FC00111249093B9038093B803E8A170
:108DA000F9A1B9978CF080911603882369F080911E
:108DB000EC029091ED02FFEF8F3F9F0729F00196A3
:108DC0009093ED028093EC028091EC029091ED0281
:108DD0008F3F910509F038F510923B0310923C0348
:108DE00010923D0310923E03109237031092380305
:108DF0001092390310923A031092A4031092A50323
:108E00001092A6031092A7031092430310924403FA
:108E100010924503109246038A3F910549F481E080
:108E20008093BE0305C08091EB0282608093EB02C9
:108E300080910A06E82FFF27EE0FFF1FE15DF84F34
:108E400080819181813591050CF462C120911603D6
:108E5000222309F05DC1E0919601F0919701E95F4D
:108E6000F94F8181E82FFF27EE0FFF1FE15DF84FDB
:108E7000808191818C3491050CF422C18091BA03D8
:108E80008F5F8093BA03893C08F442C13C3010F4F0
:108E9000299801C0299A109216031092BA031092D1
:108EA000ED021092EC0240910806E42FFF27EE0F2E
:108EB000FF1FE15DF84F8081918187349105DCF4DB
:108EC000E0919401F0919501E95FF94F8181E82FDC
:108ED000FF27EE0FFF1FE15DF84F80819181019028
:108EE000F081E02DF7FF03C0F095E195FF4FE734E7
:108EF000F1050CF48AC051E0209194013091950164
:108F0000F901E95FF94F8181A82FBB27AA0FBB1F89
:108F1000A15DB84F8D919C9111978734910544F0D4
:108F2000E42FFF27EE0FFF1FE15DF84F8081918155
:108F30008D919C918734910574F080910806E82FFB
:108F4000FF27EE0FFF1FE15DF84F8081918187348D
:108F500091050CF052E0F901E95FF94F8181E82FAA
:108F6000FF27EE0FFF1FE15DF84F8081918186346E
:108F7000910574F480910806E82FFF27EE0FFF1F7C
:108F8000E15DF84F80819181873491050CF053E0C9
:108F9000F901E95FF94F8181E82FFF27EE0FFF1FED
:108FA000E15DF84F808191818A5B9F4F74F48091DD
:108FB0000806E82FFF27EE0FFF1FE15DF84F8081C5
:108FC0009181873491050CF054E0295F394FF90104
:108FD0008181E82FFF27EE0FFF1FE15DF84F8081B1
:108FE00091818A5B9F4F74F480910806E82FFF27D8
:108FF000EE0FFF1FE15DF84F80819181863491056E
:109000000CF455E0852F0E94502EE0919401F091D0
:109010009501E95FF94F8181E82FFF27EE0FFF1FD0
:10902000E15DF84F808191810190F081E02DF7FFA3
:1090300003C0F095E195FF4F7E97BCF48091080640
:10904000E82FFF27EE0FFF1FE15DF84F8081918130
:109050008A5B9F4F54F481E080935F0488EE93E035
:10906000909326028093250253C00E94262F0E94CF
:10907000192E80E00E945A0780912E060E94F475F6
:109080008091140680FF10C080911301909114010B
:10909000875B934038F480911301909114018E5EA8
:1090A000924010F40E94E21A1092230280E00E9483
:1090B000E73881E08093BD0380932302579A1FC055
:1090C00080819181855B9F4F0CF58091BA038F5F02
:1090D0008093BA03893CE0F03C3010F4299801C039
:1090E000299A109216031092BA031092ED02109270
:1090F000EC0281E00E94E73881E08093BD030E948A
:10910000262F68E770E00E94253802C02093BA033A
:1091100080910A06E82FFF27EE0FFF1FE15DF84F51
:10912000808191818B5A9F4F0CF0F7C020911603DC
:10913000E0919601F0919701222309F0CEC0E95FFA
:10914000F94F8181E82FFF27EE0FFF1FE15DF84FF8
:1091500080819181855B9F4F0CF0BCC08091BB03E7
:109160008F5F8093BB03893C08F4D7C02093BB0377
:1091700080914404882309F0A6C08091BD03882310
:1091800009F4A1C081E090E09093ED028093EC029D
:1091900081E0809316031092A4031092A50310920D
:1091A000A6031092A7031092430310924403109257
:1091B00045031092460310923F0310924003109211
:1091C00041031092420380912306E82EFF240027DA
:1091D00011278091E9079091EA079C01442737FD08
:1091E0004095542FC801B7010E946678DC01CB017D
:1091F0008093530390935403A0935503B093560365
:109200008091F9079091FA079C01442737FD40951A
:10921000542FC801B7010E946678DC01CB0180930E
:109220004B0390934C03A0934D03B0934E03809156
:10923000730390917403A0917503B09176038093AA
:109240004F0390935003A0935103B0935203809126
:109250006B0390916C03A0916D03B0916E038093AA
:10926000470390934803A0934903B0934A03109295
:109270003B0310923C0310923D0310923E03109268
:109280003703109238031092390310923A038091F9
:10929000EB0288608093EB02909166068FE0989FC6
:1092A000900111248091310390913203820F931F1A
:1092B00068E671E00E94A57897FD019695958795DF
:1092C000809377032AC08CED95E0909326028093DB
:1092D000250223C02093BB0320C0E95FF94F8181A1
:1092E000E82FFF27EE0FFF1FE15DF84F808191818E
:1092F0008C34910584F08091BC038F5F8093BC0314
:10930000893C58F0109216031092BC031092ED02A3
:109310001092EC0202C01092BC0380919301815024
:1093200080939301809193018F3F21F08091EB0214
:1093300084FF82C30E94C3438091C7039091C803F6
:109340009C01220F331F280F391FA0900806AA2D59
:10935000BB27AA0FBB1FFD01E15DF84F90901E06D1
:10936000492D552780819181849FF001859FF00DC3
:10937000949FF00D11242E0F3F1F37FF02C02D5F69
:109380003F4FB9017595679575956795AD59B84F7C
:1093900080911F06082F11278D919C91809F70014D
:1093A000819FF00C909FF00C11246E0D7F1D709327
:1093B000C8036093C7038091C9039091CA039C01BD
:1093C000220F331F280F391FB0900906AB2DBB2782
:1093D000AA0FBB1FFD01E15DF84F80819181849F41
:1093E000F001859FF00D949FF00D11242E0F3F1F6B
:1093F00037FF02C02D5F3F4FA90155954795559501
:109400004795AD59B84F8D919C91809F7001819F78
:10941000F00C909FF00C11244E0D5F1D5093CA0369
:109420004093C9039E012F5F3F4F8FE1E4ECF1E0D1
:10943000D90101900D928A95E1F78091F802882375
:1094400009F448C0CB0177FD0396DC01B595A795DB
:10945000B595A795CA0157FD0396FC01F595E795CB
:10946000F595E7958091ED01682F772767FD709559
:109470006A9F90016B9F300D7A9F300D112480916F
:109480000004482F552747FD50954E9FC0014F9F20
:10949000900D5E9F900D1124280F391F37FF02C0D9
:1094A000295F3F4F03E0359527950A95E1F7309303
:1094B0001E0320931D036E9F90016F9F300D7E9FB2
:1094C000300D11244A9FC0014B9F900D5A9F900D63
:1094D000112444C080916606082F1127DE01A00FD9
:1094E000B11FFD0197819093ED01020F131FD80169
:1094F0008C9180930004A92FBB27A7FDB095A69F50
:109500009001A79F300DB69F300D1124E82FFF2743
:10951000E7FDF095E49FC001E59F900DF49F900D4D
:109520001124280F391F37FF02C0295F3F4F13E076
:10953000359527951A95E1F730931E0320931D0367
:10954000A49F9001A59F300DB49F300D1124E69F7C
:10955000C001E79F900DF69F900D1124281B390B39
:1095600037FF02C0295F3F4FF3E035952795FA9505
:10957000E1F730931C0320931B0380910B06E82F27
:10958000FF27EE0FFF1FE15DF84F808191819095DD
:1095900081959F4F90931A0380931903833091050F
:1095A00014F0029705C0BFEF8E3F9B0734F402967C
:1095B00090931A038093190304C010921A03109217
:1095C00019038091FC039091FD032091F8033091E1
:1095D000F903820F931FC0901D03D0901E03C81A79
:1095E000D90AD0921E03C0921D038091FA03909174
:1095F000FB032091F6033091F703820F931F009134
:109600001B0310911C03081B190B10931C030093E0
:109610001B0380910A06E82FFF27EE0FFF1FE15D75
:10962000F84FE080F180E8E7F0E0EE0EFF1EF092E8
:109630001803E09217038091AB019927AA2797FDA1
:10964000A095BA2FBC01CD010E940E78DC01CB01A0
:1096500020E030E040E251E4BC01CD010E94AF7750
:10966000DC01CB01BC01CD010E94F177DC01CB0113
:109670008093F3078091AA018093CC078091A90180
:109680009927AA2797FDA095BA2FBC01CD010E946A
:109690000E78DC01CB0120E030E040E251E4BC0177
:1096A000CD010E94AF77DC01CB01BC01CD010E944E
:1096B000F177DC01CB018093A7078091A80180930B
:1096C000BC0780916B0480FF59C08091FC078138F2
:1096D00008F454C080916404992787FD9095292D42
:1096E0003327829FA001839F500D929F500D11241C
:1096F000C40ED51ED0921E03C0921D038091650436
:10970000992787FD9095829FB001839F700D929F4E
:10971000700D1124060F171F10931C0300931B03D9
:1097200080916604282F332727FD309580911903F7
:1097300090911A03820F931F90931A038093190339
:1097400080916804282F332727FD309580911906D2
:109750009927289FD001299FB00D389FB00D112463
:10976000B0939E01A0939D018091670499278E1567
:109770009F0524F490931803809317038091170397
:109780009091180397FF04C01092180310921703CA
:109790008091140682FF02C01092CC0740911D03F5
:1097A00050911E03CA0157FD03969C0135952795DC
:1097B0003595279537FF03C0309521953F4F809110
:1097C000F0029091F10282179307B4F4CA0157FF97
:1097D00003C0909581959F4F97FD0396959587952A
:1097E000959587959093F1028093F00285369105C7
:1097F00044F084E690E001C001979093F1028093D9
:10980000F00240911B0350911C03CA0157FD0396BF
:109810009C01359527953595279537FF03C03095E1
:1098200021953F4F8091EE029091EF0282179307AE
:10983000B4F4CA0157FF03C0909581959F4F97FDDF
:10984000039695958795959587959093EF028093CC
:10985000EE028536910544F084E690E001C0019760
:109860009093EF028093EE028091EB0284FF08C098
:109870001092F1021092F0021092EF021092EE029A
:10988000EB2DFF27EE0FFF1FE15DF84F40914106E2
:10989000242F3327808191812817390744F4809140
:1098A000680682FF04C081E08093040313C0EB2D9F
:1098B000FF27EE0FFF1FE15DF84F842F99272091BE
:1098C0004206821B9109208131812817390714F43F
:1098D0001092040340910906E42FFF27EE0FFF1FAB
:1098E000E15DF84F50914106852F992722273327B4
:1098F000281B390B808191818217930744F4809152
:10990000680683FF04C081E08093030316C0809142
:109910000303882391F0E42FFF27EE0FFF1FE15D83
:10992000F84F809142069927851B9109208131814A
:109930008217930714F410920303EA2DFF27EE0F0A
:10994000FF1FE15DF84F40914106242F33278081AE
:1099500091812817390744F48091680680FF04C07C
:1099600081E08093010317C080910103882399F05F
:10997000EA2DFF27EE0FFF1FE15DF84F842F992797
:1099800020914206821B91092081318128173907D5
:1099900014F41092010340910806E42FFF27EE0F04
:1099A000FF1FE15DF84F50914106852F992722272F
:1099B0003327281B390B808191818217930744F448
:1099C0008091680681FF04C081E08093020316C085
:1099D00080910203882391F0E42FFF27EE0FFF1FF1
:1099E000E15DF84F809142069927851B91092081FE
:1099F00031818217930714F41092020380910403BB
:109A0000882319F480910303811181E08093050379
:109A100080910103882321F480910203882351F06F
:109A200081E08093060310920503109204031092C4
:109A3000030302C08093060380910503882321F469
:109A400080910603882369F0809140069927E8A158
:109A5000F9A18E179F0714F499A388A381E080933E
:109A60002B038091EB0284FF1AC010921A0310920C
:109A7000190310921E0310921D0310921C031092E2
:109A80001B039AE59093F30788E78093CC079093A4
:109A9000A7078093BC0710920503109206038091DC
:109AA000BF079091C007A091C107B091C207209154
:109AB0007303309174034091750350917603820FC4
:109AC000931FA41FB51F8093BF079093C007A09357
:109AD000C107B093C2078091C7079091C807A091B2
:109AE000C907B091CA0720906B0330906C03409077
:109AF0006D0350906E03820D931DA41DB51D8093C0
:109B0000C7079093C807A093C907B093CA0780916D
:109B1000B6079091B707A091B807B091B907E09048
:109B20006F03F09070030091710310917203EAA229
:109B3000FBA20CA31DA38E0D9F1DA01FB11F809320
:109B4000B6079093B707A093B807B093B907809171
:109B5000A8079091A907A091AA07B091AB07E09040
:109B60006703F09068030091690310916A03EEA205
:109B7000FFA208A719A78E0D9F1DA01FB11F8093DC
:109B8000A8079093A907A093AA07B093AB07F090FA
:109B90000603FAA6FF2029F480910503882309F41F
:109BA00060C01092630310926403109265031092D8
:109BB000660310925F03109260031092610310928B
:109BC00062031092BF071092C0071092C107109253
:109BD000C2071092C7071092C8071092C9071092C7
:109BE000CA071092B6071092B7071092B8071092E2
:109BF000B9071092A8071092A9071092AA0710920D
:109C0000AB078091530390915403A0915503B091F9
:109C1000560380934F0390935003A0935103B09346
:109C2000520380914B0390914C03A0914D03B0914E
:109C30004E038093470390934803A0934903B09346
:109C40004A03109237021092360210920A031092C1
:109C5000090310920C0310920B030AA5002309F0CC
:109C6000F2C180910503882309F0EDC18091F905C7
:109C70009091FA05815092402CF48091160388232C
:109C800009F4E1C190906708A09023066091E9076C
:109C90007091EA077BAB6AAB8091F9079091FA0764
:109CA0009DAB8CAB9FEF991609F4D9C0BB24CC2493
:109CB000DD24CA01B901A60195010E94DA78790173
:109CC0008A01EAA9FBA9CF01AA2797FDA095BA2F7F
:109CD000E81AF90A0A0B1B0BC201B101A601950192
:109CE0000E94DA7859016A012CA93DA9C901AA2765
:109CF00097FDA095BA2FA81AB90ACA0ADB0A292C1F
:109D0000332427FC3094432C532CC801B701A20103
:109D100091010E94667897FF04C061507E4F8F4F7B
:109D20009F4F3B014C0109E0959487947794679489
:109D30000A95D1F7C601B501A20191010E9466788A
:109D400097FF04C061507E4F8F4F9F4F5B016C01A6
:109D500019E0D594C794B794A7941A95D1F7809138
:109D6000F0029091F102813491053CF48091EE0271
:109D70009091EF0281349105D4F0D401C30197FE94
:109D800003C00196A11DB11D3C014D01959487941E
:109D900077946794D601C501D7FE03C00196A11D33
:109DA000B11D5C016D01D594C794B794A7948091BF
:109DB0000B06E82FFF27EE0FFF1FE15DF84F8081B4
:109DC00091810190F081E02DF7FF03C0F095E195BE
:109DD000FF4F7A97A4F0C401B30123E030E040E0E4
:109DE00050E00E94DA7839014A01C601B50123E04A
:109DF00030E040E050E00E94DA7859016A01809139
:109E00006908282F332727FD3095432F532F261518
:109E100037054805590514F439014A01992787FD8A
:109E20009095909581959F4FAA2797FDA095BA2F61
:109E3000681679068A069B0614F43C014D012A1522
:109E40003B054C055D0514F459016A01A816B906D5
:109E5000CA06DB060CF0CFC05C016D01CCC0EA2C59
:109E6000FF2400271127CA01B901A80197010E9408
:109E7000DA7839014A014AA95BA9CA01AA2797FDE4
:109E8000A095BA2F681A790A8A0A9B0AC201B10101
:109E9000A80197010E94DA7859016A016CA97DA98D
:109EA000CB01AA2797FDA095BA2FA81AB90ACA0A0A
:109EB000DB0AD401C30197FE03C00F96A11DB11D9B
:109EC0003C014D01F4E09594879477946794FA955A
:109ED000D1F7D601C501D7FE03C00F96A11DB11D54
:109EE0005C016D01E4E0D594C794B794A794EA951A
:109EF000D1F78091F0029091F102813491053CF408
:109F00008091EE029091EF0281349105A4F0C4019A
:109F1000B30123E030E040E050E00E94DA783901FC
:109F20004A01C601B50123E030E040E050E00E9464
:109F3000DA7859016A0180910B06E82FFF27EE0FAE
:109F4000FF1FE15DF84F808191810190F081E02D4C
:109F5000F7FF03C0F095E195FF4F7A97A4F0C40195
:109F6000B30123E030E040E050E00E94DA783901AC
:109F70004A01C601B50123E030E040E050E00E9414
:109F8000DA7859016A0171E267167104810491045B
:109F90002CF070E2672E712C812C912C80EE6816CB
:109FA0008FEF78068FEF88068FEF980644F460EE07
:109FB000662E6FEF762E6FEF862E6FEF962E91E264
:109FC000A916B104C104D1042CF050E2A52EB12C85
:109FD000C12CD12CA0EEAA16AFEFBA06AFEFCA067D
:109FE000AFEFDA0644F440EEA42E4FEFB42E4FEF5D
:109FF000C42E4FEFD42E8091530390915403A0911F
:10A000005503B091560386199709A809B909809399
:10A01000530390935403A0935503B0935603809138
:10A020004B0390914C03A0914D03B0914E038A19BC
:10A030009B09AC09BD0980934B0390934C03A093FB
:10A040004D03B0934E0380913602909137028F3FBB
:10A05000910509F008F4C4C5BAA5BB2309F04EC5A3
:10A0600080910503882309F049C580912B0388233B
:10A0700009F044C5E0914906EBA7EE2309F43EC57B
:10A080008091BF079091C007A091C107B091C2070E
:10A09000B7FF04C081509F4FAF4FBF4FE92EFA2E3C
:10A0A0000B2F112707FD1A95E092BF07F092C0070A
:10A0B0000093C1071093C2078091C7079091C8070A
:10A0C000A091C907B091CA07B7FF04C081509F4F44
:10A0D000AF4FBF4F892F9A2FAB2FBB27A7FDBA9544
:10A0E0008CA79DA7AEA7BFA78093C7079093C8076B
:10A0F000A093C907B093CA0780912306A82EBB245A
:10A10000CC24DD24209163033091640340916503E6
:10A1100050916603C601B5010E94667897FF04C09E
:10A1200061507F4F8F4F9F4F672E782E892E992435
:10A1300087FC9A9460926303709264038092650333
:10A140009092660320915F03309160034091610318
:10A1500050916203C601B5010E94667897FF04C062
:10A1600061507F4F8F4F9F4F272E382E492E5524F9
:10A1700047FC5A9420925F0330926003409261033F
:10A180005092620380915B0390915C03A0915D0308
:10A19000B0915E03B7FF04C081509F4FAF4FBF4FD8
:10A1A000892F9A2FAB2FBB27A7FDBA9580935B030E
:10A1B00090935C03A0935D03B0935E03D801C70145
:10A1C00086199709A809B9098093B0039093B10340
:10A1D000A093B203B093B30320914806E22EFF246C
:10A1E00000271127BC01CD01A80197010E94DA7850
:10A1F00059016A012093BF033093C0034093C10308
:10A200005093C2038CA59DA5AEA5BFA58219930945
:10A21000A409B5098093B4039093B503A093B60342
:10A22000B093B703BC01CD01A80197010E94DA7871
:10A230002093C3033093C4034093C5035093C603D4
:10A24000D601C501D7FE04C081509F4FAF4FBF4F0D
:10A25000892F9A2FAB2FBB27A7FDBA9590930A039E
:10A260008093090357FF04C021503F4F4F4F5F4F6A
:10A27000BB2757FDBA95A52F942F832F90930C03DE
:10A2800080930B038091F0029091F102813491054B
:10A29000DCF48091EE029091EF0281349105A4F4F8
:10A2A00080910B06E82FFF27EE0FFF1FE15DF84FAF
:10A2B000808191810190F081E02DF7FF03C0F0953E
:10A2C000E195FF4F7A97E4F0809167088F3FC1F4E2
:10A2D0008091090390910A0397FD019695958795C2
:10A2E00090930A038093090380910B0390910C03D0
:10A2F00097FD01969595879590930C0380930B039A
:10A300008091B6079091B707A091B807B091B907AF
:10A31000B7FF04C081509F4FAF4FBF4F892F9A2F77
:10A32000AB2FBB27A7FDBA958093B6079093B707CD
:10A33000A093B807B093B9078091A8079091A90797
:10A34000A091AA07B091AB07B7FF04C081509F4FFF
:10A35000AF4FBF4F892F9A2FAB2FBB27A7FDBA95C1
:10A360008093A8079093A907A093AA07B093AB077F
:10A370008091730390917403A0917503B09176035B
:10A380002AA13BA14CA15DA1281B390B4A0B5B0BF9
:10A390002093A8033093A9034093AA035093AB03DF
:10A3A00080916B0390916C03A0916D03B0916E034B
:10A3B000EEA0FFA008A519A5E81AF90A0A0B1B0BC5
:10A3C000E092AC03F092AD030093AE031093AF03A1
:10A3D0002093B0033093B1034093B2035093B3037F
:10A3E000E092B403F092B5030093B6031093B70361
:10A3F00080914F0390915003A0915103B09152036B
:10A40000821B930BA40BB50B80934F0390935003C7
:10A41000A0935103B0935203809147039091480356
:10A42000A0914903B0914A038E199F09A00BB10B6B
:10A430008093470390934803A0934903B0934A0342
:10A44000FBA5FF23E1F02091290330912A03213855
:10A4500031054CF08091840390918503019690938F
:10A4600085038093840320583F4F4CF480918403EC
:10A4700090918503019790938503809384031092B4
:10A480002A031092290381E090E09093CC038093FB
:10A49000CB03A090B003B090B103C090B203D090B2
:10A4A000B303D601C501D7FE07C088279927DC0171
:10A4B0008A199B09AC09BD0981509240A040B04067
:10A4C00034F084E090E09093CC038093CB038091B0
:10A4D000D1039091D203A091D303B091D4032091E2
:10A4E000BF073091C0074091C1075091C207821B3E
:10A4F000930BA40BB50B815E914BAF4FBF4F8F53A6
:10A500009C49A040B04028F08091680889310CF443
:10A51000FFC031E0A31630E1B30630E0C30630E0FF
:10A52000D3060CF473C08091CD03882309F46AC06C
:10A53000D601C501D7FE07C088279927DC018A19F3
:10A540009B09AC09BD099C01AD01B7FF04C02150B6
:10A550003E4F4F4F5F4FF9E05595479537952795FB
:10A56000FA95D1F78091CB039091CC03820F931F82
:10A570009093CC038093CB03D601C501D7FE03C0D3
:10A580000796A11DB11DE3E0B595A7959795879511
:10A59000EA95D1F78093BF039093C003A093C103C2
:10A5A000B093C20389589341A040B04064F088E85A
:10A5B00093E1A0E0B0E08093BF039093C003A09329
:10A5C000C103B093C2032091BF033091C0034091F7
:10A5D000C1035091C20357FF04C021503F4F4F4F5A
:10A5E0005F4F232F342F452F552747FD5A958091D4
:10A5F000090390910A03820F931F90930A0380939B
:10A60000090306C081E08093CD0302C01092CD0300
:10A6100050E0A51650EFB5065FEFC5065FEFD50613
:10A620000CF073C08091CE03882309F46AC0D60170
:10A63000C501D7FE07C088279927DC018A199B0925
:10A64000AC09BD099C01AD01B7FF04C021503E4FCC
:10A650004F4F5F4F69E055954795379527956A9518
:10A66000D1F78091CB039091CC03820F931F9093ED
:10A67000CC038093CB03D601C501D7FE03C0079658
:10A68000A11DB11D23E0B595A795979587952A95AE
:10A69000D1F78093BF039093C003A093C103B093FD
:10A6A000C20388579C4EAF4FBF4F64F488E79CEEBF
:10A6B000AFEFBFEF8093BF039093C003A093C1039C
:10A6C000B093C2032091BF033091C0034091C103F6
:10A6D0005091C20357FF04C021503F4F4F4F5F4F6F
:10A6E000232F342F452F552747FD5A958091090375
:10A6F00090910A03820F931F90930A03809309039A
:10A7000011C081E08093CE030DC01092CE030AC029
:10A710001092CC031092CB0388EE93E09093BE018D
:10A720008093BD017BA5272F33278091CB03909188
:10A73000CC032817390724F43093CC032093CB03A0
:10A74000E0916808EE2379F02E2F332727FD30950E
:10A750008091CB039091CC032817390724F43093D0
:10A76000CC032093CB034091B0035091B10360918F
:10A77000B2037091B303413851056105710574F05E
:10A7800080918803909189032091CB033091CC0371
:10A79000820F931F909389038093880340585F4FE3
:10A7A0006F4F7F4F74F480918803909189032091BB
:10A7B000CB033091CC03821B930B9093890380933E
:10A7C000880381E090E09093CC038093CB03A0902A
:10A7D000B403B090B503C090B603D090B703D601D0
:10A7E000C501D7FE07C088279927DC018A199B0974
:10A7F000AC09BD0981509240A040B04034F084E0E3
:10A8000090E09093CC038093CB038091D5039091FB
:10A81000D603A091D703B091D8032091C7073091F8
:10A82000C8074091C9075091CA07821B930BA40B1C
:10A83000B50B815E914BAF4FBF4F8F539C49A040EA
:10A84000B04018F0E9310CF4FFC011E0A11610E19E
:10A85000B10610E0C10610E0D1060CF473C080917F
:10A86000CF03882309F46AC0D601C501D7FE07C00B
:10A8700088279927DC018A199B09AC09BD099C012D
:10A88000AD01B7FF04C021503E4F4F4F5F4F09E06D
:10A8900055954795379527950A95D1F78091CB0324
:10A8A0009091CC03820F931F9093CC038093CB03A2
:10A8B000D601C501D7FE03C00796A11DB11D13E047
:10A8C000B595A795979587951A95D1F78093C3036A
:10A8D0009093C403A093C503B093C60389589341D2
:10A8E000A040B04064F088E893E1A0E0B0E080933D
:10A8F000C3039093C403A093C503B093C6032091F0
:10A90000C3033091C4034091C5035091C60357FF60
:10A9100004C021503F4F4F4F5F4F232F342F452FFF
:10A92000552747FD5A9580910B0390910C03820F98
:10A93000931F90930C0380930B0306C081E08093D8
:10A94000CF0302C01092CF0330E0A31630EFB3065E
:10A950003FEFC3063FEFD3060CF073C08091D003E6
:10A96000882309F46AC0D601C501D7FE07C088272D
:10A970009927DC018A199B09AC09BD099C01AD012D
:10A98000B7FF04C021503E4F4F4F5F4FE9E0559550
:10A99000479537952795EA95D1F78091CB0390910C
:10A9A000CC03820F931F9093CC038093CB03D601EB
:10A9B000C501D7FE03C00796A11DB11D73E0B59573
:10A9C000A795979587957A95D1F78093C303909330
:10A9D000C403A093C503B093C60388579C4EAF4FE2
:10A9E000BF4F64F488E79CEEAFEFBFEF8093C303E3
:10A9F0009093C403A093C503B093C6032091C303EF
:10AA00003091C4034091C5035091C60357FF04C061
:10AA100021503F4F4F4F5F4F232F342F452F552746
:10AA200047FD5A9580910B0390910C03820F931F61
:10AA300090930C0380930B0311C081E08093D003AB
:10AA40000DC01092D0030AC01092CC031092CB0319
:10AA500088EE93E09093BE018093BD015BA5252F06
:10AA600033278091CB039091CC032817390724F426
:10AA70003093CC032093CB0380916808882379F02E
:10AA8000282F332727FD30958091CB039091CC035D
:10AA90002817390724F43093CC032093CB0340913B
:10AAA000B4035091B5036091B6037091B703413878
:10AAB00051056105710574F08091860390918703BB
:10AAC0002091CB033091CC03820F931F9093870387
:10AAD0008093860340585F4F6F4F7F4FCCF4809137
:10AAE0008603909187032091CB033091CC03821B86
:10AAF000930B90938703809386030AC010920C03F4
:10AB000010920B0310920A031092090310922B0368
:10AB10008091CC07882341F410920C0310920B0310
:10AB200010920A03109209038091BF079091C00709
:10AB3000A091C107B091C2078093D1039093D20333
:10AB4000A093D303B093D4038091C7079091C80713
:10AB5000A091C907B091CA078093D5039093D603FB
:10AB6000A093D703B093D8031092630310926403A9
:10AB7000109265031092660310925F0310926003B7
:10AB8000109261031092620310925B0310925C03B7
:10AB900010925D0310925E031092BF071092C007DF
:10ABA0001092C1071092C2071092C7071092C807EF
:10ABB0001092C9071092CA071092B6071092B707F1
:10ABC0001092B8071092B9071092A8071092A9071F
:10ABD0001092AA071092AB07109237021092360219
:10ABE0000091190310911A03C80117FF04C08827A8
:10ABF0009927801B910B40976CF088EE93E090931F
:10AC0000BE018093BD018091140684FD03C081E0E4
:10AC10008093BE03F0902006AF2CBB24CC24DD240F
:10AC2000B801882777FD8095982F980117FF04C0F9
:10AC300022273327201B310B442737FD4095542F03
:10AC40000E9466789B01AC01C601B5010E9466783E
:10AC500097FF04C061507E4F8F4F9F4F59E09595ED
:10AC60008795779567955A95D1F79B018F2D9927F1
:10AC7000809FD001819FB00D909FB00D1124CD0118
:10AC8000B7FD03969595879595958795280F391F5C
:10AC9000442737FD4095542F2093A4033093A503F8
:10ACA0004093A6035093A7038091430390914403DC
:10ACB000A0914503B0914603821B930BA40BB50BE7
:10ACC0008093430390934403A0934503B0934603BA
:10ACD0008155934CA040B04064F080E593ECA0E037
:10ACE000B0E08093430390934403A0934503B09353
:10ACF00046038091430390914403A0914503B09192
:10AD00004603805B9C43AF4FBF4F64F480EB9CE3F2
:10AD1000AFEFBFEF8093430390934403A0934503A9
:10AD2000B0934603A0903103B0903203A114B10454
:10AD300009F478C18091140683FF74C18091730374
:10AD400090917403A0917503B0917603B7FF04C08E
:10AD500081509E4FAF4FBF4F29E0B595A79597956E
:10AD600087952A95D1F76C0197FF04C0D094C194C0
:10AD7000D108D39480916B0390916C03A0916D03E3
:10AD8000B0916E03B7FF04C081509E4FAF4FBF4FCD
:10AD900009E0B595A795979587950A95D1F7BC01D8
:10ADA00097FF03C0709561957F4FC616D7060CF4C8
:10ADB0006B01B601D7FE02C0695F7F4F2B0113E024
:10ADC000559447941A95E1F7B2E0EB2EF12C4E0C16
:10ADD0005F1C0CE112E0A00EB11E75010027F7FC0C
:10ADE0000095102F24EE3DEFA20EB31E8091F507C3
:10ADF0009091F607A091F707B091F807609099013C
:10AE000070909A0180909B0190909C01BC01CD01B3
:10AE1000A40193010E94DA78E21AF30A040B150BDD
:10AE2000C801B70128E631E040E050E00E94DA783E
:10AE3000DC01CB01ACE4EA2EAFEFFA2EE80EF91EEE
:10AE40000091BD011091BE010115110589F539E18F
:10AE5000C316D1046CF58091290390912A038E0DBD
:10AE60009F1D90932A03809329038091BE0388231A
:10AE7000F9F0C501AA2797FDA095BA2FBC01CD0115
:10AE8000A40193010E946678DC01CB018093F50751
:10AE90009093F607A093F707B093F807BC01CD0194
:10AEA0000E94DA783093300320932F031092BE0370
:10AEB000C701F4E0880F991FFA95E1F7B2010E94EB
:10AEC000A578CB01AA2797FDA095BA2F2091F50769
:10AED0003091F6074091F7075091F807280F391F76
:10AEE0004A1F5B1F2093F5073093F6074093F7073F
:10AEF0005093F807F090AE016F2D7727C69EC001E2
:10AF0000C79E900DD69E900D112497FD4F966C0113
:10AF1000E5E0D594C794EA95E1F76C197D096B01DA
:10AF200077FD7AC00115110509F06FC00091F0029C
:10AF30001091F1028091EE029091EF02080F191F1B
:10AF400017FF02C0095F1F4F73E0159507957A95AB
:10AF5000E1F7005C1F4FCA01B901A40193010E94EF
:10AF6000DA78DA01C90120912F03309130034427A8
:10AF700037FD4095542F821B930BA40BB50B845EB9
:10AF80009D4FAF4FBF4FBC01CD0128E631E040E0FF
:10AF900050E00E94DA78DC01CB01845B90408C9D0C
:10AFA000A0018D9D500D9C9D500D1124CA01B8012A
:10AFB0000E94A57883E0F89E60011124C616D7068A
:10AFC00014F4B60108C0882799278C199D096817C1
:10AFD00079070CF4BC019B01442737FD4095542FA1
:10AFE0008091430390914403A0914503B09146039F
:10AFF000820F931FA41FB51F8093430390934403B4
:10B00000A0934503B09346030DC001501040109328
:10B01000BE010093BD0106C084EF91E09093BE0194
:10B020008093BD0180912B03882381F01092370318
:10B03000109238031092390310923A0310923B0396
:10B0400010923C0310923D0310923E037090060351
:10B050007720F1F48091CC07282F332744275527F8
:10B060008091730390917403A0917503B09176035E
:10B07000BC01CD010E946678DC01CB01BC01CD0191
:10B0800028EF3AE240E050E00E94DA78290102C05D
:10B0900044245524909005039920F1F48091CC0725
:10B0A000282F33274427552780916B0390916C03F9
:10B0B000A0916D03B0916E03BC01CD010E94667832
:10B0C000DC01CB01BC01CD0128EF3AE240E050E0C9
:10B0D0000E94DA78190102C0222433248091A20749
:10B0E0009091A307893C91051CF088EC90E005C085
:10B0F00088539F4F34F488E39FEF9093A307809386
:10B10000A2078091AD079091AE07893C91051CF094
:10B1100088EC90E005C088539F4F34F488E39FEF9C
:10B120009093AE078093AD078091AF079091B007E1
:10B13000AA2797FDA095BA2F2091F307A22EBB2432
:10B14000CC24DD24BC01CD01A60195010E946678C6
:10B150009B01AC018091A2079091A307AA2797FDBC
:10B16000A095BA2F67E0880F991FAA1FBB1F6A9589
:10B17000D1F7280F391F4A1F5B1F57FF04C0215CFE
:10B180003F4F4F4F5F4F06E05595479537952795B1
:10B190000A95D1F77201E20EF31EF092B007E09229
:10B1A000AF078091A0079091A107AA2797FDA095CE
:10B1B000BA2FBC01CD01A60195010E9466789B01C2
:10B1C000AC018091AD079091AE07AA2797FDA0959D
:10B1D000BA2F17E0880F991FAA1FBB1F1A95D1F726
:10B1E000280F391F4A1F5B1F57FF04C0215C3F4FC8
:10B1F0004F4F5F4FB6E05595479537952795BA95D0
:10B20000D1F78101020F131F1093A1070093A0072C
:10B210008091EE079091EF07880F991FAA2797FD5D
:10B22000A095BA2F2091A707332744275527BC01A3
:10B23000CD010E9466785B016C0197FF08C08FE327
:10B2400090E0A0E0B0E0A80EB91ECA1EDB1EA6E08A
:10B25000D594C794B794A794AA95D1F78091BC07C9
:10B26000282F33274427552780915703909158035F
:10B27000A0915903B0915A03BC01CD010E94667898
:10B28000DC01CB01BC01CD0120EF35E540E050E011
:10B290000E94DA78B501620F731F7093EF07609315
:10B2A000EE0791E0E91690E1F90634F080E090E1D4
:10B2B0009093B0078093AF078091AF079091B0074C
:10B2C0008050904F34F480E090EF9093B0078093DB
:10B2D000AF070150104134F080E090E19093A10756
:10B2E0008093A0078091A0079091A1078050904F74
:10B2F00034F480E090EF9093A1078093A007615011
:10B30000704134F080E090E19093EF078093EE0776
:10B310008091EE079091EF078050904F34F480E0D9
:10B3200090EF9093EF078093EE0780910001482FF4
:10B33000552780911D0190911E014817590794F4DB
:10B3400020911D0130911E0168A179A1649FC00167
:10B35000659F900D749F900D1124B9010E94917802
:10B3600079A368A388A199A1880F991F880F991FB5
:10B3700099A388A34091140640FFA7C6992009F01D
:10B38000A4C6772009F0A1C6CC24DD244601809113
:10B390000703909108039093DD058093DC052091CD
:10B3A0008A0330918B032115310509F03FC080914C
:10B3B0001301909114018959934058F087B5853F46
:10B3C00020F480913A02815011C081E08093E4031F
:10B3D0004EC080911301909114018436910508F5B7
:10B3E00087B58B30D0F080913A028F5F80933A021C
:10B3F0009AE089029001112480910306821B87BD87
:10B400008CE291E090932602809325028EE591E0F4
:10B4100090938B0380938A032AC081E08093E30397
:10B4200026C07092E3037092E40321C0809111035F
:10B4300090911203A0911303B0911403E4E0880FDC
:10B44000991FAA1FBB1FEA95D1F780933B029093E7
:10B450003C02A0933D02B0933E02D0923902C092CA
:10B4600038022150304030938B0320938A0320917F
:10B47000B10141FF24C02233D8F48091C30181502F
:10B480008093C3018F3FD9F510922C038091110353
:10B4900090911203A0911303B091140380930D03B4
:10B4A00090930E03A0930F03B093100381E004C0A8
:10B4B00081E080932C0388EC8093C30120C08091AD
:10B4C0009D0190919E01820F911D209119063327B5
:10B4D000829FF001839FF00D929FF00D1124CF0108
:10B4E000AA2797FDA095BA2F80930D0390930E0382
:10B4F000A0930F03B093100381E080932C038091FD
:10B50000730390917403A0917503B0917603E0905A
:10B510009901F0909A0100919B0110919C01BC014E
:10B52000CD01A80197010E94DA7859016A01809142
:10B530006B0390916C03A0916D03B0916E03BC01FD
:10B54000CD01A80197010E94DA78B901C5010E94D6
:10B55000AC6F3C01CC971CF07CE3672E712CC301CF
:10B560000E94A76B3C0180E28093980180912C039C
:10B57000882309F436C48091EB0299279C0120713D
:10B58000307084FD2EC460916A0660FD04C0809115
:10B59000140681FD07C008A119A13093DA03209396
:10B5A000D90397C18091EB0281FF69C14091BF012E
:10B5B0005091C001CA010F962091170330911803D2
:10B5C00082179307ACF58091E303882389F5809176
:10B5D000E50381FF13C08D7F8093E5038091110304
:10B5E00090911203A0911303B091140380930D0363
:10B5F00090930E03A0930F03B09310038091E50383
:10B6000081608093E503241B350B2F50304037FFBA
:10B6100003C0309521953F4F8091D9039091DA0373
:10B62000820F931F9093DA038093D9038BE26EC04D
:10B63000CA010F9728173907ACF58091E4038823D6
:10B6400089F58091E50380FF13C08E7F8093E50329
:10B650008091110390911203A0911303B0911403F0
:10B6600080930D0390930E03A0930F03B0931003E8
:10B670008091E50382608093E503241B350B215FF5
:10B680003F4F37FF03C0309521953F4F8091D9033D
:10B690009091DA03821B930B9093DA038093D90382
:10B6A0008DE234C02091E503822F9927837090703A
:10B6B000892B59F12C7F2093E5031092DA03109225
:10B6C000D90320911103309112034091130350913B
:10B6D000140320930D0330930E0340930F035093F4
:10B6E000100361FF06C084EF91E0909326028093DF
:10B6F000250280911503882341F423333105410548
:10B7000051051CF081E0809315038DE3809398012F
:10B710002091D9033091DA03C90137FF04C088278B
:10B720009927821B930B815092400CF491C0809119
:10B7300019069927289FA001299F500D389F500D69
:10B740001124CA0160E075E00E94A578CB01AA2708
:10B7500097FDA095BA2F20910D0330910E034091D3
:10B760000F0350911003280F391F4A1F5B1F2093AE
:10B770000D0330930E0340930F0350931003109268
:10B78000DA031092D903A0901103B0901203C09075
:10B790001303D0901403D601C50180509440A040FB
:10B7A000B04082179307A407B5075CF4D601C50122
:10B7B00080509C4FAF4FBF4F281739074A075B0790
:10B7C00044F080930D0390930E03A0930F03B09366
:10B7D000100380916A0681FF06C084E690E0909392
:10B7E00026028093250280911D06882389F54091C9
:10B7F00007035091080357FF02C04D5F5F4F5595F7
:10B8000047955595479580911D0190911E01209176
:10B8100000013327489FB001499F700D589F700D5C
:10B820001124CB01B9010E94A5787093C0016093E7
:10B83000BF01663471051CF486E490E005C06739E9
:10B84000710534F086E990E09093C0018093BF01C8
:10B8500080918A0390918B03892BB9F18091110318
:10B8600090911203A0911303B091140380930D03E0
:10B8700090930E03A0930F03B093100326C0809102
:10B88000110390911203A0911303B09114038059F6
:10B890009140A040B04080930D0390930E03A0937D
:10B8A0000F03B093100380911D06882311F0992790
:10B8B00002C088E790E09093C0018093BF0188A107
:10B8C00099A19093080380930703009107031091B7
:10B8D0000803A0901103B0901203C0901303D090FE
:10B8E000140320910D0330910E0340910F035091EA
:10B8F00010032A153B054C055D0524F080916A066E
:10B9000080FDB1C280918A0390918B03892B39F01D
:10B910000091070310910803CC24DD24D7C0D60181
:10B92000C501821B930BA40BB50B8093A8039093C6
:10B93000A903A093AA03B093AB038230E0E89E076B
:10B94000EFEFAE07EFEFBE072CF481E090E8AFEF2A
:10B95000BFEF09C08F5F9F47A040B04064F08FEFFA
:10B960009FE7A0E0B0E08093A8039093A903A09381
:10B97000AA03B093AB03C090A803D090A903809111
:10B98000B001282F3327442755278091A803909191
:10B99000A903A091AA03B091AB03BC01CD010E9401
:10B9A000667897FF04C0615E7F4F8F4F9F4F55E0D1
:10B9B00095958795779567955A95D1F76093A803E4
:10B9C0007093A9038093AA039093AB0365302EEF85
:10B9D00072072FEF82072FEF92072CF484E09EEF7F
:10B9E000AFEFBFEF09C0605074408040904064F0FA
:10B9F00080E094E0A0E0B0E08093A8039093A903D6
:10BA0000A093AA03B093AB038090A8039090A903DE
:10BA1000209138023091390237FF02C0295F3F4F31
:10BA200043E0359527954A95E1F74FEF22383407E3
:10BA30001CF421E83FEF05C02038310514F020E860
:10BA400030E0C901AA2797FDA095BA2F2091B20135
:10BA5000332744275527BC01CD010E94667897FF04
:10BA600004C06D5F7F4F8F4F9F4F22E09595879564
:10BA7000779567952A95D1F79B015FEF6130750740
:10BA80001CF420E03FEF06C06F3F710519F014F081
:10BA900020E031E08091E503882349F0C90137FDBA
:10BAA00003969C0135952795359527950DC0809176
:10BAB0006A0680FF09C0C90137FD07969C01A3E013
:10BAC00035952795AA95E1F7820E931E2091AF0137
:10BAD000222309F454C060913303709134038091A0
:10BAE00035039091360397FF04C061587F4F8F4F05
:10BAF0009F4FF7E09595879577956795FA95D1F7DC
:10BB00003327442755270E94667897FF04C0615E5B
:10BB10007F4F8F4F9F4FE5E0959587957795679578
:10BB2000EA95D1F76093A8037093A9038093AA03C1
:10BB30009093AB036138AFEF7A07AFEF8A07AFEFAF
:10BB40009A072CF480E89FEFAFEFBFEF0AC06F3F7A
:10BB500071058105910569F064F080E091E0A0E055
:10BB6000B0E08093A8039093A903A093AA03B09395
:10BB7000AB038091A8039091A903880E991E809130
:10BB8000AD01282F332780916B08992787FD909569
:10BB9000289FF001299FF00D389FF00D11249F017F
:10BBA000F7FF02C021583F4F220F232F221F330BD4
:10BBB000FFEF21383F071CF420E83FEF06C02F3F7E
:10BBC000310519F014F020E031E0820E931EC4011B
:10BBD000AA2797FDA095BA2FE0900703F0900803DD
:10BBE0009701442737FD4095542FBC01CD010E9499
:10BBF000667897FF04C061507E4F8F4F9F4F59E08A
:10BC000095958795779567955A95D1F7061B170BEC
:10BC10008091D9039091DA03892B09F060C01E143A
:10BC20001F040CF05CC09601D7FE03C0309521952F
:10BC30003F4F2D33310540F48091DD039091DE03B9
:10BC40008017910774F526C02C53304045E0369597
:10BC500027954A95E1F72031310510F02FE030E0CB
:10BC60004091DD035091DE031C141D04E4F480E1D7
:10BC700090E0821B930B489F9001499F300D589F85
:10BC8000300D112494E0369527959A95E1F7201709
:10BC9000310720F58091C1019091C2010817190761
:10BCA000F4F08C011CC0205F3F4F8091C101909146
:10BCB000C201829FB001839F700D929F700D11246D
:10BCC0009B0184E0369527958A95E1F74017510747
:10BCD00014F08A0104C00217130708F08901C80193
:10BCE000AA2797FDA095BA2F1DE0880F991FAA1FBC
:10BCF000BB1F1A95D1F79301442737FD4095542F68
:10BD0000BC01CD010E94DA782093AC033093AD03DF
:10BD10004093AE035093AF030091AC031091AD0379
:10BD20008091DB039091DC039C01220F331F280FCD
:10BD3000391F200F311F37FF02C02D5F3F4FA90170
:10BD400055954795559547955093DC034093DB03F4
:10BD500080911506282F3327220F331F220F331F00
:10BD6000241735076CF48091ED07282F3327220F15
:10BD7000331F220F331F205530404217530724F042
:10BD80003093DC032093DB0380916A0680FF14C0AC
:10BD90008091DB039091DC03A8A1B9A18A179B07CE
:10BDA00024F0B093DC03A093DB03E091DB03F0917C
:10BDB000DC03F9A3E8A357C028A139A12E193F0934
:10BDC00037FF02C02D5F3F4F359527953595279555
:10BDD000E090DB03F090DC03E20EF31EF9A2E8A290
:10BDE00042C080911D06882301F560910703709180
:10BDF000080377FF02C06D5F7F4F75956795759556
:10BE0000679540911D0150911E0180910001282FDE
:10BE10003327649FC001659F900D749F900D11247E
:10BE2000B9010E94A578CB0101C099279093C00168
:10BE30008093BF018091BF019091C001873491052B
:10BE40001CF486E490E005C08639910534F086E95B
:10BE500090E09093C0018093BF0108A119A11093B5
:10BE6000DC030093DB038091EB0299279C01227095
:10BE7000307081FF1CC18091DF039091E003A0919D
:10BE8000E103B091E2030097A105B10521F0809193
:10BE900015038130B1F428A139A1C901AA2797FD62
:10BEA000A095BA2F2EE0880F991FAA1FBB1F2A95B5
:10BEB000D1F78093DF039093E003A093E103B09365
:10BEC000E20380911503813019F482E08093150319
:10BED00048A159A1CA01AA2797FDA095BA2F93019D
:10BEE000442737FD4095542FBC01CD010E94667850
:10BEF000DC01CB018093AC039093AD03A093AE0320
:10BF0000B093AF03B7FF04C08150904EAF4FBF4F07
:10BF10005C016D018DE0D594C794B794A7948A9580
:10BF2000D1F7A092AC03B092AD03C092AE03D09211
:10BF3000AF036091EC027091ED025FE0603A75072B
:10BF400050F58091DF039091E003A091E103B0915F
:10BF5000E2039C01AD010AE0569547953795279578
:10BF60000A95D1F7821B930BA40BB50BA601950183
:10BF700014E0220F331F441F551F1A95D1F7820F6B
:10BF8000931FA41FB51F8093DF039093E003A0933A
:10BF9000E103B093E20360547F4118F58091DF0321
:10BFA0009091E003A091E103B091E2039C01AD0107
:10BFB000FCE05695479537952795FA95D1F7821B62
:10BFC000930BA40BB50BA6019501E2E0220F331FE2
:10BFD000441F551FEA95D1F7820F931FA41FB51F69
:10BFE00029C0809138029091390280913802909155
:10BFF000390297FF03C0909581959F4F8436910534
:10C000000CF58091DF039091E003A091E103B091E2
:10C01000E2039C01AD017EE0569547953795279543
:10C020007A95D1F7821B930BA40BB50B8A0D9B1D40
:10C03000AC1DBD1D8093DF039093E003A093E1034B
:10C04000B093E2038091DF039091E003A091E103BC
:10C05000B091E2036EE0B695A795979587956A959E
:10C06000D1F7909308038093070340911B06442364
:10C0700099F055279C01BA010E94A578C901861B39
:10C08000970B9093DE038093DD03260F371F3093C9
:10C09000C2012093C10119C01092DE031092DD038A
:10C0A0008FEF93E09093C2018093C1010EC0109274
:10C0B00015031092DF031092E0031092E103109237
:10C0C000E20330930803209307039091B40798ABE1
:10C0D000292F3327220F331F220F331F285D3F4F95
:10C0E000A8A1B9A12A173B0714F039A328A3B0913E
:10C0F000ED07B9AB8B2F9927880F991F880F991FD0
:10C1000080559040E8A1F9A18E179F0714F499A3D8
:10C1100088A380917002882321F4809172088F3F58
:10C12000A1F08091EC029091ED020297C09768F423
:10C13000E8A0F9A01E141F0444F481E090E090935D
:10C14000ED028093EC0239A328A308A119A1109352
:10C15000C1050093C0058091A4039091A503A0910F
:10C16000A603B091A70322E0880F991FAA1FBB1F47
:10C170002A95D1F7C090EE07D090EF07C81AD90AD8
:10C18000013A11058CF0C80117FD01969595879528
:10C190008C159D050CF46C01909581959F4FC816E8
:10C1A000D90694F46C0110C011E5C116D1041CF03D
:10C1B000E0E5CE2ED12C20EBC2162FEFD20624F4D0
:10C1C00070EBC72E7FEFD72E49A9242F3327220FDC
:10C1D000331F220F331FC90168A179A1861B970B5A
:10C1E0008C159D050CF46C0188A199A1821B930B01
:10C1F000C816D9060CF46C018091AF079091B00776
:10C2000060911D0370911E03861B970B9093BE07D0
:10C210008093BD07A090CC0720913B0330913C0355
:10C2200040913D0350913E03AA2041F0461A570A1F
:10C23000C201AA2797FDA095BA2F04C0AA2797FD8F
:10C24000A095BA2F280F391F4A1F5B1F20933B036D
:10C2500030933C0340933D0350933E0380913B0356
:10C2600090913C03A0913D03B0913E0381509A4FC1
:10C27000A040B04064F080E09AEFA0E0B0E080938E
:10C280003B0390933C03A0933D03B0933E03809106
:10C290003B0390913C03A0913D03B0913E0380503D
:10C2A0009640AF4FBF4F64F480E096E0AFEFBFEF32
:10C2B00080933B0390933C03A0933D03B0933E03D4
:10C2C000B0902A062B2D33278091BD079091BE0791
:10C2D000289F7001299FF00C389FF00C11249701C2
:10C2E000F7FE02C0295F3F4F790153E0F594E794D0
:10C2F0005A95E1F70091B3011091B40198014427D8
:10C3000037FD4095542F80913B0390913C03A091C1
:10C310003D03B0913E03BC01CD010E94DA78E20EEC
:10C32000F31E90909F01692D772788279927960102
:10C33000D7FE04C0222733272C193D0937FF02C03E
:10C340002F5F3F4F3595279548A159A1240F351FE1
:10C35000442737FD4095542F0E94667897FF04C00C
:10C36000615C7F4F8F4F9F4F26E09595879577951E
:10C3700067952A95D1F79B016E157F050CF47B011B
:10C38000309521953F4FE216F3060CF47901809128
:10C39000A0079091A10760911B0370911C03861B5D
:10C3A000970B90939F0780939E07209137033091BE
:10C3B00038034091390350913A03AA2041F0261ADC
:10C3C000370AC101AA2797FDA095BA2F04C0AA2752
:10C3D00097FDA095BA2F280F391F4A1F5B1F209386
:10C3E0003703309338034093390350933A038091D5
:10C3F000370390913803A0913903B0913A038150EB
:10C400009A4FA040B04064F080E09AEFA0E0B0E026
:10C410008093370390933803A0933903B0933A0382
:10C420008091370390913803A0913903B0913A037A
:10C4300080509640AF4FBF4F64F480E096E0AFEF7E
:10C44000BFEF8093370390933803A0933903B093E1
:10C450003A032B2D332780919E0790919F07289FA9
:10C46000D001299FB00D389FB00D11249D01B7FF59
:10C4700002C0295F3F4F5901B3E0B594A794BA9524
:10C48000E1F79801442737FD4095542F80913703F9
:10C4900090913803A0913903B0913A03BC01CD01CA
:10C4A0000E94DA78A20EB31E692D77278827992774
:10C4B0009601D7FE04C0222733272C193D0937FFE8
:10C4C00002C02F5F3F4F35952795E8A1F9A12E0FA8
:10C4D0003F1F442737FD4095542F0E94667897FFF1
:10C4E00004C0615C7F4F8F4F9F4FF6E09595879515
:10C4F00077956795FA95D1F79B016A157B050CF442
:10C500005B01309521953F4FA216B3060CF45901FB
:10C51000EEEC6E2EE6E07E2E75E8872E76E0972E06
:10C520006BE0362E5DEC452E57E0552ED4012C9154
:10C5300012160CF0DFC0203419F408A119A11EC096
:10C54000E8A1F9A1CF01AA2797FDA095BA2F33271B
:10C5500027FD3095432F532FBC01CD010E946678F3
:10C5600097FF04C0615C7F4F8F4F9F4F46E09595CA
:10C570008795779567954A95D1F78B01F4012181CD
:10C58000203419F40E0D1F1D22C0203C19F40E1981
:10C590001F091DC0C701AA2797FDA095BA2F3327F1
:10C5A00027FD3095432F532FBC01CD010E946678A3
:10C5B00097FF04C0615C7F4F8F4F9F4F36E095958A
:10C5C0008795779567953A95D1F7060F171FF40170
:10C5D0002281203419F40A0D1B1D22C0203C19F4BD
:10C5E0000A191B091DC0C501AA2797FDA095BA2FDE
:10C5F000332727FD3095432F532FBC01CD010E94D7
:10C60000667897FF04C0615C7F4F8F4F9F4F26E095
:10C6100095958795779567952A95D1F7060F171FFA
:10C62000F4012381203419F40C0D1D1D22C0203C7F
:10C6300019F40C191D091DC0C601AA2797FDA09564
:10C64000BA2F332727FD3095432F532FBC01CD013F
:10C650000E94667897FF04C0615C7F4F8F4F9F4FA9
:10C66000B6E09595879577956795BA95D1F7060FBA
:10C67000171FD2018D919C91801791075CF4BC012A
:10C68000600F711F77FF02C06F5F7F4F8B011595A1
:10C69000079504C0000F111F081B190BB8A98B2F99
:10C6A0009927880F991F880F991F8017910754F4B5
:10C6B000E9A98E2F9927880F991F880F991F0817AE
:10C6C00019070CF08C01C80117FD03969595879505
:10C6D00095958795F3018183880F991F880F991F7E
:10C6E0009801281B390BC901880F8283D2010D9351
:10C6F0001C9303C0F301118212823A9402E010E00D
:10C70000400E511E24E030E0820E931E48E050E0BF
:10C71000640E751E37FE0ACFE2E1CB5C0C941179F2
:10C720008091F2039091F303A091F403B091F5038B
:10C730008093EA039093EB03A093EC03B093ED0393
:10C740008091EE039091EF03A091F003B091F1037B
:10C750008093E6039093E703A093E803B093E90383
:10C7600008951092FD031092FC031092FB031092A7
:10C77000FA03089584B1806A84B93D9A82E58CBD3C
:10C780001DBC459A81E08093FF078AEA80931008D8
:10C7900083E8809311088AE08093120810921408AD
:10C7A00010921308109216081092150810926A0839
:10C7B0001092320808953091FF07332309F085C0A5
:10C7C0000DB407FE82C084E080932402459A2EB502
:10C7D0008091010499278130910589F0823091057B
:10C7E0001CF4892B21F03EC00297B9F03BC0309376
:10C7F0003108209302042138A9F581E008C02535CD
:10C8000049F480910204820F8093020482E08093B5
:10C81000010428C03093010425C080913108E82F1D
:10C82000FF27E35BF74F20838F5F80933108909160
:10C8300002048A31A0F0291769F48AE1ADE4B8E076
:10C84000E3E3F8E00D9001928A95E1F781E08093AF
:10C85000320802C0309332081092010403C0920FD4
:10C860009093020420910F08203208F028C04598C8
:10C8700000000000000000000000000000000000B8
:10C8800000000000000000000000000000000000A8
:10C890000000000000000000000000000000000098
:10C8A000E0910808F0910908E20FF11D80818EBD2A
:10C8B00080912F089081890F80932F0803C081E019
:10C8C0008093FF072F5F20930F080895EF92FF9248
:10C8D0000F931F93809123069927880F991F880F24
:10C8E000991F7C010027F7FC0095102F809173039E
:10C8F00090917403A0917503B0917603BC01CD01B2
:10C90000A80197010E94DA78309314082093130845
:10C9100080916B0390916C03A0916D03B0916E03B5
:10C92000BC01CD01A80197010E94DA783093160866
:10C93000209315082091F5073091F6074091F707ED
:10C940005091F807DA01C901E3E0880F991FAA1F87
:10C95000BB1FEA95D1F7820F931FA41FB51F820F4B
:10C96000931FA41FB51F2091990130919A01409106
:10C970009B0150919C01BC01CD010E94DA7830935B
:10C980001C0820931B0880918403909185032091BB
:10C99000460230914702821B930B909322088093AA
:10C9A0002108E0917A03F0917B038091C407909174
:10C9B000C507BF010E94A578CB019B01220F331F41
:10C9C000220F331F280F391F280F391F37FF02C0CE
:10C9D0002D5F3F4F3595279535952795309318084E
:10C9E000209317088091F1079091F207BF010E94F0
:10C9F000A5789B01220F331F220F331F260F371FED
:10CA0000260F371F37FF02C02D5F3F4F3595279503
:10CA10003595279530931A082093190810927B03B7
:10CA200010927A031092C5071092C4071092F20771
:10CA30001092F1078091120899278D30910509F421
:10CA400066C08E3091055CF48B30910509F48EC080
:10CA50008C3091050CF00FC10A9761F0A8C18F309E
:10CA6000910509F47CC18F3091050CF45CC14097AD
:10CA700099F19DC180910003809323088091FF026A
:10CA8000809324088091FE02809325088091FD0206
:10CA9000809326088091FC02809327088091FB02F6
:10CAA000809328088091FA02809329088091F902E6
:10CAB00080932A088091EB0280932B088091EB02EF
:10CAC000837F8093EB020E94262F80932C08809115
:10CAD000770380932D086BC180916C0890916D084D
:10CAE0009093240880932308809170089091710896
:10CAF000909326088093250880911D0190911E0136
:10CB000080932708809100018093280850C180916C
:10CB100055068093230880915606809324088091BF
:10CB200057068093250880915806809326088091A7
:10CB300059068093270880915D068093280880918C
:10CB40005E068093290880915F0680932A08809171
:10CB5000620680932B088091600680932C08809158
:10CB6000610680932D0880916306DAC0F894809165
:10CB70000A06E82FFF27EE0FFF1FE15DF84F019037
:10CB8000F081E02DE038F1051CF0EFE7F0E006C0A1
:10CB90002FEFE138F20714F4E1E8FFEFE093230808
:10CBA00080910B06E82FFF27EE0FFF1FE15DF84F86
:10CBB0000190F081E02DE038F1051CF0EFE7F0E0A6
:10CBC00006C06FEFE138F60714F4E1E8FFEFE093F9
:10CBD000240880910906E82FFF27EE0FFF1FE15D73
:10CBE000F84F0190F081E02DE038F1051CF0EFE7FF
:10CBF000F0E006C08FEFE138F80714F4E1E8FFEF4A
:10CC0000E093250880910806E82FFF27EE0FFF1F0D
:10CC1000E15DF84F0190F081E02DE038F1051CF066
:10CC2000EFE7F0E006C02FEFE138F20714F4E1E897
:10CC3000FFEF7894E09326088091200380932708E3
:10CC400080912103809328088091220380932908F2
:10CC50008091230380932A088091240380932B08DA
:10CC60008091250380932C088091260380932D08C2
:10CC70008091270355C080915F04863018F0109290
:10CC80005F0485E0809323088091640680932408E4
:10CC90008091110390911203A0911303B09114039A
:10CCA000BC01CD0125E030E040E050E00E94DA78A0
:10CCB000309326082093250880910D0390910E0350
:10CCC000A0910F03B0911003BC01CD0125E030E02D
:10CCD00040E050E00E94DA7830932808209327083B
:10CCE00080915A068093290880915B0680932A08D8
:10CCF00080915C0680932B0880911F0380932C0801
:10CD000080912F079091300780932D088091C00566
:10CD10009091C10597FD0396959587959595879573
:10CD200080932E0844C01092230880E58093240845
:10CD300085E0809325088EE080932608809102018B
:10CD400080932708809144048093280880914504AB
:10CD5000809329088091460480932A0828C08091F6
:10CD60003C06809323088091690680932408809173
:10CD7000A50180932508809135068093260880912F
:10CD80003606809327088091370680932808809183
:10CD9000A401809329088091390680932A08809104
:10CDA0003A0680932B0880913B0680932C08809153
:10CDB0003208882309F4CFC08AEF8093EC014091B8
:10CDC000340850913508CA0181509E4F8F5F9340BF
:10CDD000B0F42091360830913708C90181509E4F38
:10CDE0008F5F934060F48091140685FF08C05093D4
:10CDF000FD034093FC033093FB032093FA038091DF
:10CE00003A0890913B0821E08936920724F49093E8
:10CE1000320380933103809131039091320320914A
:10CE20002F0330913003821B930B845E9D4F68E685
:10CE300071E00E94A578845B904090932E038093CC
:10CE40002D0320913E0830913F088091250290915A
:10CE500026028217930740F480915F04882321F40F
:10CE60003093260220932502809133089927883633
:10CE7000910549F18936910524F48736910531F001
:10CE800072C08936910509F445C06DC08091400893
:10CE900080936708809141088093690880914208D7
:10CEA000809368088091430880936A0880914408C1
:10CEB00080936B08809145088093ED01809146082E
:10CEC0008093000450C08091400880930A088091AC
:10CED000410880930B088091420880930C08809150
:10CEE000430880930D088091440880930E08809138
:10CEF000B00590914508892B8093B0059091460824
:10CF00009093FE038091B10583709C70892B809370
:10CF1000B10529C0809140088093000880914108A4
:10CF20008093010880914208809302088091430811
:10CF300080930308809144089091450890930508D8
:10CF400080930408809146089091470890930708C1
:10CF50008093060808C01092FD031092FC03109203
:10CF6000FB031092FA031F910F91FF90EF90089529
:10CF70008091FF07882309F43BC0459880E198E041
:10CF800090930908809308089091FF03E92FFF27E9
:10CF9000ED51FE4F9F5F9093FF03808180931208B5
:10CFA000993010F01092FF031092FF070E94666400
:10CFB00081E080930F0800000000000000000000E6
:10CFC0000000000000000000000000000000000061
:10CFD0000000000000000000000000000000000051
:10CFE0000000000000008091100880932F088EBD83
:10CFF000089587B18C6087B94298439810920404D1
:10D0000080E88093EF01109203048093EE0108956D
:10D01000809109048150809309048F3F09F0F4C086
:10D0200094E0909309048091EB02807BE1F0809181
:10D030005306882349F080910C04882311F49093BF
:10D04000040481E080930C04809154068823B9F095
:10D0500080910D04882319F484E08093030481E017
:10D0600080930D040CC080930C0480930D04809178
:10D070004F0680930A048091510680930B0480919F
:10D080000C04882309F040C080916806282F3327BC
:10D0900024FF07C080911603882319F425FD4DC095
:10D0A0004EC090915006983F50F08091C6078D3D3C
:10D0B00030F080910A0488230CF43FC040C0983FB0
:10D0C00048F08091C6078A3028F480910A048823AA
:10D0D000B4F133C0809104048150809304048F3FE5
:10D0E00079F58091C6078150809304048091EF0107
:10D0F000813011F480E801C086958093EF01809122
:10D10000EF0190910A0417C080910404815080932C
:10D1100004048F3FA9F489E0809304048091EF0117
:10D12000813011F480E801C086958093EF018091F1
:10D13000EF0190915306892311F0429A01C0429861
:10D1400080910D04882309F043C080916806282F40
:10D15000332724FF07C080911603882319F426FD86
:10D1600050C034C090915206983F50F08091EC0727
:10D170008D3D30F080910B0488230CF442C026C012
:10D18000983F48F08091EC078A3028F480910B0496
:10D190008823E4F036C08091030481508093030417
:10D1A0008F3F91F58091EC0781508093030480912B
:10D1B000EE01813011F480E801C086958093EE0184
:10D1C0008091EE0190910B048923D9F4439808953E
:10D1D000809103048150809303048F3FA9F489E078
:10D1E000809303048091EE01813011F480E801C046
:10D1F00086958093EE018091EE01909154068923EB
:10D2000011F0439A0895439808954FB724E130E010
:10D21000F8948091C9008F778093C9008091C900EC
:10D220008F7B8093C9008091C9008F7D8093C90056
:10D230005A9A52985B9A539A832F99278093CD00DC
:10D240002093CC008091C80082608093C80080E168
:10D250008093C9008091CA008F778093CA00809123
:10D26000CA008F7B8093CA008091CA008F7D809313
:10D27000CA008091CA008F7E8093CA008091CA0044
:10D28000877F8093CA008091C9008B7F8093C900FB
:10D290008091CA0084608093CA008091CA00826035
:10D2A0008093CA008091C80087FF03C08091CE00A0
:10D2B000F9CF8091C90080688093C9004FBF08955D
:10D2C000FF920F931F93CF93DF9380E197E20E9429
:10D2D0008E16EC01FF248091C9008F778093C900DE
:10D2E0008091C9008F7E8093C9005A988FE29AE09E
:10D2F0009F938F9307E612E11F930F93E0912B0406
:10D30000F0912C0409950F900F900F900F9002C090
:10D310004A996CC0CE010E9497168823C9F3E09108
:10D320002B04F0912C04FF2009F468C085E69AE0F4
:10D330009F938F931F930F930995529A0F900F907D
:10D340000F900F90CE010E9497168823D9F383E6A1
:10D3500090E05A9A019797FFFCCF8FE891E05A9896
:10D36000019797FFFCCF89E090E05A9A019797FFC9
:10D37000FCCF89E090E05A98019797FFFCCF8FE8A7
:10D3800091E05A9A019797FFFCCF8FE891E05A9865
:10D39000019797FFFCCF89E090E05A9A019797FF99
:10D3A000FCCF89E090E05A98019797FFFCCF8FE877
:10D3B00091E05A9A019797FFFCCF8FE891E05A9835
:10D3C000019797FFFCCF89E090E05A9A019797FF69
:10D3D000FCCF89E090E05A98019797FFFCCF8FE847
:10D3E00091E05A9A019797FFFCCF13C08AE590E02D
:10D3F0000E948E16EC0191E0F92E91CF8BE69AE017
:10D400009F938F931F930F9309950F900F900F90F9
:10D410000F9052985A980E940569E5E0CDB7DEB7A3
:10D420000C941E79EF92FF920F931F93CF93DF938B
:10D43000482F00E010E08091F001813061F41092FB
:10D44000F00184E480930E041092100410920F04F3
:10D45000109211042BC180910E04882319F421E04D
:10D4600030E001C0980190910F04992371F4232BAF
:10D4700011F081E010C084E480930E0490931004B6
:10D4800090930F0490931104FAC0913069F4232B08
:10D4900009F0EBC082E080930F04809110048F5F4D
:10D4A0008093100483E0E9C09230D1F4232B09F07B
:10D4B000DCC083E080930E0440931104909110042B
:10D4C000923039F41092120447FF03C081E0809338
:10D4D000120483E080930F049F5F90931004CFC0E9
:10D4E000933009F0C2C0232B09F0BFC090930E0403
:10D4F00082E080930F04809110048F5F809310046A
:10D5000020911104822F9927782F6627842F99273D
:10D51000682B792B80912E06813049F47370CB01F2
:10D520008050924063E070E00E94A57817C082307E
:10D5300061F47770CB018050944066E070E00E9407
:10D54000A5782695269526950BC073706856714070
:10D55000CB0177FD0196BC017595679526952695BB
:10D56000022F11270F7010700F5F1F4F0D30110524
:10D5700008F074C07801E00EF11EF701E15DF84F8C
:10D58000808191819B01281B390BC90137FF03C0A2
:10D59000909581959F4F069794F480911F03883C46
:10D5A00030F480911F03865F80931F0308C088ECCE
:10D5B00080931F0380916F008F7D80936F00F70130
:10D5C000E15DF84F808191819C01220F331F280F6C
:10D5D000391F260F371F37FF02C02D5F3F4FE9016C
:10D5E000D595C795D595C795CB0101968C179D0705
:10D5F00014F4219706C061507040C617D7070CF489
:10D60000219680911F03843BD0F0F701E15DF84F34
:10D6100080819181FE01E81BF90BCF0163E070E08E
:10D620000E94A578CB01880F991F860F971F23E6CC
:10D6300037E0E20EF31EF7019183808307C023E6F3
:10D6400037E0E20EF31EF70111821082000F111F66
:10D65000015D184FF801D183C08311C0023111055B
:10D6600070F081E08093F0010AC081E08093F001C6
:10D67000109210041092120484E480930E0480919E
:10D680001004803198F080911204882331F4809145
:10D69000F001882311F480939301109210041092EA
:10D6A000120410920F0484E480930E04E6E0CDB7D8
:10D6B000DEB70C941D79CF93FC0197FF05C0CFEF27
:10D6C000F095E195FF4F01C0C1E028E631E0CF01C0
:10D6D000B9010E94A578FC018B35910554F08B555A
:10D6E00090408A35910538F484EB90E08E1B9F0BB7
:10D6F000FC0141E00DC0CF01855B90408A3591056A
:10D7000018F4E45BF04003C02E1B3F0BF9014FEF10
:10D71000EE0FFF1FEA58F54F259134918C2F992772
:10D7200087FD9095289FB001299F700D389F700D3F
:10D730001124842F992787FD9095689FA001699FE8
:10D74000500D789F500D1124CA01CF9108952AE5FC
:10D7500030E0281B390BC9010E945B6B0895CF9301
:10D76000DF9380E00E94907180911D0190911E01D5
:10D770006AE070E00E94A5789F938F9380911D01CD
:10D7800090911E016AE070E00E94A5787F936F93EC
:10D7900084E49BE09F938F93C3E8D1E7DF93CF931B
:10D7A000E0912B04F0912C0409952DB73EB7285F2A
:10D7B0003F4F2DBF8091EC018823B9F186E00E9494
:10D7C000907180910408909105086AE070E00E94D1
:10D7D00091787F936F938FED90E09F938F938091DB
:10D7E000F5079091F607A091F707B091F8072091FF
:10D7F000990130919A0140919B0150919C01BC018B
:10D80000CD010E94DA783F932F938DE49BE09F93A4
:10D810008F93DF93CF93E0912B04F0912C04099523
:10D820008DB79EB70A968DBF12C086E00E94907198
:10D8300089E59BE09F938F93DF93CF93E0912B0437
:10D84000F0912C0409950F900F900F900F908091FC
:10D85000FE038823C1F086E00E9490718091FE0350
:10D8600099279F938F9380E69BE09F938F93DF93FD
:10D87000CF93E0912B04F0912C0409952DB73EB77E
:10D880002A5F3F4F2DBF80E10E9490718091F70188
:10D890009091F8016CE370E00E9491789F938F93D0
:10D8A0008091F7019091F8016CE370E00E9491780B
:10D8B0007F936F9380917008909171089F938F93DD
:10D8C0008BE69BE09F938F93C3E8D1E7DF93CF93E1
:10D8D000E0912B04F0912C040995809114062DB74A
:10D8E0003EB7265F3F4F2DBF80FF29C08AE10E94CF
:10D8F00090718091980199279F938F938091110344
:10D9000090911203A0911303B0911403BC01CD01B7
:10D9100024E630E040E050E00E94DA783F932F9315
:10D9200088E79BE09F938F93DF93CF93E0912B0445
:10D93000F0912C0409958DB79EB708968DBFDF91A5
:10D94000CF910895CF93DF9380E00E9490718091F2
:10D95000ED06992787FD90959F938F938091E5061B
:10D96000992787FD90959F938F938091DD06992746
:10D9700087FD90959F938F938091D506992787FD7A
:10D9800090959F938F938FE79BE09F938F93C3E82E
:10D99000D1E7DF93CF93E0912B04F0912C0409950C
:10D9A00080E10E9490712DB73EB7245F3F4F2DBF9D
:10D9B00080910D07992787FD90959F938F93809174
:10D9C0000507992787FD90959F938F938091FD067A
:10D9D000992787FD90959F938F938091F5069927BE
:10D9E00087FD90959F938F938FE89BE09F938F93F4
:10D9F000DF93CF93E0912B04F0912C040995809153
:10DA000006062DB73EB7245F3F4F2DBF853098F4F3
:10DA100080E10E9490718FE99BE09F938F93DF9349
:10DA2000CF93E0912B04F0912C0409950F900F9067
:10DA30000F900F9018C08730B0F488E10E94907169
:10DA40008FED90E09F938F9380EB9BE09F938F935C
:10DA5000DF93CF93E0912B04F0912C0409958DB7BF
:10DA60009EB706968DBFDF91CF9108950F931F93B8
:10DA700080E00E9490712AE030E080916C089091E3
:10DA80006D08B9010E9491789F938F9380916C08E3
:10DA900090916D08B9010E9491787F936F93809166
:10DAA0001D0190911E01B9010E94A5789F938F934B
:10DAB00080911D0190911E01B9010E94A5787F936C
:10DAC0006F9389EB9BE09F938F9303E811E71F937C
:10DAD0000F93E0912B04F0912C04099580E10E94B2
:10DAE00090718DB79EB70C968DBF80917008909104
:10DAF00071089F938F9380916E0890916F089F9308
:10DB00008F938CEC9BE09F938F931F930F93E091E7
:10DB10002B04F0912C0409958DB79EB708968DBF04
:10DB20001F910F9108950F931F93CF93DF938091CF
:10DB3000EC01C3E8D1E7882309F478C080E00E94B3
:10DB400090718091010899279F938F93809103088A
:10DB500099279F938F9388ED9BE09F938F938E01DE
:10DB6000DF93CF93E0912B04F0912C0409958DB7AE
:10DB70009EB708968DBF80910208833031F48CE007
:10DB80000E94907187EE9BE005C08CE00E9490712E
:10DB90008CEE9BE09F938F93DF93CF93E0912B04C8
:10DBA000F0912C0409950F900F900F900F90809199
:10DBB000000881FF12C08CE00E94907181EF9BE011
:10DBC0009F938F931F930F93E0912B04F0912C045C
:10DBD00009950F900F900F900F9080E10E94907127
:10DBE0008FED90E09F938F938091060890910708A6
:10DBF0009F938F9380910408909105086AE070E0EC
:10DC00000E9491787F936F9386EF9BE09F938F9311
:10DC100083E891E79F938F93E0912B04F0912C047C
:10DC200009958DB79EB70A968DBF12C082E00E94FB
:10DC3000907186E09CE09F938F93DF93CF93E09168
:10DC40002B04F0912C0409950F900F900F900F90DA
:10DC5000DF91CF911F910F910895CF93C82F2091FD
:10DC600013042093140499278F32910509F180330E
:10DC700091051CF44F97A1F02CC08F34910501F150
:10DC80008F38910531F5222319F481E090E038C0F6
:10DC900086E0289FF0011124E45DF44F849117C0C1
:10DCA00086E0289FF0011124E35DF44F84910FC0BA
:10DCB00086E0289FF0011124E25DF44F849107C0B3
:10DCC00086E0289FF0011124E15DF44F8491809358
:10DCD000130490911304809114049813C0E00E94DF
:10DCE00096719091130486E0989FF0011124E05DF5
:10DCF000F44F259134918C2FF901099580E090E043
:10DD0000CF91089510926D0810926C0810927108CE
:10DD10001092700810926F0810926E08109272089C
:10DD20008AE090E00E948E1690931604809315046A
:10DD30000895CF93DF9380911504909116040E946B
:10DD40009716882309F4AFC08091150490911604AA
:10DD50000A969093160480931504E0E0F0E09F018A
:10DD600090E05FEFAEECB6E04BE0ED018B8187FF1A
:10DD70000BC09F5F8D81E80FF11D8981280F311D38
:10DD80008E81851708F4582F4150189647FFEDCF24
:10DD900050937208232B41F520911B0430911C04F1
:10DDA00040911D0450911E04BB27A52F942F832F53
:10DDB00090931A0480931904AA27BB27281B390BB8
:10DDC0004A0B5B0BCF01AA27BB27280F391F4A1F1D
:10DDD0005B1F20931B0430931C0440931D0450933D
:10DDE0001E04E5E0F0E013C02091190430911A04FC
:10DDF0002E173F0718F4E21BF30B02C0E0E0F0E03F
:10DE0000892F9927880F991FE80FF91F3596F093EE
:10DE10006D08E0936C08EF3FF10578F480911D01E7
:10DE200090911E018E9F90018F9F300D9E9F300D0F
:10DE30001124C90164E670E013C0CF01969587955F
:10DE40009695879520911D0130911E01289FA00174
:10DE5000299F500D389F500D1124CA0169E170E0CF
:10DE60000E94917870936F0860936E082091170458
:10DE7000309118042E0F3F1F30931804209317047D
:10DE80005EE02131350778F080917008909171083B
:10DE90000196909371088093700820513E40309312
:10DEA000180420931704DF91CF91089500242227AE
:10DEB0003327442751E0BB27EE27FF27A0E1660F59
:10DEC000771F881F991F001C221F331F441F660FD6
:10DED000771F881F991F001C221F331F441F2AF41D
:10DEE000050E2B1F3E1F4F1F04C0051A2B0B3E0BA8
:10DEF0004F0B550FBB1FEE1F587F556047FD52500B
:10DF0000AA95E9F6E695B7955795E695B79557958D
:10DF1000852F9B2F08952227332741E0552768E05E
:10DF2000880F991F221F331F880F991F221F331F2D
:10DF30001AF4240F351F02C0241B350B440F551F44
:10DF4000487F456037FD42506A9551F75695479591
:10DF500056954795842F0895AA2797FF04C080956A
:10DF600090958A1F9A1F77FF04C0609570956A1F6D
:10DF70007A1F669F9001779FA001679F300D411D1A
:10DF80005A1F300D411D5A1F889FF001999F2E0F77
:10DF90003F1F401D511D899F300D411D5A1F300DDF
:10DFA000411D5A1FCA01B901112480CF4FB720E487
:10DFB00030E0F8948091C9008F778093C9008091F8
:10DFC000C9008F7B8093C9008091C9008F7D8093A9
:10DFD000C9005A9A52985B9A539A832F9927809333
:10DFE000CD002093CC008091C80082608093C8004F
:10DFF00088E18093C9008091CA008F778093CA001E
:10E000008091CA008F7B8093CA008091CA008F7D67
:10E010008093CA008091CA008F7E8093CA0080914D
:10E02000CA00877F8093CA008091C9008B7F80934C
:10E03000C9008091CA0084608093CA008091CA00A0
:10E0400082608093CA008091C80087FF03C08091DE
:10E05000CE00F9CF8091C90080688093C9004FBF7E
:10E0600008950F931F93CF93DF93482F4F5F89310C
:10E0700008F089C080912E07841710F440932E0772
:10E08000CB0183539B4268E170E00E94A578A42FE6
:10E09000BB27FD01EA0FFB1FE15DF84F80819181F5
:10E0A0009B01281B390BC90137FF03C0909581954F
:10E0B0009F4F069794F480911F03883C30F4809121
:10E0C0001F03865F80931F0308C088EC80931F03A3
:10E0D00080916F008F7D80936F00FD01EA0FFB1F21
:10E0E000E15DF84F808191819C01220F331F280F41
:10E0F000391F260F371F37FF02C02D5F3F4FE90141
:10E10000D595C795D595C795CB0101968C179D07D9
:10E1100014F4219706C061507040C617D7070CF45D
:10E12000219680911F03843BD8F08D010A0F1B1F9D
:10E13000F801E15DF84F80819181FE01E81BF90B48
:10E14000CF0163E070E00E94A578CB01880F991F92
:10E15000860F971F0D59184FF8019183808307C0D0
:10E16000AA0FBB1FAD59B84F11961C921E92E42FF7
:10E17000FF27EE0FFF1FE15DF84FD183C0834430CE
:10E1800011F410929301DF91CF911F910F91089597
:10E19000CF93DF9320917308822F9927807F90700F
:10E1A000409709F06CC02F3109F046C08091740887
:10E1B000809323042091760820932504809177088A
:10E1C00080932404822F99279093300780932F0700
:10E1D000222309F054C080910806282F3327220FEC
:10E1E000331FF901ED59F84F118210828091090611
:10E1F000A82FBB27AA0FBB1FFD01ED59F84F1182B5
:10E20000108280910B06E82FFF27EE0FFF1FCF0132
:10E210008D59984FEC0119821882215D384FE90120
:10E2200019821882A15DB84F11961C921E92E15D71
:10E23000F84F1182108223C0C22FCF70CA30F8F479
:10E240008091740880939D088091750880939C0844
:10E250008091760880939F088091770880939E082C
:10E2600060919C0870919D088C2F0E943170609184
:10E270009E0870919F088C2F8F5F0E943170DF91F4
:10E28000CF910895CF93C82F8F3F49F480912604F2
:10E290008F3F29F4109228041092270432C0209155
:10E2A0002804222339F4CF3111F485E001C084E041
:10E2B0008093290480912904909127048217A0F467
:10E2C000892F8095809327048F3F19F48EEF8093D8
:10E2D000270480912704C81711F40E94C870109277
:10E2E0002804109227040BC0E22FFF27ED58F74FA8
:10E2F000C0832F5F209328049C0F90932704C09322
:10E300002604CF91089590912204933240F4E92F8E
:10E31000FF27E758F74F80839F5F9093220408956B
:10E32000833218F48D5F80932204089590E2ECE725
:10E33000F8E08FE19193815087FFFCCF0895CF9350
:10E34000CFB723E031E0F8948091C9008F778093B4
:10E35000C9008091C9008F7B8093C9008091C9005A
:10E360008F7D8093C9005A9A52985B9A539A832F53
:10E3700099278093CD002093CC008091C8008260C3
:10E380008093C80088E18093C9008091CA008F778C
:10E390008093CA008091CA008F7B8093CA008091CD
:10E3A000CA0080628093CA008091CA008061809315
:10E3B000CA008091CA0088608093CA008091C90019
:10E3C00084608093C9008091CA0084608093CA00F1
:10E3D0008091CA0082608093CA008091C80087FF44
:10E3E00003C08091CE00F9CF8091C90080688093EE
:10E3F000C9008091C90080648093C9000E94967111
:10E40000CFBFCF910895282F99278F709070892BB7
:10E4100031F4209580912104822B8093210408956A
:10E420008091F301882309F441C08091EB0285FFBC
:10E430000AC082E98093790883E280937A0885E5AF
:10E4400080937B0802C0109279088091F4018F308C
:10E4500071F4809121040E942D6E882341F081E99E
:10E460008093790880937A0881E380937B081092E7
:10E47000F3018091C80085FFFCCF8091C9008F7E99
:10E480008093C9008091C9008E7F8093C9008091DC
:10E490007908882311F48EEF01C08EE78093CE00B7
:10E4A000809121048093F4011092210408951F9219
:10E4B0000F920FB60F9211248F939F93EF93FF93B8
:10E4C0009091F301992309F040C080912A04882398
:10E4D00061F480917908882311F483E003C08139C5
:10E4E00099F481E080932A040FC0833099F48091DD
:10E4F0007908882349F0909379088091C9008E7F2C
:10E500008093C9008EEF1EC08091C9008160809306
:10E51000C9000EC0833261F48091C9008E7F809360
:10E52000C9008FEF8093CE0081E08093F30114C087
:10E5300080912A04E82FFF27E758F74F8F5F8093D9
:10E540002A0480818093CE0007C010922A04809113
:10E55000C90080618093C900FF91EF919F918F91D5
:10E560000F900FBE0F901F901895EF92FF920F9390
:10E570001F93CF93DF937C018B01EA01452B39F088
:10E58000F80181918F01F70109952197C9F7E6E01C
:10E59000CDB7DEB70C941D79EF92FF920F931F93C6
:10E5A000CF93DF937C018B01EA01452B41F0F80109
:10E5B0000F5F1F4F8491F70109952197C1F7E6E09E
:10E5C000CDB7DEB70C941D790F931F93CF938C01B9
:10E5D000C62F161634F480E2F8010995C1501C16B6
:10E5E000D4F3CF911F910F9108950F931F93CF9361
:10E5F0008C01C62F161634F480E3F8010995C1503A
:10E600001C16D4F3CF911F910F910895A5E3B0E0AC
:10E61000ECE0F3E70C94F5782E96EEADFFAD2E9777
:10E6200088249924540180912004882321F42C9675
:10E630001FAE1EAE2C975EE4452E512C4C0E5D1E77
:10E640006F01B60105C0153239F00894C11CD11C08
:10E65000F60114911123B9F7A601461B570B31F0AF
:10E660002C968EAD9FAD2C970E94CC72112309F48D
:10E670006AC20894C11CD11CFF24FDA6FCA64FEF62
:10E68000E42EF9A6F6010894C11CD11C149115378B
:10E6900021F0812F80628837B1F4F0FE0AC0F201C8
:10E6A00024E030E0420E531E80809180A280B3802F
:10E6B0000AC0F20142E050E0440E551E8081918173
:10E6C0004C01AA24BB24103221F489A58823D1F659
:10E6D0001DC0133219F458E0F52AD4CF1A3211F0C4
:10E6E0001D3291F41A3259F4F20182E090E0480EA2
:10E6F000591EE081ECA7EE232CF6E195ECA790E102
:10E70000F92AAFEDFA22BECF1B3211F419A7BACF06
:10E710001E32C1F5F6010894C11CD11C14911A32A5
:10E7200079F4F20122E030E0420E531E4081518123
:10E730003FEF4F3F530714F44FEF5FEFE42EA2CFAC
:10E7400040E050E0812F80538A30A0F4CA0133E0CA
:10E75000880F991F3A95E1F7840F951F480F591FAD
:10E76000410F511D40535040F6010894C11CD11C6B
:10E770001491E8CF8FEF4F3F580714F44FEF5FEF3E
:10E78000E42E85CF103329F4F4FC7CCF90E2F92AF3
:10E7900079CF812F81538930D8F440E050E0CA010D
:10E7A00023E0880F991F2A95E1F7840F951F480FE2
:10E7B000591F410F511D40535040F6010894C11C90
:10E7C000D11C1491812F80538A3048F34CA75FCF1E
:10E7D000183619F4A4E0FA2A55CF1C3619F4B1E022
:10E7E000FB2A50CF133661F43E010894611C711C62
:10E7F000F20122E030E0420E531E808189833CC149
:10E80000143421F0143611F0193651F5143411F482
:10E8100031E0F32AF0FE0AC0F20144E050E0440E79
:10E82000551E80809180A280B3800CC0F20182E0EE
:10E8300090E0480E591E808191814C01AA2497FCDA
:10E84000A094BA2CB7FE0AC0B094A094909480947F
:10E85000811C911CA11CB11C8DE289A70AE06FC02C
:10E860001F3411F01F3631F41F3411F491E0F92AEE
:10E8700008E064C0103779F4F201A2E0B0E04A0E7B
:10E880005B1E808191814C01AA24BB2400E1B0E48D
:10E89000FB2A18E753C01337C1F5F20122E030E03C
:10E8A000420E531E608071806114710489F43E0130
:10E8B0000894611C711C88E289838EE6F3018183D0
:10E8C00085E78B838CE68C838D8389E28E831F8220
:10E8D000E7FC13C08E2D992787FD9095AC0160E071
:10E8E00070E0C3010E94A177009729F0382E3618F6
:10E8F000E3140CF0C3C03E2CC1C0F3010190002012
:10E90000E9F731973E2E3618B9C0153511F0153795
:10E9100031F4153511F4F1E0FF2A0AE00FC0183583
:10E9200019F0183709F0A0C000E1F3FE07C0811408
:10E930009104A104B10411F020E4F22A19A6EDA675
:10E94000E7FC02C03FEDF32289E2682E712C6C0EC9
:10E950007D1E81149104A104B10421F44DA544232A
:10E9600009F47BC0802F9927AA27BB278EA79FA7D2
:10E97000A8ABB9AB202E332490E0891690E099061D
:10E9800091E0A90690E0B90648F0C501B4012EA5B2
:10E990003FA548A959A90E94B87817C0AFEF8A16B9
:10E9A0009104A104B10449F040F0C401B1010E94F6
:10E9B00091789B014427552708C0882D602F0E941D
:10E9C0008578282F3327442755272AAB3BAB4CAB00
:10E9D0005DAB0A3059F48AA9880F880F880F9AA96D
:10E9E000990F890F382D381B832F10C0003139F44F
:10E9F0008AA98295807F482D481B842F07C08AA949
:10EA0000880F880F880F582D581B852F90E02EA552
:10EA10003FA548A959A982169306A406B50608F091
:10EA200091E08AA89BA8ACA8BDA88A3010F4805DAC
:10EA300004C0895A183509F48F7DD3018E933D01A6
:10EA4000992309F099CF083041F4F3FE06C08033D2
:10EA500021F080E3FD0182933F01CE010196382E23
:10EA60003618F8E23F0E0BC0112309F46CC03E01CA
:10EA70000894611C711C1983B1E03B2E19A6032D6B
:10EA80002DA4231827FC222489A5882311F00F5FC9
:10EA900002C0F6FC0E5F020DEF2CFF24C70180734D
:10EAA0009070892B49F48CA5801B682F2C968EAD15
:10EAB0009FAD2C970E94E47289A5882331F041E034
:10EAC00050E0BE01675D7F4F0AC0E6FE0EC080E3E6
:10EAD0008AA71BA742E050E0BE01665D7F4F2C96DF
:10EAE0008EAD9FAD2C970E94B572C7018073907058
:10EAF000809749F48CA5801B682F2C968EAD9FAD16
:10EB00002C970E94F572622D2C968EAD9FAD2C979E
:10EB10000E94F572832D992787FD9095AC01B30172
:10EB20002C968EAD9FAD2C970E94B572E4FE89CDD8
:10EB30002CA5201B2CA7622F2C968EAD9FAD2C9759
:10EB40000E94E4727ECDE2E1CB5C0C9411792FB788
:10EB500040E0F894E0E0F0E081E280935700949187
:10EB6000E2E0F0E0809357003491E4E0F0E080933D
:10EB7000570084912FBF9E3199F4363941F4893082
:10EB800011F441E00DC08A3059F442E009C0373930
:10EB900039F4863011F443E003C0853009F444E0D1
:10EBA000842F992708959FB7F8948091C900877F93
:10EBB0008093C9008091C9008F7E8093C9008091A5
:10EBC000C9008F778093C9008091C9008F7B8093A3
:10EBD000C9008091C9008F7D8093C90052985A9ACC
:10EBE00053985B9A9FBF08951F93CF93DF93182F7D
:10EBF00080912004882309F48DC08091F2011817B8
:10EC000009F488C080911F04882321F40E94A7750D
:10EC100080931F048FEF9CE09F938F93C7E6D2E110
:10EC2000DF93CF93E0912B04F0912C0409950F9082
:10EC30000F900F900F90812F99278230910501F14D
:10EC4000833091052CF4009761F0019769F024C09E
:10EC500084309105D9F084309105ACF00597C9F066
:10EC60001BC08FEE9CE002C08DED9CE09F938F93C4
:10EC7000DF93CF93E0912B04F0912C04099518C0F9
:10EC800084EC9CE0F3CF81EA9CE0F0CF83E99CE048
:10EC9000EDCF8BE89CE0EACF8CE09DE09F938F93D3
:10ECA000DF93CF93E0912B04F0912C04099510E0B1
:10ECB0000F900F900F900F9080911F04843011F0EF
:10ECC000823099F40E94D375812F8150833018F4DB
:10ECD0000E9405691DC0143019F40E949F7118C06C
:10ECE0001530B1F40E94D66F13C0112389F082E26F
:10ECF0009DE09F938F9387E692E19F938F93E0919E
:10ED00002B04F0912C0409950F900F900F900F9009
:10ED10001093F201DF91CF911F9108950F931F93EC
:10ED200081E0809320044091F101EBE3FCE020E0DE
:10ED300030E05FE4849199272F5F3F4F829FB001BD
:10ED4000839F700D929F700D11244627515031966C
:10ED500057FFF0CF4093F101E3E1FCE020E030E029
:10ED600057E2849199272F5F3F4F829FB001839F85
:10ED7000700D929F700D112446275150319657FF08
:10ED8000F0CF4093F10180911F04882321F40E9469
:10ED9000A77580931F048091F101833459F088E1B5
:10EDA00090E029E20FB6F894A895809360000FBE1A
:10EDB0002093600086E093E790932C0480932B04CB
:10EDC0008DE39DE09F938F9307E612E11F930F93CE
:10EDD000E0912B04F0912C0409950F900F900F9067
:10EDE0000F9086E690E09F938F9380E590E09F934D
:10EDF0008F931F921F92809102016AE00E94857892
:10EE0000892F99279F938F93809102010E94857883
:10EE100099279F938F9383E69DE09F938F931F93F2
:10EE20000F93E0912B04F0912C0409958BE39CE067
:10EE30009F938F931F930F93E0912B04F0912C04D9
:10EE4000099583E19CE09F938F931F930F93E0912B
:10EE50002B04F0912C0409958DB79EB746968DBF73
:10EE600087E99DE09F938F931F930F93E0912B046D
:10EE7000F0912C04099583EC8093810080916F00C0
:10EE8000806280936F000F900F900F900F901F91F2
:10EE90000F91089580912004882361F08091F20100
:10EEA000843011F40E9410728091F101833411F0CA
:10EEB0001092200408951F920F920FB60F92112402
:10EEC0002F933F934F935F936F937F938F939F9372
:10EED000AF93BF93EF93FF932091CE009091F201F7
:10EEE000892F8150833020F4822F0E94126A0BC038
:10EEF000943021F4822F0E94037205C0953019F4DA
:10EF0000822F0E944271FF91EF91BF91AF919F912B
:10EF10008F917F916F915F914F913F912F910F90C2
:10EF20000FBE0F901F901895FB01DC0140FF05C03C
:10EF300002C005900D9205900D9242505040C8F7C6
:10EF40000895FC014150504030F001900616D1F771
:10EF50003197CF0108958827992708955058192E81
:10EF600084D001D06AC0BA17620773078407950777
:10EF7000B1F188F40EF410940B2EBA2FA02D062EAA
:10EF8000622F202D072E732F302D082E842F402D19
:10EF9000092E952F502DFF275523B9F0591B49F005
:10EFA000573E98F0469537952795A795F04053958D
:10EFB000C9F776F0BA0F621F731F841F30F487956C
:10EFC00077956795B795F040939517FA0F2E0895AA
:10EFD000BF1BBB27BA0B620B730B840BF6CFDEF69D
:10EFE00070C097FB4ED09F3738F0FEE9F91B982F81
:10EFF000872F762F6B2F05C061C0969587957795E3
:10F000006795F150D0F73EF4909580957095619595
:10F010007F4F8F4F9F4F0895E89403C097FB0EF4E6
:10F02000F3DFB62F672F782F892F9EE9002405C0C4
:10F030009A95BB0F661F771F881F11249923A1F093
:10F040008823B2F79F3F59F0BB0F48F421F400200A
:10F0500011F460FF04C06F5F7F4F8F4F9F4F881F79
:10F060009795879597F9089529C0052E092607FADF
:10F07000440F551F5F3F79F0AA27A51708F051E00C
:10F080004795880F991F9F3F31F0BB27B91708F0AC
:10F0900091E0879508959F919F91112414C097FB4B
:10F0A000880F991F9F3F31F0BB27B91708F091E0F7
:10F0B000879508959F919F91112405C06627772712
:10F0C0008827992708959FEF80EC0895629FD001CB
:10F0D000739FF001829FE00DF11D649FE00DF11D13
:10F0E000929FF00D839FF00D749FF00D659FF00DC2
:10F0F0009927729FB00DE11DF91F639FB00DE11DAF
:10F10000F91FBD01CF0111240895991B79E004C0B6
:10F11000991F961708F0961B881F7A95C9F7809556
:10F120000895AA1BBB1B51E107C0AA1FBB1FA6174E
:10F13000B70710F0A61BB70B881F991F5A95A9F7A0
:10F1400080959095BC01CD01089597FB092E072667
:10F150000AD077FD04D0E5DF06D000201AF47095C0
:10F1600061957F4F0895F6F7909581959F4F08958B
:10F17000A1E21A2EAA1BBB1BFD010DC0AA1FBB1FBB
:10F18000EE1FFF1FA217B307E407F50720F0A21B2D
:10F19000B30BE40BF50B661F771F881F991F1A949A
:10F1A00069F760957095809590959B01AC01BD01C4
:10F1B000CF01089597FB092E05260ED057FD04D0E8
:10F1C000D7DF0AD0001C38F4509540953095219532
:10F1D0003F4F4F4F5F4F0895F6F79095809570958C
:10F1E00061957F4F8F4F9F4F08952F923F924F927F
:10F1F0005F926F927F928F929F92AF92BF92CF92C7
:10F20000DF92EF92FF920F931F93CF93DF93CDB7CF
:10F21000DEB7CA1BDB0B0FB6F894DEBF0FBECDBF47
:10F2200009942A88398848885F846E847D848C8418
:10F230009B84AA84B984C884DF80EE80FD800C8121
:10F240001B81AA81B981CE0FD11D0FB6F894DEBF04
:10F250000FBECDBFED010895EE0FFF1F0590F49195
:10F26000E02D0994F999FECFB2BDA1BDF89A11968F
:10F2700000B40895F7DF01921A94E1F70895F2DFE0
:10F28000E02DF0DFF02D0895F999FECFB2BDA1BDBC
:10F2900000BC11960FB6F894FA9AF99A0FBE089529
:10F2A000F3DF012CF1DF112408950190EDDF1A94B2
:04F2B000E1F70895E5
:10F2B4005E010A010164FF01FFFF01FC01FC010181
:10F2C400737373FF03007D0000C409C40964001153
:10F2D40048656C6C6F20576F726C6400000000000E
:10F2E400000000000000000000000000000000001A
:10F2F400000000000000000000000000000000000A
:10F3040000000000000000000000000000000000F9
:10F3140000000000000000000000000000000000E9
:10F3240053706F727400004E6F726D616C00004216
:10F334006567696E6E6572000051756164726F0075
:10F344000064000101000300200B050000ECFF64D1
:10F3540040415A4664640A02969696960840403A9A
:10F3640010FB30380190D0030090D00300F40178F2
:10F3740000FF0364000204060708080807060402E5
:10F3840000FEFCFAF9F8F8F8F9FAFCFE00020406AB
:10F394000708080B0A0D0B0C0E0B0F10FA200101C5
:06F3A4000170FF010F00E3
:00000001FF
